:020000040000FA
:040000006FD00400B9
:101000006F00907E00000000000000009020002093
:10101000AA220020A9BDF9F56C23002000000000E1
:10102000000000006C230020902000200000000041
:101030000000000090200020000000009020002010
:101040000000000090200020902000209020002030
:101050009020002090200020582F00209424002071
:101060000000000090200020902000201E2400207E
:1010700090200020D22300209020002090200020EB
:101080009020002090200020902000209020002020
:101090009020002001A04111B7170040985F3AC688
:1010A000945F3247E39CE6FE3245410182800111A4
:1010B00013078008F337078093F787083EC20100C3
:1010C0000100B7170040930570052380B70413068D
:1010D00080FA2380C7040100010083C6B70493F699
:1010E000F60DA385D704238007049246F3A6068055
:1010F0000100010093760502D5CEF336078093F602
:10110000860836C4010001002380B7042380C70489
:1011100001000100B70614007D89558D88C70100C4
:1011200001000100010023800704A246F3A6068007
:101130000100010073370780137787083AC6010062
:1011400001002380B7042380C704010001000100CF
:1011500001003727004093061005A303D7802380A2
:101160000704B247F3A70780010001009307800836
:10117000F3B7078093F787083ECE01000100B71749
:101180000040130770052380E704130780FA2380CB
:10119000E7040100010003C7B70413670708A3852C
:1011A000E70423800704F247F3A70780010001004A
:1011B0000561828093760504BDC6F336078093F6F9
:1011C000860836C8010001002380B7042380C704C5
:1011D00001000100B7061400938606047D89558D31
:1011E00088C7010001000100010023800704C246F6
:1011F000F3A6068001000100733707801377870884
:101200003ACA010001002380B7042380C70401000B
:1012100001003727004093062005A303D7802380D1
:101220000704D24781B773370780137787083ACC12
:10123000010001002380B7042380C70401000100DE
:1012400098471367070C98C723800704E24719BF24
:101250000111814601468145114506CE97000000E7
:10126000E780605893078008F3B7078093F78708F3
:101270003EC601000100B717004013077005238028
:10128000E704130780FA2380E7040100010003C785
:101290006704136717002383E70423800704B2471A
:1012A000F3A7078001000100F2400561828041112F
:1012B000814601468145114597000000E780A05214
:1012C00013078008F337078093F787083EC40100AF
:1012D0000100B7170040130670052380C70493066A
:1012E00080FA2380D70401000100FD552396B70240
:1012F00023800704A245F3A5058001000100733790
:101300000780137787083AC6010001002380C704CD
:101310002380D7040100010003C767041367170087
:101320002383E70423800704B247F3A70780010063
:10133000010001A0B1473305F50201007D1575FDDF
:101340008280411122C426C206C6AA8401446317C2
:101350009400B24022449244410182800504130566
:10136000803E420497000000E78000FD4180C5B741
:101370009305000273A04580824573901534924016
:101380002242B2424243D2436244F2440255925551
:101390002256B2564257D2576258F25806499649D9
:1013A000264AB64A464BD64B664CF64C065D965DD1
:1013B000265EB65E465FD65F09617300203041113C
:1013C000B7170040985F3AC6945F3247E39CE6FE49
:1013D000324541018280B71700401307000323887C
:1013E000E702854717170000232EF74873002030C7
:1013F000411122C42D6426C24AC006C637190040D6
:101400001304A4AAB704002023208900976000E0F9
:10141000E780C04C9C408297976000E0E780004CDA
:10142000E5B737370040834747009146BD8B639E41
:10143000D702B73600401306F00F973500009385AA
:10144000E5209737000083D7673003C7A6001377DE
:10145000F70F1DE3B7E70400BC4F09468945171590
:1014600000000345A5F8829731A099466394D70000
:10147000834757007300203003C786001377F70FA8
:10148000E365F6FC13851700AE9717380000231F9D
:10149000A82A2380E70075B7B787004003C7670015
:1014A000098B6309071003C77700930600031377BE
:1014B0000703630DD708173800000348387C173638
:1014C00000001306A6780547B30606012380E60050
:1014D00083C577001737000013074779429793F5C4
:1014E000F50F2300B70003C58700973500009385EB
:1014F000E576C2951375F50F2380A5000347070015
:1015000089451377F703630CB70C63E7E50A6306B5
:10151000071A8545630CB7129737000083C7177603
:101520003307F600034707001377F70F19CB85073A
:1015300093F7F70F3D476363F71A17370000A30FC0
:10154000F772B787004009472383E700B787004059
:1015500083C77700E207E18763DE0704973700005F
:1015600083C7D771173700001307476E3E9785462C
:101570002300D700173700001307476F3E979306E5
:1015800000032300D700173700001307276D3E978D
:10159000A14685072300D70093F7F70F3D47636403
:1015A000F71417370000A30BF76CB7870040094703
:1015B0002383E70073002030930610026300D70EE8
:1015C000930620026305D70693060002E316D7F4BC
:1015D00003C727021377C70F13672700D5A803C7D0
:1015E00067001377070465CB03C7A702173800000D
:1015F00013084847173500001305853E13470708B1
:101600002385E70203C7A7021377370F1367870005
:101610002385E702814713070004B305F5008C41D9
:10162000B306F80091078CC2E399E7FEF5B503C74E
:10163000A702134707042385E70203C7A70213770E
:10164000C70F136727002385E702F9B503C76700B3
:101650001377070449C303C767021738000013084C
:101660002834173500001305652B1347070823831B
:10167000E70203C767021377370F136787002383D7
:10168000E702814713070004B305F5008C41B30658
:10169000F80091078CC2E399E7FEBDBD03C767025E
:1016A000134707042383E70203C767021377C70FB3
:1016B000136727002383E70285B503C76700137705
:1016C000070411CB03C727021377370F136787006F
:1016D0002381E70291B5238006003DBD97370000C6
:1016E000A38E0758B9BD97370000A389075875BD69
:1016F0002303048015472303E48001002302A48010
:10170000828083076480E3CE07FE23030480828007
:1017100083076480E3CE07FE03454480828083070D
:101720006480E3CE07FE2302A4808280411126C498
:101730004AC24EC006C61377F50BAD47AA892E895B
:101740009544630CF700194597000000E78080FA84
:1017500097000000E78020FB8D444E859700000035
:10176000E78040F9FD59FD1463983401B240A2446A
:101770001249824941018280135509011375F50F01
:1017800097000000E780E0F92209F1BF011126CCA3
:1017900006CEB704080097000000E780C0F61545A4
:1017A00097000000E78000F597000000E78080F6D2
:1017B00097000000E78000F62AC697000000E78047
:1017C00080F432459377150089EB13651500137586
:1017D000F50FF240E24405618280FD14E9F0014515
:1017E000CDBF397126DC4ADA4ED852D656D45AD2F9
:1017F0005ED006DE62CE66CCB7E700E07D5783AAF6
:10180000070022C603AA470023A0E71823A2E7186F
:10181000B7170040130770052380E704130780FA09
:101820002380E70483C74704930B75FFB684E20760
:1018300093FBFB0F8546AA892E8B32893724004003
:10184000E187015763FA76016308D50089461307DB
:1018500000026313D5000157D98F93F7F70FB71C18
:1018600000402382FC0411472303E4801305F00F9A
:1018700097000000E78000E8094C97000000E7802F
:1018800080E863657C15B7050700DA9537870700A0
:10189000795563FEE504B3879500636AF704370B57
:1018A0000800A94733EB65016395F90881E8814495
:1018B00097000000E78020E5268515A8DA85094510
:1018C00097000000E780C0E605090345F9FFFD1415
:1018D000050B97000000E780C0E481C49377FB0FFD
:1018E000E5F797000000E780A0EA69F17D55B7179A
:1018F0000040130770052380E704130780FA238054
:10190000E70403C74704418B2382E704F250B7E79B
:1019100000E023A0571123A24711E2543244525948
:10192000C259325AA25A125B825B724CE24C21615C
:101930008280A547639BF90685691309F00FB306FA
:101940009900B3742B01B6941349F9FFB37499004D
:10195000856B33796901416B9387F9FFB3F72701F1
:1019600099E363FC340193D94900C147E3E637FFAB
:101970003DBF0569C1697D19D9B71305800D63881D
:101980006901130500026384790113051008CA85F3
:1019900097000000E780C0D997000000E78040DF93
:1019A00031D54E99B38434416DBFDA852D4597000A
:1019B0000000E780E0D7CA94E30B99EE0509970091
:1019C0000000E78020D5A30FA9FEFDB79387F9FF9C
:1019D00093F7F70F636DFC0C83C71C0413073008E3
:1019E0006315F706370708006361EB06B3079B0032
:1019F000B706100063FBD704334BEB0089476399AC
:101A0000F9068980D549E38404EADA850945970017
:101A10000000E780E0D111090327C9FF9147232087
:101A2000E48003076480E34E07FE23033481FD173F
:101A3000EDFBFD14110B81C49377FB0FE9FF9700B9
:101A40000000E780E0D461F155B5B717004003C747
:101A50005704B70708001377070219E3B787070091
:101A60007955E376FBE833079B00E3F9E7F841B5E6
:101A70008547E380F9F0DA852D4597000000E7807F
:101A800020CB9389F4FFE38404E297000000E78011
:101A900060C893F7390091EB83260480032709007F
:101AA00093074900E396E6E03E89CE84D9BFB54767
:101AB0006399F9001305900B97000000E78080C33D
:101AC000FDB3B1471305B00AE388F9FE9947639760
:101AD000F904B7050800B365BB002D459700000069
:101AE000E78000C581448D4BA14997000000E78045
:101AF00060C263967401832704802320F900850463
:101B0000E39534FF8327048013172B0163550700E7
:101B10002312F90069BB2322F90051BB9D47639F43
:101B2000F90281451305B00497000000E78040C02A
:101B3000BD442320090023220900FD59970000001D
:101B4000E78040BD93F77400CA9703C70700FD14F0
:101B5000398D2380A700E39334FF91BBA14763979E
:101B6000F90697000000E780A0C28144630D0B00D6
:101B70008D479304C0036308FB00930400056304CE
:101B80008B01930440041375C507E30295D21945F0
:101B900097000000E78000B697000000E780A0B63D
:101BA000054597000000E780E0B426859700000017
:101BB000E78020B7094597000000E78080B69700CE
:101BC0000000E780E0BCE31405CE0DB39147639FAE
:101BD000F9001305600697000000E780A0B19700A8
:101BE0000000E78040B213059009F9B5E38109CC04
:101BF000F1547DB9BD6601471736000013068625EE
:101C0000938606A685458347060093F7F70F91C391
:101C100082800507E3F9E6FE97370000238CB722A0
:101C2000DDB77D166206618693178601E18763D46E
:101C3000070001458280931726003307F500AE9711
:101C400018439C4363E7E7007D16E37FF7FC7D556F
:101C5000828005458280FD15E205E18513978501A7
:101C6000618793F7F50F63480700FD15139725006B
:101C70002A97584365D713851700620561858280CE
:101C80003308B5021C4283A80600B335B502C297DB
:101C900033B50701AE98469585486367B5006394F0
:101CA000A50063E3070181480C43C6950CC388C2B5
:101CB0001CC2828081471397870161876343B70005
:101CC0008280139727002A97232007008507E5B70E
:101CD0008147014793968701E18663C5B6001335B6
:101CE0001700828093962700AA9694428507558F05
:101CF000D5B793D755408A07AA979C430545331516
:101D0000B5007D8D828017F3FFDFE702833D2A84D3
:101D100097000000E78060F405C5931725003E9406
:101D20000327C4FF814711EB7D1516053E9542053B
:101D3000418517F3FFDF6700033D05838507E5B79E
:101D40000145C5BF81471397870161876343C7007A
:101D5000828013972700B386E50094422A9785076F
:101D600014C3D5B77D1662066186014793178601B5
:101D7000E18763D50700133517008280931726008B
:101D8000B306F500AE9794429C437D16B58F5D8FE8
:101D9000F1BF8A05AA9501476363B500828083A6D7
:101DA000C5FFF11593D71600D98F9CC11397F60183
:101DB000E5B72A830148014701456343D700828084
:101DC000B387050183A80700B30706019C43C697A4
:101DD000AA976384F80033B517010507B308030118
:101DE000620723A0F80061871108C1BF2A83014759
:101DF0008147014563C3D70082803388E50083288B
:101E00000800330EE600032E0E003388A840330886
:101E1000C8416384080133B508018507B308E300AE
:101E2000E20723A00801E1871107E9B717F3FFDFF5
:101E3000E702232B0111B286B2842E86AA850A8579
:101E400097000000E780C0FA2A84A6850A859700DB
:101E50000000E78020E833348000060413351500C5
:101E6000018D056117F3FFDF6700E32917F3FFDF3B
:101E7000E702A3244111AA89AE8A328BB68402C23A
:101E800002C402C60144131C8401135C8C416349E3
:101E90009C02939B1400FD1B0549138CF4FFF15C1D
:101EA00033048901620461846340740792478E049D
:101EB000CE9423AEF4FE410117F3FFDF67006323E6
:101EC00013192400B30B2B01014A93172A00D6974C
:101ED00083A50B0088437800340050009700000071
:101EE000E78040DA050A93178A01E187F11BE35E78
:101EF000FCFC92474E9905042320F900A2473EC2FC
:101F0000B24702C63EC441B7131A8901135A8A4127
:101F1000131D240093178A01E18763CF970092472E
:101F20000A044E941CC0A24705091379F90F3EC25A
:101F3000B24702C63EC4ADB7B3079A0313152A00D1
:101F400056950841780034005000050AEA97DA9760
:101F50008C4397000000E780E0D26DBF197106C284
:101F600012C416C61AC81ECA22CC26CE2AD02ED219
:101F700032D436D63AD83EDA42DC46DECAC0CEC2C9
:101F8000D2C4D6C6DAC8DECAE2CCE6CEEAD0EED2F9
:101F9000F2D4F6D6FAD8FEDA971500009385058EAE
:101FA0008841E700050092402242B2424243D243B8
:101FB0006244F244025592552256B2564257D257C5
:101FC0006258F25806499649264AB64A464BD64BBD
:101FD000664CF64C065D965D265EB65E465FD65F45
:101FE0000961730020300000972100209381810156
:101FF000175100201301018117F5FFFF1305C500DC
:102000009705002093850500171600201306C6FDCE
:1020100063FAC5008322050023A055001105910530
:10202000E3EAC5FE170502001305051F97150020FA
:102030009385C5FB171600201306C66763FAC50013
:102040008322050023A0550011059105E3EAC5FE92
:102050001715002013050566974500209385852BED
:102060006377B500232005001105E36DB5FEFD4241
:10207000739002BC8D4273904280B722000093821D
:10208000828873900230970200209382A2F793E235
:102090003200739052309752000093828296739070
:1020A00012346FB0F47573002030397101436EC67D
:1020B00019A0397141536AC866CA62CC5ECE19A0B4
:1020C000397101535AD056D252D44ED64AD826DA54
:1020D00022DC06DE33016140828241114AC026C201
:1020E00022C406C68282B24D4101024D924C224C5E
:1020F000B24B4101024B924A224AB2494101024984
:1021000092442244B240410182803D432A87637356
:10211000C3029377F700BDEFADE5937606FF3D8AE6
:10212000BA960CC34CC30CC74CC74107E36BD7FE30
:1021300011E28280B306C3408A0697020000969699
:102140006780A6002307B700A306B7002306B700E1
:10215000A305B7002305B700A304B7002304B70005
:10216000A303B7002303B700A302B7002302B700FD
:10217000A301B7002301B700A300B7002300B700F5
:10218000828093F5F50F93968500D58D9396050182
:10219000D58D61B7939627009702000096968682A8
:1021A000E78086FA9680C1171D8F3E96E374C3F8C8
:1021B000A5B73367B500FD530D8B79E7B7877F7FF0
:1021C0009387F7F710419441B372F6003363F6003A
:1021D000BE92B3E262006397720C6318D606504158
:1021E000D441B372F6003363F600BE92B3E26200EC
:1021F0006398720A631BD60410459445B372F600C7
:102200003363F600BE92B3E262006391720A631E0A
:10221000D6025045D445B372F6003363F600BE9241
:10222000B3E26200639A72086311D60210499449BE
:10223000B372F6003363F600BE92B3E262006393BA
:1022400072085105D105E30FD6F6131706019397CF
:102250000601631CF7001357060193D706013305E7
:10226000F7409375F50F91E982804183C18333056F
:10227000F7409375F50F91E182801377F70F93F78D
:10228000F70F3305F74082800346050083C605003B
:10229000050585056313D60065FA3305D6408280AF
:1022A00011059105E312D6FE014582802105A105A5
:1022B000E31CD6FC014582803105B105E316D6FC4E
:1022C000014582804105C105E310D6FC01458280AD
:1022D000B717004003C777051377E70FA38BE70411
:1022E000130700F8A38DE7043D47238CE704130789
:1022F0005003A38CE70403C7A7051377D70F238DDB
:10230000E7048280B717004003C7E7020D89411137
:102310001377C70F498F93068008F3B6068093F6AC
:10232000860836C601000100930670052380D70495
:10233000930680FA2380D704010001002387E70277
:1023400023800704B247F3A7078001000100410181
:10235000828041112A83014E930E407E130F001993
:10236000930F400663E56E129308001913034006AD
:10237000B3781503854E0D4FA14F337365020D8958
:102380001335150063EFBE121308F6FF79467298F5
:102390004208135808013307C70213D61700BE07B7
:1023A00032976146B3F6C60213068070B386C60242
:1023B0003697A166F58F42075D8FB716004083C739
:1023C000F60293F70708A303F1000346710083C7E1
:1023D000F60293F70708E394C7FE83477100B71628
:1023E000004093F7F70F6388071293078008F3B74D
:1023F000078093F787083EC401000100B71700402B
:10240000930670052380D704930680FA2380D704AF
:102410000100010023AA070383C6170393E60608F9
:10242000A388D70223800704A247F3A707800100EF
:1024300001001166B71700407D16D45BC85F938515
:102440004703A98EF18EF5FA93068008F3B606804D
:1024500093F6860836C601000100930670052380B6
:10246000D704930680FA2380D7040100010098C1A5
:1024700003C7170313670704A388E7022380070431
:10248000B247F3A7078001000100410182807D135C
:102490003368E3039308E016630E08003368F30320
:1024A0009308D016630808009378330093B8180097
:1024B0009388D81633081E01131E0801135E0E01FF
:1024C00055B56393E5030548638608000148630337
:1024D00003002A8871087298FD15131E0801C205B1
:1024E000135E0E01C18179BD13F8150063F4BF00BE
:1024F0007908D5B713381800E5BF83C7F60293F7FC
:102500000708A303F1000346710083C7F60293F79F
:102510000708E394C7FE8347710093F7F70FF1DFD5
:10252000E9B531714AD966CB06DF22DD26DB4ED70D
:1025300052D556D35AD15ECF62CD6AC96EC7AA8C26
:1025400002D897100000E78020B12A8993078008FD
:10255000F3B7078093F787083EDA01000100B71749
:102560000040130770052380E704130780FA2380D7
:10257000E7040100010003C7F7021377770FA38771
:10258000E70203C7F70213678700A387E7022380E8
:102590000704D257F3A70780010001000545970003
:1025A0000000E78060D6130780C13347E902116A53
:1025B00093070AE893065002BD69930BA004814A71
:1025C000014B13048008930470057D1AB347F90288
:1025D0003307D7023EC0FD873ECC938709A69309F7
:1025E000803E3347F7023AC27D873AC43347390306
:1025F0008549B399990193D93940B306D702B30BF2
:102600007703B3C6F602B3CBFB0236C6FD8636C8E7
:1026100093D6FB4136CEB7460F0093860624334946
:10262000D9028566938606FAB3969601B389E902C4
:10263000130760553309D90293060010B389E902E4
:102640003349D902B3C9F9029316390036CA37198A
:102650000040FD8636D0930D090493D7F9413ED250
:10266000F336048093F6860836DC010001009307F8
:1026700070052380FD00930680FA2380DD000100B1
:1026800001008346390593F6860FA309D9048346D2
:10269000390593E61600A309D90423800D00E256FC
:1026A000F3A6068001000100130C80FA116DF336C9
:1026B000048093F6860836DE01000100930770055A
:1026C0002380FD0023808D01010001008346390530
:1026D000216693E60602A309D90483560905B3E6E9
:1026E000A6012318D90483560905D18E2318D904CD
:1026F00023800D00F256F3A60680010001008346F8
:10270000390593F606026381061A03463905218AC4
:102710006DDE081897100000E7800098733604807B
:1027200013768608B2C20100010023809D00238039
:102730008D0101000100B717004003C6370513766D
:10274000F60DA389C70403C6370513660602A389DD
:10275000C704835609052166B3E6A6012318D904E8
:1027600083560905D18E2318D90423800D0096467F
:10277000F3A60680010001008346390593F60602A0
:10278000638B061483463905A18AEDFE970000206D
:10279000E7806090AA8636D497000020E780A08F5B
:1027A000A256E30AD5FE835609054255B3E6A601B3
:1027B0002318D90497100000E780C08F834639059D
:1027C000A18AEDDE03560905834629058247337643
:1027D000CA00B306DA0293D5F641B296B388F64042
:1027E000E24733B8C6002E983308F840A247B3B684
:1027F00016013308D84063C70701631DF8009247EC
:1028000063FA1701C247634FF80E63950701B24799
:1028100063EAF80E894663E9660FF24693151800DD
:1028200013D3F8015E8613951800B365B30042D642
:1028300046D497C00100E78000FB3258050B137B9C
:10284000FB0F63470001631A0838A25863870838F2
:1028500013081500B336A800B69513D6F5013298C3
:10286000B336C800AE9613581800FE06B3E606014C
:102870007336048013768608B2C6010001002380F7
:102880009D0023808D01010001000356C902B2960C
:10289000C206C1822316D90223800D00B646F3A6D4
:1028A00006800100010021B5F336048093F6860806
:1028B000B6C00100010023809D0023808D0101002E
:1028C00001008346390593E60602A309D904238053
:1028D0000D0086460DB5F336048093F68608B6C41F
:1028E0000100010023809D0023808D010100010073
:1028F0008346390593E60602A309D90423800D0017
:10290000A646BDB5E30B0BF0F336048093F68608BC
:10291000B6C801000100930680FA23809D00238041
:10292000DD00010001008346390593F5FC0F93F6A5
:10293000860FA309D90483463905CD8EA309D9048E
:1029400023800D00C646F3A6068001000100130592
:1029500080FA03463905930639051D8A631C9629BA
:102960007336048013768608B2CC0100010013068A
:1029700080FA23809D002380CD000100010003C662
:1029800006001376F60D2380C60003C60600136604
:1029900006022380C600835609051166D18E2318CE
:1029A000D904835609052166D18E2318D9042380C2
:1029B0000D00E646F3A6068001000100130680FA2A
:1029C0008346390593F60602638006268346390559
:1029D000130C3905A18AFDDA081897000000E7807A
:1029E000A06BF336048093F68608B6D00100010090
:1029F000930680FA23809D002380DD000100010002
:102A000083460C00116693F6F60D2300DC00834626
:102A10000C0093E606022300DC0083560905D18EE4
:102A20002318D904835609052166D18E2318D904A9
:102A300023800D008656F3A60680010001001306D0
:102A400080FA8346390593F60602638A0620834698
:102A50003905A18AEDFE97F0FF1FE780C0632A8C3D
:102A600097F0FF1FE7802063E30C85FF835609057D
:102A700011664255D18E2318D90497000000E780D3
:102A800060638346390513063905A18AFDDAF336FA
:102A9000048093F68608B6D401000100930680FAFC
:102AA00023809D002380DD00010001008346060095
:102AB00093F6F60D2300D60023800D00A656F3A64C
:102AC0000680010001008356090503462905D24707
:102AD000B376DA003306CA021305800C9355F6412B
:102AE0003696330DF6408257333CD6002E9C333653
:102AF000A601330CFC40330CCC40330885039256BE
:102B00004E86B335A5033305A503C29597C00100D2
:102B1000E78060CD63468001631E0C16630C0D16C2
:102B2000130615003335A6002E959356F5013696FB
:102B3000B335D600AA959396F50105828585D18E89
:102B40006346B000639D051A638B061A0356C902DB
:102B500015823305D6003336C500B2956348B00000
:102B6000639105241306F00F637DA622894663F363
:102B7000561593078008F3B7078093F78708BED6EA
:102B80000100010037170040930770052300F70488
:102B9000930780FA2300F704010001008356C7025F
:102BA00089678117D58FC207C1832316F7022300D7
:102BB0000704B657F3A7078001000100FA506A54D2
:102BC000DA544A59BA592A5A9A5A0A5BFA4B6A4C49
:102BD000DA4C4A4DBA4D296182801308F5FF33352E
:102BE000A800FD152E951356F5013298B336C8008E
:102BF000AA9695B9F336048093F68608B6CA010002
:102C0000010023809D002380AD0001000100834668
:102C10003905CD8EA309D90423800D00D646F3A62D
:102C200006800100010035B3F336048093F6860870
:102C3000B6CE0100010023809D002380CD0001005D
:102C400001008346390593E60602A309D9042380CF
:102C50000D00F646F3A606800100010095B3F33699
:102C6000048093F68608B6D20100010023809D00FF
:102C70002380CD00010001008346390593E606025A
:102C8000A309D90423800D009656F3A606800100FF
:102C9000010045BB9306F5FF33B5A600FD152E9543
:102CA0009355F501AE96B3B5B600AA951396F50106
:102CB000858269B5F336048093F68608B6D801009C
:102CC0000100930680FA23809D002380DD0001002F
:102CD00001008356C9020566011693F6F60FD18EE0
:102CE000C206C1822316D90223800D00C656F3A660
:102CF000068001000100850A93FAFA0F95B233E6C7
:102D0000B60045C20356C9023305D0403338A0008F
:102D1000B305B040B385054115826345B000D1E1EC
:102D20006371A608894663F0560593078008F3B7D8
:102D3000078093F78708BEDA01000100B71700404B
:102D4000130770052380E704130780FA2380E70444
:102D50000100010003D7C7027D8B2396E702238081
:102D60000704D65781BDF336048093F68608B6DC97
:102D700001000100930680FA23809D002380DD007E
:102D8000010001008356C9020566011693F6F60F8D
:102D9000D18EC206C1822316D90223800D00E656C9
:102DA000B9B793078008F3B7078093F78708BEDEAB
:102DB0000100010037170040930770052300F70456
:102DC000930780FA2300F704010001000356C702AD
:102DD00093975600B297C207C1832316F7022300C8
:102DE0000704F657C1BB914763EEB70217D701003E
:102DF0001307C73C8A05BA959C41BA978287B717D3
:102E0000004003A7470B1345F5FF698F23AAE70A84
:102E100003A7070B698F23A8E70A03A7070A798D81
:102E200023A0A70A8280B717004083A6470B134749
:102E3000F5FFF98E23AAD70A83A6070B558D23A881
:102E4000A70A83A6070A758F23A0E70A8280B7170F
:102E5000004003A7470B498F23AAE70A03A7070BE4
:102E60001345F5FF45BFB717004083A6470B13472F
:102E7000F5FF758F23AAE70A03A7070A598D4DB7F7
:102E8000B717004003A7470B498FEDB7914763EE93
:102E9000B70217D701001307A7338A05BA959C41DB
:102EA000BA978287B717004003A7470D1345F5FF70
:102EB000698F23AAE70C03A7070D698F23A8E70CE6
:102EC00003A7070C798D23A0A70C8280B7170040B9
:102ED00083A6470D1347F5FFF98E23AAD70C83A6C7
:102EE000070D558D23A8A70C83A6070C758F23A06B
:102EF000E70C8280B717004003A7470D498F23AA2C
:102F0000E70C03A7070D1345F5FF45BFB7170040B2
:102F100083A6470D1347F5FF758F23AAE70C03A778
:102F2000070C598D4DB7B717004003A7470D498FC0
:102F3000EDB7797122D43714004026D24AD0035914
:102F400024028354040206D64209C2044ECE52CC57
:102F500056CA13590901C1802DE11379F9F793F489
:102F6000F49F4209C20413590901C18093078008E4
:102F7000F3B7078093F787083EC401000100930769
:102F800070052300F404930780FA2300F404010081
:102F90000100231124032310940223000404A247F8
:102FA000F3A7078001000100B25022549254025945
:102FB000F249624AD24A45618280B7F507008146EC
:102FC0003000B105194597000020E7808081A247B5
:102FD00013972701E34A07FC1369090893E40440A7
:102FE00093098008F3B7098093F787083EC0010072
:102FF0000100930A700523005405130A80FA230088
:10300000440501000100231124032310940223002E
:1030100004048247F3A7078001000100294597F0C7
:10302000FF1FE7802031F3B9098093F989084EC268
:1030300001000100230054052300440501000100A4
:103040008357040293E707202310F40223000404AB
:103050009247B9B7B7170040884742054181937737
:10306000050491EB9377F5013755E80113050580C9
:103070003345F50282809377050C130700046397AC
:10308000E7009377F50137459C1CCDB72165130503
:1030900005D0828037E700E01C435443A183E20659
:1030A000D58F1CC1FD572320F7182322F7188280E3
:1030B00013178500B7E700E023A0E710618123A282
:1030C000A7108280B7F700E08847CC47828081470D
:1030D00037370040A14663C4C7003285828003456C
:1030E000B740E38EA6FE3385F5000345050085074E
:1030F0002304A740CDB797070020938727EF9C4371
:1031000017370020130707213E95636EE500173738
:1031100000201307274F6368A70017070020232705
:10312000A7EC3E858280FD57EDBF8280411122C40D
:1031300006C62A8497000000E78000F22947B307FB
:10314000E502B2408D83B3D7870222449507B3D7F7
:10315000E70237370040C207C1832316F700410159
:103160008280411137150E0006C697000000E780E7
:1031700020FCB7370040130770F82381E7000D47A4
:10318000A381E70013070004A380E7000547238716
:10319000E700B24041018280B737004003C7170003
:1031A00019C9D98DA380B70003C70700136787002B
:1031B0002380E700828093C5F5FFF98DA380B700D7
:1031C0008280AE872A87B7360040214637380040D4
:1031D00089E717030000670083F583C8B600E30999
:1031E00016FF05078348F7FFFD17C20723041801E0
:1031F000C183F9BF411122C406C62A84970000008A
:10320000E78080E52947B307E502B2408D83B3D755
:10321000870222449507B3D7E70237370040C20739
:10322000C1832316F7404101828071654111130566
:10323000052006C697000000E78000FCB737004075
:10324000130770F82381E7400D47A381E740130778
:103250000004A380E74005472387E740B2404101CF
:103260008280CC41411106C6328503C6150083C554
:10327000050022064D8E42068D654186138875A293
:10328000630C0611634BC804138845A26300060D46
:10329000634AC800938535A26301B60823900600EF
:1032A00029464DA0138855A26305060D938565A296
:1032B000E316B6FE8D451D4663E6E5081146198EF8
:1032C00063F3C7003E86B7E704002390C600FC47BF
:1032D00097D50100938505F29DA0138895A26303FD
:1032E0000611634E060D1388A5A26300061393858D
:1032F00005A5E315B6FA99451D4663E5E504198E63
:1033000063F3C7003E86B7E704002390C600FC477E
:10331000970500209385C5D71DA09D451D4663E3F5
:10332000E5022146198E63F3C7003E86B7E7040025
:10333000FC472390C6009705002093852538BA9551
:1033400082970146B240328541018280AD451D46DB
:10335000E3EAE5FE3146198E63F3C7003E86B7E720
:1033600004002390C600FC4797D50100938505EB28
:10337000F9B7B1451D46E3E7E5FC3546198E63F321
:10338000C7003E86B7E704002390C600FC4797D5E8
:1033900001009385A5E965B78D451D46E3E4E5FA8F
:1033A0001146198E63F3C7003E86B7E704002390E9
:1033B000C600FC4797D50100938585E449B78D4544
:1033C0001D46E3E1E5F81146198E63F3C7003E861A
:1033D000B7E704002390C600FC4797D5010093850A
:1033E000A5E6B1BFA5451D46E3EEE5F42946198ED5
:1033F00063F3C7003E86B7E704002390C600FC478E
:1034000097D50100938585E01DBFB5451D46E3EBCB
:10341000E5F23946198E63F3C7003E86B7E704002C
:103420002390C600FC4797D501009385A5DB01BF1B
:10343000B7E7040003A3071397060020938646C44A
:103440004146A54517050020130585BA02832D4581
:103450005DE703C505000947631FE50803A84500AC
:10346000411106C6034718003285034608002207AB
:103470004168518F930828FE6307170563E9E80048
:1034800005186303070323900600294591A8130636
:1034900048FE630AC7041518E31707FF15463E8761
:1034A000637BF600154701A8130600023E8763748C
:1034B000F60013070002B7E704002390E600FC477C
:1034C0001316070111A83E8691C30546B7E704000D
:1034D000FC472390C6004206CC45418282970145B5
:1034E000B24041018280130600083E87E375F6FC76
:1034F00013070008C9B72390060005458280828023
:10350000416779176304E504411122C406C6854763
:103510002A84639FF500B7E7040022852244B24065
:1035200003A3871397050020938585334101028308
:1035300089476399F500B7E7040083A7070B854522
:10354000829771D9B2402244410182808280797190
:1035500026D252CCAE842A8A97D501009385C5D055
:1035600017D501001305C5D206D63AC622D44AD0D3
:10357000368432894ECE97B00100E7800072A28572
:1035800017D501001305C5D197B00100E780E070A1
:10359000294597B00100E780207583C7840093F721
:1035A0000702F9E383C9040089470545324763965A
:1035B000F908D44083C7160083C60600A207D58F3A
:1035C000C166138616FE638CC7028D16638FD706FD
:1035D0008D669386269029456391D706B7E7040048
:1035E000A286225403A34714B250F2494A86A68504
:1035F000025992545285624A8547456102832D459E
:103600000DEF93070002354563E98702B7E7040031
:10361000FC47C84413060002CA8582978149970770
:1036200000209387A7249C43014581CB9C4391C7ED
:103630004E852286CA8582970145B2502254925403
:103640000259F249624A456182802D457DF7930710
:10365000700F3545E3E387FEB7E70400FC47C84435
:103660002286CA85829765BF2145C1BF411122C408
:1036700037E404008327841326C2AA84416506C662
:10368000970500209385C51D7D1582978327C40A61
:1036900017050000130505E78588829795C0032369
:1036A00004132244B2409244970600209386C6AF8A
:1036B0004146C545170500201305059E41010283BB
:1036C000B2402244924401454101828019C59707C6
:1036D000002023ADA718014582804545828011470F
:1036E000636AA70A97D601009386C6B60A0536957F
:1036F0001841411106C63697AE87B2850287130777
:1037000000026145639DE700B7E70400FC4713062C
:103710000002170500201305E5FA82970145B24023
:103720004101828005476145E39BE7FEB7E704005E
:10373000FC470546170500201305C5FAF9BF130716
:10374000700F6145E39DE7FCB7E70400FC471306F3
:10375000700F17050020130525F9C1B713070008DE
:103760006145E39EE7FAB7E70400FC47130600084B
:10377000170500201305C5064DB715476145E390B1
:10378000E7FAB7E70400FC471546170500201305C4
:10379000650D61B709458280411126C2B7E4040076
:1037A00083A7C41322C44AC006C62E8497050020EE
:1037B0009385050B2A898297058905C597070020FF
:1037C0009387878D83D7A70BA28503A3440D23106E
:1037D000F4002244B24092444A8502490146410124
:1037E0000283B24022449244024949454101828009
:1037F00097070020238E07069707002023AC0706B3
:10380000B717004003A7070CB706C0FFFD16758F5A
:1038100023A0E70C03A7070DB7064000558F23A888
:10382000E70C03A7070C3D9B23A0E70C03A7070D9C
:103830001367070123A8E70C8280B717004003A590
:10384000470C83A7470C598113451500C18B058987
:1038500099E3136525009707002083C767016380FC
:10386000A702970700202385A70011C9970700200A
:103870009387470003A3070063030300028382804A
:10388000114517F3FFFF670003CA011122CC06CED2
:103890003714004026CA4AC84EC652C48344740531
:1038A000034AB405834984050349940597F0FFFF53
:1038B000E78040A28347A40593F4F40F137AFA0F2C
:1038C00093E71700230DF40493F9F90F1379F90F17
:1038D000B717004003C7A705058B6DFF03D5C705C4
:1038E000A38D4705238C3705A38C2705A38B97044D
:1038F000F2406244D2444249B249224A0561828080
:1039000041119397050122C406C626C2C1872E84A1
:1039100063DC0700B7E40400FC54829719C1BC546F
:1039200082972165218D15A893F7150013C5150001
:103930008DE793F725009DC797000000E78020F0F2
:10394000B7E70400BC4F1306000A8945170500209D
:103950000345C5F2829713452400B24022449244A5
:10396000410182809397250163D80702B7E40400E0
:1039700083A7C41E829797000000E780A0F0BC4C8C
:1039800037560700130606308965170500200345E2
:10399000E5EE8297096579B7939715010145E3DE56
:1039A00007FA17D501001305A59797B00100E78026
:1039B000A046B7E70400BC4F1306006491651705E5
:1039C00000200345A5EB82971165A9BF1D71A2CC0C
:1039D00037E404005C5C485886CE494697D5010020
:1039E0009385858F829711E917D5010013050590FE
:1039F00097B00100E780404201A0B7F600E0795798
:103A000098CAFD57DCCA0567B7E700E023A0E710B6
:103A10001306F00290C223A0E71801000100370747
:103A2000002018471306000481459706002023A5AF
:103A3000E6E44157A38AE7403C4408088297971779
:103A40000020938727803EC88567138707409387A8
:103A500057D1231AE1002312F1021307B00F97F791
:103A6000FFFF938767662310E1023ED8154797074B
:103A700000009387C7E1B7F50700A30FE1003EDC24
:103A80000547970700009387E7DF81463000E1058F
:103A900019452301E1023EDE97F0FF1FE78060D465
:103AA00018088147994630003E9603460600850770
:103AB0000507A30BC700E398D7FEC24791C703577A
:103AC000410185676373F70001A0B7E7040083A78E
:103AD000470A08088297AA8511C917D5010013055E
:103AE000258297B00100E780401B01A0F6406644A4
:103AF00025618280411126C2B7E4040083A704082F
:103B000006C622C4170500001305C5DF82971704F7
:103B100000201304A4D62300A40097000000E7802F
:103B2000800297000000E780E0CC034504002244B7
:103B300003A38405B2409244130600328965410113
:103B40000283797106D622D413078008F3370780E1
:103B500093F787083EC201000100B71700409305A4
:103B600070052380B704130680FA2380C704010080
:103B7000010083C6F70293F6A60FA387D70223801E
:103B800007049246F3A60680010001007337078000
:103B9000137787083AC4010001002380B70423800B
:103BA000C7040100010003C7F70213672700A387BA
:103BB000E70223800704A247F3A707800100010062
:103BC000054597E0FFFFE780207497000000E7803D
:103BD00060CB014781468147054685451305407EF8
:103BE00097E0FFFFE780207737E404003C4468005B
:103BF000514681458297B707C0A83EC8B787E803FA
:103C0000938707D03ECA97E7FF1F9387477B3EC63F
:103C10007C5868008297B2502254456182804111DD
:103C200097D501009385C5D317C5010013054566D7
:103C300006C697B00100E780400617D501001305BE
:103C400065EC97B00100E7804005B240294541018D
:103C500017B3010067004309411197D5010093850F
:103C600065D117C501001305A56206C697B001000E
:103C7000E780A00217D50100130585E797B0010082
:103C8000E780A001B2402945410117B30100670058
:103C9000A305411122C406C6834705002A849DC797
:103CA00097D50100938545D417C501001305455EDE
:103CB00097B00100E78060FE4C4017D50100130566
:103CC000A5F697B00100E78040FD3DA058410DEFFB
:103CD00097D50100938545D117C501001305455BB4
:103CE00097B00100E78060FB17D50100130545F58B
:103CF00097B00100E78060FA2244B24029454101B3
:103D000017B30100670043FEA1679386D7036313CF
:103D1000D70297D50100938525CD17C5010013055E
:103D2000255797B00100E78040F717D5010013052C
:103D300025F27DBFED0797D501009385E5CA17C52C
:103D400001001305E554631BF70097B00100E780FD
:103D5000C0F417D501001305E5F059BF97B0010075
:103D6000E780A0F34C4017D501001305A5F191BFE2
:103D7000411197D50100938525C117C50100130591
:103D8000255106C697B00100E78020F1B2402945D1
:103D9000410117B30100670023F5797122D426D2BF
:103DA0004AD02E842A898145B2844800714606D6BD
:103DB00097E0FFFFE780A03597F7FF1F9387C76065
:103DC000DC4783D70700231421012313F100975008
:103DD0000000E78020039547A305F1009307401FEB
:103DE0003EC6FD572305A100230AF10097500000AD
:103DF000E78080152686A285480097500000E7805E
:103E00004003B250225492540259456182804111BC
:103E1000814617F6FF1F13066657854517050020D4
:103E20000355452706C697C00000E780C05815C94E
:103E300097D501009385C5B717C501001305454502
:103E400097B00100E78060E517D501001305C5D9DB
:103E500097B00100E78060E4294597B00100E78052
:103E6000A0E897D501009385A5B417C501001305F7
:103E7000254297B00100E78040E217D50100130505
:103E8000E5D797B00100E78040E1294597B00100F0
:103E9000E78080E597F7FF1F93870753DC470547C7
:103EA00097D501009385C5B02390E70017C50100A1
:103EB0001305053E97B00100E78020DE17D501000D
:103EC000130505D597B00100E78020DDB2402945F4
:103ED000410117B30100670023E1172500200355B6
:103EE000E5869307E5FFC2072167C1839306D7FFE5
:103EF00063F5F6029707002083C7479997060020CD
:103F000083C6D698A207D58F9306E7FFFD8E1305CB
:103F1000001081C67D1733F5E7008280411126C26B
:103F2000B7E40400FC4406C622C44AC02A844146C1
:103F300097D50100938585D717F5FF1F1305054613
:103F4000829797000000E78080F917090020130985
:103F5000091E2310A90097D501009385A5A617C5B2
:103F600001001305E53297B00100E78000D38355C7
:103F70000900228617D50100130585D797B00100E7
:103F8000E780A0D1294597B00100E780E0D52286DF
:103F9000224403A38405B24092440249170500203D
:103FA0000345458E894541010283011122CC06CE8D
:103FB00026CA4AC84EC693F715002E84A5CB970093
:103FC0000000E78000E5930710F817070020230D95
:103FD000F7169707002083D7A70B914517050020F8
:103FE0001305851617070020A300F716A1831707EE
:103FF0000020230CF71497070020A388071497606C
:104000000000E780C0A697200000E780A04005459B
:1040100097600000E780A0AE93441400F240624431
:1040200026854249D244B2490561828093F7250032
:10403000E9CF170700200357870F69C7AD64B71989
:1040400000409384A4AA23A0990097060020938699
:10405000660E944297D70100938787CD17060020FC
:104060000346060D814517F5FF1F1305253397708D
:104070000000E780005023A0990097F7FF1F2391CD
:10408000A7242A8941C197D501009385659B17C54F
:1040900001001305E51F97B00100E78000C0CA8545
:1040A00017C501001305853697B00100E780E0BE13
:1040B000294597B00100E78020C397070020239887
:1040C0000706930710F817070020230FF706970736
:1040D000002083D7E7FB17070020A307F706A1837B
:1040E000170700202303F70691458D471705002089
:1040F0001305850517070020A309F7049760000042
:10410000E780E0969344240011BF93F70510C1CFD8
:10411000AD64371900409384A4AA23209900171591
:1041200000200355A56297200000E780E059232076
:10413000990097000000E78080DA2A899700010043
:10414000E780E0DB9344041031C1171400200354CE
:104150002463631D240397D501009385658E17C5DD
:1041600001001305E51297B00100E78000B3A285B6
:1041700017C501001305452B97B00100E780E0B19A
:10418000294597B00100E78020B649BDB7E7040094
:10419000BC4F130600149305002017F5FF1F0345BD
:1041A000656E8297A5BD93F705209DCFAD67371744
:1041B00000409387A7AA1CC397000100E78020D482
:1041C00009CD8547170700202302F7F697700000F6
:1041D000E780004A9344042091B51305000A970034
:1041E0000000E780E0D3FDB793F74500D1C397D532
:1041F00001009385E58417C501001305650997B093
:104200000100E78080A917C501001305A52397B019
:104210000100E78080A8294597B00100E780C0AC85
:10422000930720F8170700202300F7F297070020D4
:1042300083D747E817070020A308F7F0A1831707E3
:1042400000202304F7F0854717070020A30FF7EE9F
:1042500097500000E78040CF9145170500201305D7
:10426000A5EE97600000E7808080934444007DB312
:1042700093F78500A9C797C501009385657C17C58D
:1042800001001305E50097B00100E78000A117C504
:1042900001001305651C97B00100E78000A02945C7
:1042A00097B00100E78040A4934484009707002062
:1042B000239F07E697700000E780803B85B393F764
:1042C0000501D1C38545170500200355A5DE97607C
:1042D0000100E78080F197C501009385657617C5D9
:1042E00001001305E5FA97B00100E780009B17C5B0
:1042F00001001305A51797B00100E780009A294532
:1043000097B00100E780409E930730F81707002020
:10431000230CF7E29707002083D7C7D9170700209F
:10432000A304F7E28D45A183170500201305C5E11D
:1043300017070020230BF7E0934404019750000077
:10434000E780E072E1B993F70502D1C797C5010094
:104350009385056F17C50100130585F397B001001C
:10436000E780A09317C501001305851297B00100DF
:10437000E780A092294597B00100E780E096930777
:1043800040F8170700202301F7DC9707002083D7A8
:10439000A7D017070020A309F7DAA1831707002089
:1043A0002305F7DA854717070020A300F7DA9707F8
:1043B0000020239307CE97500000E780E0B8914596
:1043C00017050020130545D897500000E780206AA4
:1043D00093440402A1B193F70504FDC397C50100FE
:1043E0009385056617C50100130585EA97B001009E
:1043F000E780A08A17C501001305050B97B00100DF
:10440000E780A089294597B00100E780E08D9707F4
:10441000002083C767D31307700A6386E706130774
:10442000800A638CE7081307600A6393E704930725
:1044300060F8170700202309F7D09707002083D7DB
:10444000C7CE17070020A301F7D0A18317070020CC
:10445000230DF7CE854717070020A30CF7CEB145F3
:1044600017050020130545CE97500000E780206017
:1044700097500000E78040AD934404049707002064
:10448000239507CA61BE930770F817070020230D14
:10449000F7CA9707002083D747C917070020A3054D
:1044A000F7CAA183170700202301F7CA854717071A
:1044B0000020A30DF7C8994565B7930780F8F1B7B9
:1044C00093F705088144E38B07B497C501009385F2
:1044D000255717C501001305A5DB97A00100E7804C
:1044E000C07B17C501001305A5FD97A00100E7805B
:1044F000C07A294597A00100E780007F9307A0F8C4
:10450000170700202302F7C49707002083D7C7C2EC
:1045100017070020A30AF7C2A1831707002023066C
:10452000F7C2854717070020A301F7C297070020AD
:10453000239407C097500000E78000A1914517051C
:104540000020130565C097500000E7804052934457
:104550000408E9B4411122C497C501009385054AB6
:104560002A8417C501001305A5D206C697A001002D
:10457000E780A0724C4017C501001305656497A041
:104580000100E7808071294597A00100E780C07590
:10459000034704009307F00F631FF70297C501005C
:1045A0009385C54517C50100130585CE97A0010069
:1045B000E780A06E4C4017C501001305656197A008
:1045C0000100E780806D2244B2402945410117A3D4
:1045D000010067006371B240224441018280970765
:1045E00000202399A7AA970700202393B7AA8547FD
:1045F0004111171700202315B71817C5010013051F
:1046000025C997C501009385A539170700202312F6
:10461000F7A8171700202307F70206C697A0010086
:10462000E780A0679715002083D5851517C5010081
:104630001305856E97A00100E7802066294597A0A5
:104640000100E780606A97F7FF1F9387E7D7DC4791
:1046500003D70700C167FD176310F702B7E704002F
:10466000B24003A3870517F5FF1F0345A5211306D5
:10467000000A854541010283B24041018280B1C1F7
:10468000411122C417C50100130585C02E8497C5AA
:1046900001009385253006C697A00100E780E05F02
:1046A000A28517C501001305E56397A00100E78007
:1046B000C05E2244B2402945410117A301006700B2
:1046C000A362828097170020239C070A9717002077
:1046D000238A07F6B7E70400FC47411106C64146A6
:1046E00097C501009385855B17F5FF1F130505CB63
:1046F000829717070020034727A59307F00A631541
:10470000F7029307F0F88945170500201305C5A3A4
:1047100017070020230AF7A297070020A38607A205
:1047200097500000E780A03497500000E7800060B9
:104730008145370504009707002023AD079E9707A2
:1047400000202396079E970700202383079E970744
:1047500000202391079697070020239F0792970731
:1047600000202394079C970700202397079C9730ED
:104770000000E780A0B7014597500000E78020388F
:104780009707002083C7879A1305000A99C79707E0
:104790000020238D079813050064B240410117F3F0
:1047A000FFFF6700E377B7E7040003A3870513065D
:1047B00000149305001017F5FF1F0345A50C028395
:1047C000011122CC37E404005C5C06CE354697C567
:1047D00001009385653417D501001305A50982975B
:1047E00011E917C50100130565B097A00100E78026
:1047F000A06201A097F7FF1F938787093EC4B7F512
:104800000700856793870780814617F6FF1F130609
:10481000A607E10519453EC697E0FF1FE78060FC4B
:104820007C44194697F5FF1F938505061705002060
:10483000130585888297340017F6FF1F1306C604F8
:1048400097D501009385C58017D501001305C58153
:1048500097700000E780E0A62A841DCD97C501006F
:104860009385051D17C50100130585A297A00100BA
:10487000E780A042A28517C501001305E52A97A08D
:104880000100E7808041294597A00100E780C045ED
:10489000F24062440561828097E00000E780E00C0E
:1048A00017C501001305451F97600000E780209B96
:1048B00097A00000E780206197600100E780A0C515
:1048C00017F5FF1F1305C5AB97600100E78040AEE9
:1048D00017C501001305451D97600100E78020C63C
:1048E0002A8497600000E780600197100100E7804C
:1048F000809D97800100E780A03697700000E780D8
:10490000405D97600000E780607797300100E780A6
:10491000E05E97C501009385A51117C50100130539
:10492000259719C897A00100E7802037A28517C5F1
:1049300001001305A521A1B797A00100E780E0358C
:1049400017C501001305C52297A00100E780E034D8
:10495000294597A00100E780203997300100E780C2
:10496000C03A97F00000E78080597DC18545370542
:10497000040097300000E780609797C50100938599
:10498000250B17C501001305A59097A00100E7802E
:10499000C03017C501001305251F97A00100E7804F
:1049A000C02F294597A00100E780003497F7FF1F2B
:1049B0009387079083D70700171700202312F7DC8F
:1049C000854717170020230FF7C697F7FF1F938718
:1049D000A79FDC4703D70700C167FD176316F700E1
:1049E00097F0FFFFE780E04297700000E78080D8F3
:1049F0001305C51497700000E78080D89720000049
:104A0000E78060B897200000E780C0A0171500205D
:104A1000035505D797500000E780C0DA0545975049
:104A20000000E780C00D97C501009385650017C59C
:104A300001001305E58597A00100E780002617C552
:104A400001001305A51697A00100E780002525BDEC
:104A500097500000E780A00A1305000A97F0FFFFB7
:104A6000E780004CC9B7411122C437E40400832712
:104A7000041A06C6829797500000E78060D8832703
:104A8000040817F5FFFF13058552829797F7FF1F5C
:104A9000238AA7DE17F5FF1F130505939740000033
:104AA000E780207D2244B2404101170300006700E7
:104AB00063D1B7E70400FC471171A2DDCAD986DFD4
:104AC000A6DBCED72E8432892E86AA8517F5FF1F46
:104AD00013058567829717F7FF1F1307E76683475C
:104AE0000700930680029387E70793F7F70FE3EC3D
:104AF000F610BA898A0717C701001307A782BA9769
:104B00009C43BA9782878D4797C50100938585F4AA
:104B100017B501001305C577630FF40097A00100D6
:104B2000E780A01717C50100130505B097A0010085
:104B3000E780A016BDA497A00100E780001617C566
:104B400001001305E5AF97A00100E7800015294596
:104B500097A00100E7804019930720F8114697F5C8
:104B6000FF1F9385655E4A8517F7FF1F230EF75CCD
:104B700097F7FF1FA38B075C97F0FFFFE7802022CA
:104B80002A841DC997C501009385C5EC17B501009E
:104B90001305057097A00100E7802010A28517C5B6
:104BA00001001305A5AD97A00100E780000F29457E
:104BB00097A00100E780401397C50100938585E920
:104BC00017B501001305C56C97A00100E780E00C44
:104BD00017C501001305C5AB97A00100E780E00BE6
:104BE000294597A00100E78020104165930730FA1E
:104BF000054697F5FF1F938525557D1517F7FF1F70
:104C00002304F75497F0FFFFE78060192A841DC939
:104C100097C50100938505E417B5010013054567A5
:104C200097A00100E7806007A28517C50100130562
:104C3000E5A497A00100E7804006294597A0010060
:104C4000E780800AB7E70400BC4F0566130606C874
:104C5000A14517F5FF1F0345E5C28297FE506E542C
:104C6000DE544E59BE591161828091476303F402AC
:104C700097C50100938505DE17B501001305456151
:104C800097A00100E780600117C50100130585A307
:104C900071BDB7E70400FC4F914517F5FF1F0345B1
:104CA00065BE829797C501009385C5DA17B50100E7
:104CB0001305055E97A00100E78020FE17C50100DF
:104CC000130505A297A00100E78020FD294597A0C4
:104CD0000100E780600197400000E780E0269145F1
:104CE00035A485476303F40297C50100938585D6F3
:104CF00017B501001305C55997A00100E780E0F939
:104D000017C501001305459F15B597F7FF1F23939E
:104D1000273BB7E704000566BC4F130606C8C1452C
:104D20000DBF8D476303F40297C50100938585D2BB
:104D300017B501001305C55597A00100E780E0F500
:104D400017C501001305059DD5B3930740F811461B
:104D500097F5FF1F9385453F4A8517F7FF1F2305EA
:104D6000F73E97F7FF1FA382073E97F0FFFFE7800C
:104D700000032A84E30405EE97C50100938585CDE1
:104D800017B501001305C55097A00100E780E0F0BA
:104D9000A28517C501001305658E97A00100E78065
:104DA000C0EF294597A00100E78000F445BD914779
:104DB000E31CF4F6B7E70400FC4F9305000217F577
:104DC000FF1F034525AC829797C50100938585C8D1
:104DD00017B501001305C54B97A00100E780E0EB74
:104DE00017C5010013058594F1BD894763E3870268
:104DF00097C50100938505C617B501001305454900
:104E000097A00100E78060E917C5010013054593ED
:104E100031BB97F4FF1F83C4443397F7FF1F83C749
:104E2000B73297C501009385E5C2A20417B501000A
:104E300013050546DD8C97A00100E78000E6A285FA
:104E400017C501001305059197A00100E780E0E474
:104E5000C204294597A00100E78000E9C1849305B9
:104E6000D4FF93960401C1824A8693F5F50F17F596
:104E7000FF1F1305952D97200000E780E04AE35FB0
:104E800090DC930750F817F7FF1F230FF72A83C70B
:104E90003900228697F5FF1F9385052B85074A85E4
:104EA00017F7FF1FA303F72A97F0FFFFE78020EF14
:104EB0002A84E30505DA97C501009385A5B917B5DE
:104EC00001001305E53C97A00100E78000DDA28505
:104ED00017C50100130505E0C9B5894763E38702DB
:104EE00097C50100938505B717B501001305453A2D
:104EF00097A00100E78060DA17C501001305458718
:104F000035B197400000E7802004A28517F5FF1F08
:104F10001305852397500000E78060B581B38D4766
:104F20006303F40297C501009385C5B217B501006C
:104F30001305053697A00100E78020D617C50100AC
:104F40001305C584E5B6B76602000146B7750200D1
:104F5000054597E0FF1FE780C088930760F817F7C3
:104F6000FF1F2303F71E97F7FF1FA380071E93075A
:104F7000000617F7FF1F230BF71C894717F7FF1FC2
:104F8000A306F71C97F7FF1F2383071C97F7FF1F44
:104F9000A38F071AC14717F7FF1F230BF71A9307B1
:104FA00020F917F7FF1FA305F71A314697F7FF1FE0
:104FB000A381A71A97F5FF1F938505194A8597F7CF
:104FC000FF1F2388071897F0FFFFE78040DD2A8442
:104FD000E30605C897C501009385C5A717B501006D
:104FE0001305052B97A00100E78020CBA28517B5FC
:104FF00001001305257B55B3B1476303F40297C540
:105000000100938525A517B501001305652897A014
:105010000100E78080C817B501001305657A39B62D
:10502000B7E70400FC4F9305000417F5FF1F034585
:105030006585829797400000E78000F1B145F9B59A
:10504000914763E3870297C501009385A5A017B533
:1050500001001305E52397A00100E78000C417B500
:1050600001001305A577D9B497F4FF1F83C4040E7C
:1050700097F7FF1F83C7770DA204DD8C8E04B777E7
:1050800002006D14BE942286A68517B50100130593
:10509000257697A00100E78040C0B7E70400FC47F1
:1050A000228697F5FF1F9385750A2800829793162D
:1050B0000401C1823000A685094597D0FF1FE78013
:1050C00040722A8409C917B501001305257497A0F9
:1050D0000100E78060D4930770F8194697F5FF1F29
:1050E000938585064A8517F7FF1F230FF70497F767
:1050F000FF1FA38D870497F0FFFFE78040CA2A8433
:10510000E30E05B497C501009385C59417B501005A
:105110001305051897A00100E78020B8A28517B5F0
:1051200001001305A56F95B99947630BF41297C554
:1051300001009385259217B501001305651597A009
:105140000100E78080B517B501001305A56EF9BA17
:10515000914763E3870297C501009385A58F17B533
:1051600001001305E51297A00100E78000B317B511
:1051700001001305A56D5DBA97F4FF1F83C404FDFC
:1051800097F7FF1F83C777FCA204DD8C8E04B777E7
:1051900002006D14BE942286A68517B50100130582
:1051A000256C97A00100E78040AFB7E70400FC47FB
:1051B000228697F5FF1F938575F92800829793162D
:1051C0000401C1823000A6850D4597D0FF1FE780FE
:1051D00040612A8409C917B501001305256A97A003
:1051E0000100E78060C3930780F8194697F5FF1F19
:1051F000938585F54A8517F7FF1F2307F7F497F77F
:10520000FF1FA38587F497F0FFFFE78040B92A844A
:10521000E30605A497C501009385C58317B5010072
:105220001305050797A00100E78020A7A28517B501
:1052300001001305E56595B699476303F40297C528
:1052400001009385258117B501001305650497A01A
:105250000100E78080A417B501001305E564F9B0EB
:10526000B7E70400FC4F9305000417E5FF1F034553
:105270006561829797400000E78000CD994579B13C
:105280008D476303F40297B501009385A57C17B59C
:1052900001001305E5FF97A00100E78000A017B506
:1052A00001001305E56159B017B50100130545620A
:1052B00097A00100E78040B61305C01297D0FF1FEA
:1052C000E7802008014597E0FFFFE780E0DC0D451F
:1052D00097100000E78080A0294597D0FF1FE78046
:1052E000400697D0FF1FE780A0F68DBA9947630369
:1052F000F40297B501009385E57517B50100130514
:1053000025F997A00100E780409917B50100130522
:10531000E55C29B817F7FF1F034757E397F7FF1F0F
:1053200083C7C7E222075D8F9166BA96C2061166EF
:10533000C1821306F6EF8D476365D60297E7FF1F1C
:10534000938787089C4B17F6FF1F034616E093864A
:10535000C7002DC203D6070069CA8907E39CD7FEA0
:1053600089471307A0F8114697F5FF1F9385C5DD00
:105370004A8597F6FF1F2389E6DC17F7FF1FA30670
:10538000F7DC97F0FFFFE78080A12A84E308058C13
:1053900097B501009385056C17B50100130545EF1E
:1053A00097A00100E780608FA28517B50100130563
:1053B0002554E5B203D60700630EE60A8907E39B8E
:1053C000F6FE8D4779BF91476304F40297B501005B
:1053D0009385456817B50100130585EB97A001007B
:1053E000E780A08B17B50100130505526FF00FF48D
:1053F000B7E70400FC4F9305000817E5FF1F0345BE
:1054000065488297C9B897B501009385A56417B51B
:1054100001001305E5E797A00100E780008817B5B4
:1054200001001305E54F6FF06FF02390E70017E5DB
:10543000FF1F130565F997300100E78080B297B52B
:1054400001009385256117B50100130565E497A058
:105450000100E780808417B501001305654D97A012
:105460000100E7808083294597A00100E780C0877D
:105470008147C5BD2390070017E5FF1F1305C5F43D
:1054800097300100E780E0AD97B501009385855C1A
:1054900017B501001305C5DF97900100E780E07F95
:1054A00017B501001305454A5DBF411122C406C668
:1054B000834705002A849DC797B50100938545550C
:1054C00017B501001305C5DC97900100E780E07C6B
:1054D0004C4017C501001305A58697900100E78091
:1054E000C07BC9A85841B707CF009387777D631267
:1054F000F70897B501009385A55117B5010013056D
:1055000025D997900100E78040791C448356E40038
:105510008355C40003C6070017C501001305C583E2
:1055200097900100E7806077294597900100E78018
:10553000A07B0357E4009707002083D76724630EFE
:10554000F7008355C4000844854717070020230E41
:10555000F71E97300000E780C03E0356E4008355F5
:10556000C40008442244B240410117F3FFFF670022
:105570008354B707CC009387777D6315F70497B5FD
:1055800001009385E54817B50100130565D0979094
:105590000100E78080701C448356E4008355C400FA
:1055A00003C6070017B501001305057B979001009E
:1055B000E780A06E2244B2402945410117930100C3
:1055C00067008372B707CE009387777D6304F70285
:1055D00097B501009385C54317B50100130545CB69
:1055E00097900100E780606B4C4017B501001305F0
:1055F0006569E5B5B240224441018280B7E7040005
:10560000FC4741112E8606C622C426C24AC02E84FB
:105610002A89AA8517F5FF1F130505B3829797B549
:1056200001009385E54417B50100130565C6979001
:105630000100E780806697F5FF1F83C5E5B017B5C9
:105640000100130565E997900100E7800065294591
:1056500097900100E780406997F4FF1F9384C4AEE0
:1056600083C7040041479387070693F7F70F636EDC
:10567000F75A17B70100130727D58A07BA979C4333
:10568000BA9782879D476307F40297B50100938517
:10569000253E17B501001305A5BF97900100E780CF
:1056A000C05F17B501001305A5E397900100E780DF
:1056B000C05E8DA497F7FF1F83C717A9DDCB17F72F
:1056C000FF1F034797A897F7FF1F83C707A8220765
:1056D0005D8F97F7FF1F83C767A7C2075D8F97F797
:1056E000FF1F83C7B7A6E207D98F17F7FF1F232332
:1056F000F7A483C7640097B501009385653717B594
:1057000001001305E5B817F7FF1F2303F7A29790D1
:105710000100E780805897F7FF1F9387A7A18C436C
:1057200017F6FF1F0346C6A017B50100130505DDD8
:1057300097900100E7806056294597900100E78027
:10574000A05A97F7FF1FA38107A02244B2409244BA
:105750000249930700F817F7FF1F2307F79E9D459F
:1057600017F5FF1F1305459E410117430000670011
:10577000033097600000E78020FF97F7FF1F238624
:10578000A79C9357850017F7FF1FA300F79C93571B
:1057900005012A8417F7FF1F230AF79A93578501FB
:1057A000014517F7FF1FA303F79A97600000E780F2
:1057B000000097F7FF1F238CA79897B501009385EA
:1057C000252B17B501001305A5AC97900100E780C4
:1057D000C04C17F6FF1F03468697A28517B5010038
:1057E000130545D3B1B7CD476303F40297B5010064
:1057F0009385052817B50100130585A99790010029
:10580000E780A04917B50100130545D279BD37E4FB
:1058100004007C44414697F5FF1F9385F59217E5F8
:10582000FF1F1305A5B7829797F7FF1F83C7E7925E
:1058300017F7FF1F03475792A20703238405D98F49
:1058400017F7FF1F2315F78E1306000A8945224418
:10585000B2409244024917E5FF1F0345A5024101EA
:1058600002838D476303F40297B5010093854520B9
:1058700017B501001305C5A197900100E780E0412D
:1058800017B50100130545DA0DB517F4FF1F0344E2
:10589000C48B97F7FF1F83C7378B97B5010093859C
:1058A000251D220417B501001305859E5D8C979078
:1058B0000100E780803EA28517B50100130585C869
:1058C00097900100E780603D294597900100E780AF
:1058D000A0410D4697F5FF1F93850587228597E028
:1058E000FFFFE780C04BAA8421C197B501009385D3
:1058F000251817B501001305A59997900100E780B9
:10590000C039A68517B50100130505C5979001009C
:10591000E780A0382244B24092440249294541011F
:10592000179301006700433C97E7FF1F2394877894
:10593000B7E70400116603A38705130606E891453F
:1059400039B78D476303F40297B50100938545127B
:1059500017B501001305C59397900100E780E03368
:1059600017B50100130505DB89B317E4FF1F0344D6
:10597000C47D97E7FF1F83C7377D97B501009385E7
:10598000250F220417B50100130585905D8C9790B3
:105990000100E7808030A28517B50100130505BD21
:1059A00097900100E780602F294597900100E780DC
:1059B000A0330D4697E5FF1F93850579228597E073
:1059C000FFFFE780C03DAA841DC197B50100938504
:1059D000250A17B501001305A58B97900100E780F4
:1059E000C02BA68517B50100130585B905B797E744
:1059F000FF1F2393876AB7E70400116603A3870597
:105A0000130606E89305000299B5894763E3870208
:105A100097B501009385C50517B5010013054587A6
:105A200097900100E780602717B50100130545D165
:105A3000ADB997E4FF1F83C4447197E7FF1F83C785
:105A4000B77097B501009385A502A20417B50100B0
:105A500013050584DD8C97900100E7800024A6855E
:105A600017B50100130545B397900100E780E022C8
:105A7000294597900100E7802027228697E5FF1FA0
:105A80009385856C268597E0FFFFE78040312A8467
:105A9000630E051A97B50100938585FD17A50100D2
:105AA0001305057F97900100E780201FA28517B599
:105AB00001001305A5AF99BD854763F98718834594
:105AC00019002244B24092440249B335B00097E72E
:105AD000FF1F238BB75E17B50100130565AE4101AB
:105AE000179301006700631BA2852244B2409244D1
:105AF0004A85024941011703000067006324994762
:105B00006303F40297B50100938585F617A501009C
:105B10001305057897900100E780201817B501005C
:105B20001305C5DB59B617E4FF1F0344046297E76A
:105B3000FF1F83C7776197B50100938565F3220442
:105B400017A501001305C5745D8C97900100E780CF
:105B5000C014A28517B50100130505A89790010090
:105B6000E780A013294597900100E780E0171946C8
:105B700097E5FF1F9385455D228597E0FFFFE7804E
:105B80000022AA841DC197B50100938565EE17A573
:105B900001001305E56F97900100E7800010A685CE
:105BA00017B50100130545A495B397E7FF1F23958B
:105BB0008758B7E70400116603A38705130606E8B4
:105BC0009305000869B1854797B50100938545EABB
:105BD00017A501001305C56B630BF4009790010036
:105BE000E780A00B17B50100130545A17DBC979078
:105BF0000100E780800A17B501001305A5A1979061
:105C00000100E7808009294597900100E780C00DD9
:105C10002244B2409244024997E7FF1F239907505C
:105C20004101176300006700A3A497B501009385A5
:105C300025E417A501001305A56597900100E780ED
:105C4000C00517B501001305A5CD85B4B2402244A7
:105C50009244024941018280411106C622C497E064
:105C6000FFFFE780C01321CD97E7FF1F83D7E745EC
:105C700085072A8417E7FF1F2319F74497B501000A
:105C8000938585E097E7FF1F2392A74417A501009E
:105C90001305056097900100E7802000A28517B5E5
:105CA00001001305250397900100E78000FF2244BF
:105CB000B24029454101179301006700E30297E7CD
:105CC000FF1F83D7C740B2402244850717E7FF1F55
:105CD000231FF73E41018280411122C491462A844C
:105CE00017E6FF1F130686549D652D4506C697D0FF
:105CF000FF1FE78000AFB7F7070003C70701A547FD
:105D00006313F70001A09306001001469D65254529
:105D100097D0FF1FE780E0AC97E7FF1F23888750ED
:105D20002244B240914617E6FF1F130626509D6598
:105D30002945410117D3FF1F6700A3AA1171CED7D0
:105D4000B7E9040083A7C904CAD917E9FF1F1309DB
:105D5000A93FA2DD2E8686DFA6DB2E84AA854A8592
:105D6000829797E7FF1F83C7273E1307700A638553
:105D7000E710636DF7001307600A6385E704FE50C0
:105D80006E54DE544E59BE59116182801307800A49
:105D90006385E7161307900AE393E7FE8D476306D2
:105DA000F41C97B501009385A50617A501001305FE
:105DB000254E97900100E78040EE17B501001305CE
:105DC000650225A08D47630CF40297B50100938509
:105DD000250417A501001305A54B97900100E78046
:105DE000C0EB17B50100130525F997900100E78076
:105DF000C0EA294597900100E78000EF49B7854741
:105E000017B50100130505F917E7FF1F230EF72A41
:105E100097900100E7804000B7750200B766020066
:105E20000146054597D0FF1FE780A09B930760F8C8
:105E300017E7FF1F230AF73097E7FF1FA3870730F5
:105E40009307002617E7FF1F2322F730E577938794
:105E5000072117E7FF1F231DF72EB14597E7FF1F07
:105E60002389072E97E7FF1FA385A72E4A85970052
:105E70000000E780E01621B7914763E3870297B5FA
:105E800001009385E5F817A501001305654097907B
:105E90000100E78080E017B501001305A5F1B1B757
:105EA00097E4FF1F83C4842A97E7FF1F83C7F7295E
:105EB000A204DD8C83A7C9046D14228697E5FF1F19
:105EC0009385D528280082978E0493160401B77510
:105ED0000200C1823000A695094597D0FF1FE780D8
:105EE0004090930770F817E7FF1F230FF724994599
:105EF00097E7FF1FA38CA72495BF914763E3870211
:105F000097B501009385C5F017A501001305453825
:105F100097900100E78060D817B50100130505EBE5
:105F2000E9B597E4FF1F83C4642297E7FF1F83C787
:105F3000D721A204DD8C83A7C9046D14228697E5BE
:105F4000FF1F9385B520280082978E0493160401C5
:105F5000B7750200C1823000A6950D4597D0FF1F8E
:105F6000E7802088930780F8BDBF17B501001305AF
:105F7000A5E897900100E78020EA930790F82304B2
:105F8000F100834719008D452800A304F1008347E1
:105F900029002305F10097000000E7806004130545
:105FA000C01297C0FF1FE780C039014597D0FFFF9F
:105FB000E780800E0D4597000000E78020D229453C
:105FC00097C0FF1FE780E03797C0FF1FE78040289A
:105FD0007DB397E7FF1F23A3A726828097E7FF1FC4
:105FE0009387C72503A307006303030002831743B6
:105FF00000006700C3A741114AC097F6FF1F83D670
:106000002678328917F6FF1F0356467422C426C22B
:1060100006C62A84AE8497000000E780006235C17E
:106020002DC0994763FF970483471400034704007A
:10603000A207D98F13978700A183D98FC207316731
:10604000C1831307C755639EE70297F7FF1F83D7E6
:10605000E76FA301F400A1832302F40097F7FF1F69
:1060600083D7077291C7A302F400A1832303F4002E
:10607000A68517B501001305A5DD97900100E780FF
:10608000C0C197F7FF1F83C7E75BB9CF97F5FF1F25
:1060900083D5C56B17B50100130545DD9790010049
:1060A000E780A0BF2686A28517F5FF1F0355056A66
:1060B00097000000E78080BA6301090497E7FF1F9B
:1060C00083C707189DCB95C897E7FF1F83C7C7FFF6
:1060D0008DE722852244B2400249A68592444101BF
:1060E000174300006700A39817B50100130505D9F1
:1060F00097900100E78040D2C1B7B2402244924459
:10610000024941018280834755008345450017B508
:1061100001001305A5D2A207DD8D179301006700CA
:10612000C3B717B50100130565D0179301006700C9
:10613000A3CE8D4763FBB70A011126CA06CE22CC37
:106140000344350097E4FF1F83C4940F97B5010003
:10615000938585D3B337800017E7FF1FA302F70E9F
:1061600009C497B501009385E5D217B50100130561
:10617000E5D297900100E78040B297E7FF1F83C701
:10618000370C6386970097000000E780A03397E7FD
:10619000FF1F83C7F70A8DC785472306F100B7E7BE
:1061A000040083A747177000854513055030829778
:1061B00017B50100130585CF97900100E780C0C592
:1061C0009967938757EE2316F1006800854791453C
:1061D000A30781002307F10097000000E78040E05B
:1061E000F2406244D244056182808280894763F331
:1061F000B70A011122CC06CE26CA83442500854762
:106200002A84639DF404914763F5B70483474500EE
:1062100003473500A207D98F17F7FF1F2318F7523E
:1062200097E0FFFFE78060589967938767EE231434
:10623000F1008347340023059100A305F100834753
:106240004400954528002306F10097000000E780F0
:1062500020D9F2406244D24405618280FDF897F76C
:10626000FF1F83D7A74E9386E7FFC2062167C1822F
:1062700075176376D70097F7FF1F83D767501967A5
:10628000130767EEA305F1002314E10023050100C5
:10629000A18345BF82800111996722CCD51717F4DD
:1062A000FF1F1304243A2314F1008347040026CA75
:1062B00097F4FF1F9384C44C2305F10083D7040097
:1062C00028009545A305F100A18306CE2306F10021
:1062D00097000000E780C0D003D604008345040087
:1062E00017B50100130505BE97900100E780E09AFD
:1062F000F2406244D244056182809D677971D9176A
:106300002316F10097F7FF1F83C7C73306D623076D
:10631000F100A9C3B7E70400FC47414697D5FF1F2A
:106320009385C5071305F10082976800CD45970056
:106330000000E780E0CA97F5FF1F83C5A53017B5B9
:106340000100130525BB97900100E7800095B2502E
:1063500045618280B7E70400BC474146814513058B
:10636000F1008297D9B745C5411106C622C49307EB
:1063700050FA2300F5009307A005A300F500894714
:106380002301F5009147A301F50093071003A30231
:10639000F50097F7FF1F9387E72A83C707002302BB
:1063A00005002A842303F50097E7FF1F938757E929
:1063B00083C70700414697D5FF1F938525FEA3039A
:1063C000F50097F7FF1F83D7A73B2304F500A183B0
:1063D000A304F50097F7FF1F83D747372305F50080
:1063E000A183A305F500B7E70400FC4731058297B8
:1063F0002285F14597000000E7802020230EA400AD
:106400002181A30EA400B2402244410182808280F7
:106410005D710A8586C6A2C497000000E780E0F49B
:1064200037E404007C448A850810794682973C440E
:106430001305E10309468145829710109305000278
:10644000014597D0FFFFE780C029B640264461612F
:106450008280011122CC2D6426CA4AC84EC652C47D
:1064600056C25AC006CEB71400401304A4AA80C076
:1064700037E900E0B70940002A8AAE8A328B232030
:106480003919010001008566AA850146254597C096
:10649000FF1FE7800035DA865686D285294597C0EA
:1064A000FF1FE78000342320391180C0F24062448E
:1064B000D2444249B249224A924A024B0561828043
:1064C0000111B7C7A55A22CC9387C73317E4FF1F22
:1064D000130414D73EC4834704002C0021461965D9
:1064E00006CE3EC697000000E780E0F68345040034
:1064F00017B50100130585AE97800100E780E079AC
:10650000F2406244056182800111A1463000996524
:106510002D4522CC06CE97C0FF1FE780802CA247D6
:1065200037C4A55A1304C43363958702B24517B51F
:1065300001001305659EB335B00097E7FF1FA381E7
:10654000B7D097800100E7804075F2406244056152
:1065500082809165A1463000938505F02D4597C056
:10656000FF1FE7800028A247E38287FC854717E7E3
:10657000FF1FA307F7CC854517B501001305059C40
:10658000C9B77971D146700091652D4522D406D6E0
:1065900097C0FF1FE780E024B24737C4A55A130411
:1065A000F43563988702B7E70400FC4717D5FF1F4F
:1065B0001305C5DE41460C08829717B50100130587
:1065C000659D97900100E7802085B2502254456177
:1065D00082809165D1467000938505E82D4597C06E
:1065E000FF1FE7800020B247E38F87FA17B501004D
:1065F0001305459CF9B7C16769768146FD17050605
:106600001397060141836364B7003E858280330798
:10661000D50003470700B98F214713F8170085837A
:1066200063050800B18FC207C1837D171377F70F89
:106630006DF78506F1B741C5A547054763F2B70871
:1066400083471500034705003168A207D98F1397C8
:106650008700A183D98FC207C1831308C855054796
:1066600063900707411106C622C426C203442500D1
:10667000914763F087049307540063ECF502A3018C
:10668000C50021822302C5009304340091C6A302F1
:10669000D500A1822303D5002A84A6859700000097
:1066A000E780A0F526942300A4002181A300A40084
:1066B0000147B240224492443A8541018280054715
:1066C0003A8582800111B7C7A55A22CC9387E73457
:1066D0002A842AC621462C00156506CE3EC49700A2
:1066E0000000E78040D7A28517B50100130505918A
:1066F00097800100E780605A97000000E78080D112
:10670000F2406244056182800111A1463000956526
:106710002D4522CC06CE97C0FF1FE780800CA247F4
:1067200037C4A55A1304E43463958702B24517B5FC
:1067300001001305A58297F7FF1F2399B700C20533
:10674000C18197800100E7804055F24062440561B5
:1067500082809165A1463000938505EE2D4597C056
:10676000FF1FE7800008A247E38287FC17B50100FE
:106770001305C58097F7FF1F239A07FC9780010038
:10678000E7808069D9B797B701009387278B13D724
:10679000C5003E97034707001105230EE5FE13D7FA
:1067A00085003D8B3E9703470700A30EE5FE13D7F8
:1067B00045003D8BBD893E97AE970347070083C7D1
:1067C0000700230FE5FEA30FF5FE8280011122CC06
:1067D00006CE26CA4AC84EC693F715002E84638E8D
:1067E0000716AD679387A7AA371700401CC397F712
:1067F000FF1F83C787F599EF97F7FF1F83C767F8D8
:10680000850793F7F70F1D47636AF70217F7FF1F16
:106810002309F7F6B7E70400BC4F130600198545B6
:1068200017D5FF1F034545BC829713451400F2405E
:106830006244D2444249B2490561828097F7FF1F02
:10684000238107F4B75720419304D00393877774CB
:1068500097F5FF1F83D5C5F217F5FF1F130595EFB9
:106860001309000217F7FF1F2324F7EE97F7FF1F06
:10687000238297EE97000000E78020F12300250196
:1068800097F7FF1F83C707DCB337F0009387070331
:10689000A301F5009309000593072004A300350127
:1068A0002301950023022501A302F500230395008F
:1068B00097D5FF1F83D505B11D0597000000E78020
:1068C000C0EC23002501A3003501930750042301E8
:1068D000F500A301950097D5FF1F83D5659E11058F
:1068E00097000000E78060EA9307B00423002501C9
:1068F00023019500A300F50097D7FF1F83C707AAC0
:10690000A20797D5FF1F83C575A9DD8D0D059700DB
:106910000000E78080E797D7FF1F83C747A8A2073B
:1069200097D5FF1F83C5B5A7DD8D97000000E780D1
:10693000C0E5B5472300F500A947A300F50093057E
:10694000250017F5FF1F1305A5E0898DC205C1813C
:1069500097200000E780000875BD93F7250081CBE4
:1069600097F7FF1F239207DE13C52500C9B593F7DC
:1069700045000145E38D07EA17A501001305C56928
:1069800097800100E780404997300000E780C03BD6
:106990001345440069BD411122C437E404005C5C26
:1069A00006C6354697A501009385051717B5010062
:1069B000130545EC829711E917A5010013058566BB
:1069C00097800100E780404501A08327041C82973F
:1069D0002A84054597C00000E78080F89760010091
:1069E000E780A07D97600100E780A05297B000008B
:1069F000E780000A2285B240224441018280411191
:106A0000054506C622C426C297C0FFFFE780A052F4
:106A10001305A00497B0FF1FE78060697575854571
:106A20007D1597C0FFFFE780403C7D7585451305C8
:106A3000F53697C0FFFFE780A04537140040832755
:106A4000840A8D451305002093E707202324F40AC8
:106A500097C0FFFFE7806039B7E4040097C0FFFFED
:106A6000E780E07CC85897800100E780E03A17B5DE
:106A70000100130525E097800100E780E0398327B6
:106A8000840C8545414593E707082324F40C97C0FF
:106A9000FFFFE780E03F8D451305000897C0FFFF2B
:106AA000E780003F97C0FFFFE780E06B37A5070056
:106AB0001305051297C0FFFFE78080679D450145DC
:106AC00097C0FFFFE780806DB7E700E0370700045D
:106AD00023A0E7180100010097D0FFFFE78040EFF7
:106AE00097D0FFFFE780400197000000E780E0EAD1
:106AF00097000000E78080A197000000E78000C1B8
:106B000097E0FFFFE78060F697000000E780A02590
:106B100097000000E780801083A704081705000095
:106B2000130505CB829797D7FF1F238FA78ABC4CED
:106B3000130600648545829797C0FF1FE780408B4E
:106B400001458280AD67371700409387A7AA1CC311
:106B5000B7E700E03707400023A0E7180100010075
:106B6000B7F7070003C70701A5476316F700939718
:106B7000450191C301A04111AE860146AA85254574
:106B800006C697C0FF1FE780C0C5B240B7E700E068
:106B90003707400023A0E710410182804111B286EF
:106BA0002E86AA852D4506C697C0FF1FE78060C3C5
:106BB000B2400145410182809307000463ECC704A1
:106BC0001D71A2CC2A840808A6CACAC886CE32C6BD
:106BD00097800100E7800001AD6737170040938779
:106BE000A7AA1CC3B7E400E03709400023A024197A
:106BF00001000100B2461008A285294597C0FF1F79
:106C0000E78020BEF640664423A02411D6444649BE
:106C1000256182803955828041110D658D4506C6FA
:106C200097C0FFFFE780601CB71700408D6623A662
:106C3000D70A17F5FF1F1305E5B41387C70A938713
:106C4000870A1CC15CC5856689675CC958C114C5C3
:106C500018C9B7E70400B24003A3871E41010283AD
:106C60008145B307B5008387070089E71723000034
:106C7000670023CD8505C205C181E5B797A701004F
:106C80009387475A1357C5003E97034707000111E2
:106C900006CE2304E100135785003D8B3E97034742
:106CA000070023060100A304E100135745003D8BB4
:106CB0003D893E97AA970347070083C7070028002E
:106CC0002305E100A305F10097000000E78080F9AB
:106CD000F24005618280411126C2E97797F4FF1FD7
:106CE0009384C4BA22C49387A7552E842381B40009
:106CF0002E86AA8517F5FF1F130585B906C62390B2
:106D0000F400A381040097800100E780A0ED9305C3
:106D10002400C205C18117F5FF1F130545B7970071
:106D20000000E780808DB38784002382A700218143
:106D3000A382A700930564002244B24026859244B2
:106D4000C205C181410117230000670083BF09C943
:106D50009307800263E6B700170300006700E3F7BC
:106D6000828097F7FF1F83C747B599EF411106C689
:106D700097200000E780C0B4B240854717F7FF1F97
:106D8000230DF7B2410182808280630E0554638C2B
:106D900005545D71A2C4A6C286C6CAC04EDE52DCCE
:106DA00056DA5AD85ED662D466D26AD0B9472A84F7
:106DB000AE8463F9B706394697A501009385852F00
:106DC00097800100E780A0DF31ED8347E4001307DF
:106DD00010036394E702854717F7FF1F2306F7AAFE
:106DE00017A501001305052E97F7FF1F239D07A880
:106DF00097000000E78000E771A01307000317A5C4
:106E000001001305252FE395E7FE97F7FF1F238D5C
:106E100007A697F7FF1F239807A617A501001305DC
:106E2000E52BF9B797F7FF1F83C707A663890722EA
:106E3000BD6AB96B938CFA55014A17FBFF1F130B00
:106E40002B96138CEB65938AFA6605A8B307440169
:106E500083C6070097F7FF1F83D7E7A2B1E3930725
:106E6000A005639BF600854717F7FF1F231DF7A0BA
:106E700097F7FF1F2386D792050A93170A01C1834C
:106E8000E3E697FCB640264496440649F259625A16
:106E9000D25A425BB25B225C925C025D616182808D
:106EA000054D639BA7039307500A639EF60089472D
:106EB00017F7FF1F2319F79C930750FA17F7FF1FC7
:106EC000A300F78E55BF9307A005E387F6FA97F75F
:106ED000FF1F239A079A4DB7138717004207DA97C7
:106EE00041832380D70017F6FF1F231EE6988D47A6
:106EF000E3F4E7F817F9FF1F0349B98A97F7FF1F73
:106F000083C7278A22093369F9009307F9FFC2076B
:106F1000C1839306F00DE3ECF6FA93076900C2070C
:106F2000C183E31BF7F493052900C205C18117F55E
:106F3000FF1F1305058797F0FFFFE780006C3307FD
:106F40002B018347570003474700A207D98F17F744
:106F5000FF1F231A07926319F50E8149630DA901DA
:106F600097F9FF1F83C90984A20997F7FF1F83C7F9
:106F70007783B3E9F90017050000130585DD97F065
:106F8000FFFFE780400563878907636D3C039387B4
:106F9000EB556382F90497F7FF1F83C7A780054766
:106FA0006389E70681CB1387A7051377F70F8D4613
:106FB00063F2E6081307F0072300E100A300F100E5
:106FC00089459DA063829905E39759FD97F0FFFFDE
:106FD000E780E03211A8CA8517E5FF1F1305857CFD
:106FE00097F0FFFFE7802015014597F0FFFFE7804E
:106FF00080FE59B5CA8517E5FF1F1305A57A97F0DE
:10700000FFFFE780E01ECDB797F0FFFFE780E028A5
:10701000E1BF930710F8130511002300F10097F06A
:10702000FFFFE7808034FD450A8597000000E78078
:10703000C0CA5DBFCA8517E5FF1F1305A57697F087
:10704000FFFFE780E0CF4DB79307F00789450A853A
:107050002310F10097000000E78020C831BDBD4734
:1070600063F39722414697A501009385E50A22859F
:1070700097800100E780A0B4631C051417A50100E8
:107080001305C50A97000000E780C0BD17E5FF1F84
:107090000355056F97000000E78080BE97E7FF1F4C
:1070A00083C7475A17A501001305C5FF89E717A530
:1070B00001001305A5FF97000000E780A0BA17A5FF
:1070C00001001305250897000000E780A0B917C547
:1070D000FF1F0355252F97000000E78060BA17A512
:1070E00001001305650697000000E780A0B717E5CB
:1070F000FF1F0355A56597000000E78060B817A53E
:1071000001001305E50497000000E780A0B517D53E
:10711000FF1F0355C5FB97000000E78060B617A569
:1071200001001305650397000000E780A0B317D5A1
:10713000FF1F035585F997000000E78060B417A58D
:1071400001001305E50197000000E780A0B117D505
:10715000FF1F0355A5F797000000E78060B217A551
:1071600001001305250097000000E780A0AF17C5B8
:10717000FF1F0355E51497000000E78060B017A5D6
:1071800001001305A5FE97000000E780A0AD97C79A
:10719000FF1F83C7A720A20717C5FF1F03451520A0
:1071A0005D8D97000000E780A0AD97C7FF1F83C7E4
:1071B000071FA20717C5FF1F0345751E5D8D9700AA
:1071C0000000E780E0AB179501001305E56A0DB1FB
:1071D000414697A501009385A5F922859780010076
:1071E000E780E09D4DE1C114C20493060401C18013
:1071F000510401498D452545154663FC9500639F63
:1072000086001307E9FF4207A1674183F51763FA78
:10721000E70417A50100130525F8D9BE83C70600AA
:10722000138707FD1377F70F637CE5001387F7FBE0
:107230001377F70F636EE600938797FC13F7F70F4A
:1072400012093369E900420913590901850675B726
:107250001387F7F91377F70FE36DE6FA938797FA39
:10726000F1BF97E7FF1F2393274F97D0FFFFE780DA
:10727000C05317A501001305E5F097000000E78053
:10728000609E4A852DBFC147E3FE97BE414697A544
:1072900001009385A5F2228597800100E780209266
:1072A000E31205BE8347040113071003639CE70044
:1072B000854717E7FF1F2303F74E17A501001305A6
:1072C00025F13DB61307000317A50100130545F38B
:1072D000E390E7B297E7FF1F2382074C17A5010051
:1072E000130585F031B68280411126C2AE848D45EA
:1072F00022C406C62A8497C0FFFFE78060B9B7178B
:10730000004099C803A5C70C418D23A6A70CB24025
:10731000224492444101828003A5870C418D23A41D
:10732000A70CF5B78347050003471500A207D98FBF
:10733000C2076177C18713072720639AE700834557
:1073400025003705040017030000670023FA828038
:1073500017E6FF1F1306C6568147B2861303F00FC8
:10736000A9483308F6000348080013F7F70F63072E
:10737000A80C630668008507E39517FF2947B387C4
:10738000E6002380A70097E7FF1F938727545DA897
:10739000411113D765001347170006C693F6350051
:1073A000058B954791CA054699476387C6000946EC
:1073B0009D476383C600A14713F645003336C000DE
:1073C00093F68503050685C2A145638BB604E145A6
:1073D000638AB604930580026388B604930580032C
:1073E0006393B600914697E5FF1F2386F57497E5F2
:1073F000FF1F2381C57497E5FF1FA38DD572BE853E
:1074000017A50100130505E697800100E780E088D5
:10741000B240854717E7FF1FA30FF7704101828035
:107420008546D1B78946C1B78D4675BF17A50100FE
:107430001305C5E5178301006700238617E7FF1FC3
:107440001307C748BA972380B700E147E302F5F472
:1074500093077002E30CF5FC82802A8723800500E5
:10746000814717E5FF1F1305A5451308F00F2946AF
:10747000B306F50083C606006396E60297E6FF1F93
:107480009386C644B69783C7070005452380F50059
:107490009947636EF7029D4763FDE700E147630D7F
:1074A000F7008280638506018507E393C7FC0145E9
:1074B000C5B7238005008280B737004003C7370077
:1074C00083C7050093F70704D98F2380F5008280D6
:1074D0005D7152DC56DA5ED6716A97EBFF1F938BB3
:1074E000AB768D6AA6C24EDE62D486C6A2C4CAC07E
:1074F0005AD866D26AD06ECEC1495E8C97E4FF1F1F
:107500009384843D130A0A20938A7ADC17E9FF1FCB
:1075100003498976B3872B0183C7070093F7F70FD9
:10752000C9EFB787004003C76700058BE310077CEE
:1075300003C76700118BE30D077E83C75700918B4C
:1075400099E36F10200317E7FF1F03470773854771
:107550006304F7006F10400197E7FF1FA38DE75CFE
:1075600097E7FF1F238A074297E7FF1F2388074EED
:1075700097E7FF1F2386075A97E7FF1F2383075AC2
:1075800097E7FF1FA38A074097E7FF1FA388074CD1
:1075900097E7FF1FA386075897E7FF1FA3830758A6
:1075A00097E7FF1FA38A075897E7FF1FA387076C7A
:1075B000B787004011476F0070779307190093F762
:1075C000F70F3D476364F70617E7FF1F2306F76AC7
:1075D00097E7FF1F93874769CA9783C70700130779
:1075E000100293F7F703638EE71E6366F704054402
:1075F0006385871CE38C07620947638EE7101307D6
:107600000002E384E74EB7E700E03707400023A01D
:10761000E71801000100629923000900FD1923A069
:10762000E71093F9F90FE39309EEE5BD97E7FF1F24
:107630002384076471BF130730026388E70C63E893
:10764000E71613074002638CE70A13070003E39C65
:10765000E7FA97E7FF1F93872760CA9703C70700DA
:10766000A1471377F70FE31BF71483C7640097E66E
:10767000FF1F2389F64A97E7FF1F83C7572691C745
:10768000FD5797E6FF1F238FF64897E5FF1F83C539
:10769000B52497E7FF1FA387B74897E7FF1F83C766
:1076A000A72313FB07089306000493F70706639FBD
:1076B000D74C9307A009638DF51663EAB7129307B9
:1076C000F0056386F54A930750096384F52A01445F
:1076D00097E7FF1F83C717451547E392E736B7E7DC
:1076E00000E03707400023A0E71801000100B7863B
:1076F000004023808602130680FC6F00500EFD5769
:1077000017E7FF1F230FF740FDBDFD5717E7FF1FCA
:107710002308F740CDBD17A501001305A5C8977034
:107720000100E780606F97E7FF1F9387E752CA97D2
:1077300003C40700014B97ECFF1F938C6C3213744A
:10774000F40F17AD0100130D6DC663478B04294577
:1077500097700100E7804059854717E7FF1FA30F87
:10776000F72E17E7FF1F230C872E17E7FF1F2305B0
:10777000F73C37E700E0B70640002320D7180100A8
:107780000100378600408347A60293F7370F230591
:10779000F6022320D71085BDB3876C0183C507008F
:1077A0006A85050B97700100E780204F79BF8547F8
:1077B00017E7FF1F2304F72AB9B517E7FF1F1307C1
:1077C000A7494A970347070097E6FF1FA386F61CC1
:1077D00097E6FF1F2383E61C17E7FF1F230EF734EE
:1077E0001DB5854717E7FF1F2308F71A29BD930723
:1077F000400A6389F5349307200B6384F5369307B9
:10780000100AE396F5EC838724000144E3D207ECE9
:1078100097E7FF1F83C7770C93F63700638A061A32
:107820000546638AC62209466395C61A1D4755A2B6
:1078300017E5FF1F0345650AC94797ECFF1F83CC77
:10784000DC0997E5FF1F83C5650917E4FF1F0344A3
:10785000F4086315F510CD476392FC109307700888
:10786000639CF5021307300FB7170E006308E4009E
:107870001307900DB7B704006314E40817E7FF1F60
:107880002328F72ABE8517A501001305A5B2977016
:107890000100E780804025BD93078008639DF500C7
:1078A000B307804013F4F70FB7774600938787CD6F
:1078B000B3D78702E1B793079008639AF500B3073F
:1078C000804013F4F70F91679387C766D5B7930786
:1078D000A008639BF500B307804013F4F70FB717B8
:1078E0003D0093870790E9B79307B008639AF500C6
:1078F000B307804013F4F70F9167938797D04DBF7C
:1079000093F5F5078D47639BF500B307804013F4AB
:10791000F70FB7975B00938707D859BF8947639BD9
:10792000F500B307804013F4F70FB7770B00938788
:10793000071BBDBF8547639AF500B307804013F46A
:10794000F70FDD67938767E3A5B7D28785F9B3079C
:10795000804093F7F70FB3D7FA020DB797000000F6
:10796000E780409FA285668597000000E780809EA3
:10797000B9BB9305610017E5FF1F034505F617E442
:10798000FF1F034494F597000000E78040AD930586
:107990007100228597000000E78060AC3C0017E78B
:1079A000FF1F2321F72A834761002304F100834747
:1079B0007100A304F100894717E7FF1F2304F7169E
:1079C0008357810017E7FF1F2318F7F0094409B315
:1079D000154793F64700B336D00093F78703850623
:1079E00085C32146638BC7066146638AC7061306B3
:1079F00080026388C706130680036393C70091471C
:107A000017E6FF1F2308D61297E6FF1FA384F6127E
:107A100097E7FF1F2381E71217E7FF1F034707ECD4
:107A20009376070497E7FF1F83C757EB8DEE137715
:107A3000770C93067008630CD7021377F7078D460F
:107A40006312D70CB307F040B7955B0093F7F70FBD
:107A5000938505D849A81947ADBF854755B78947CC
:107A600045B78D4771BF930670086311D70213079E
:107A7000300FB7150E006389E7021307900DB7B5F5
:107A800004006383E7021307700845BF9306800C68
:107A90006311D702B307F040B775460013F7F70F2D
:107AA000938785CDB3D5E70297E7FF1F23A2B708D9
:107AB000D9BB9306900C631CD700B307F04093F535
:107AC000F70F91679387C766B3D5B702F1BF9306E7
:107AD000A00C631DD700B307F040B7153D0093F726
:107AE000F70F93850590B3D5F5027DBF9306B00CD3
:107AF000E315D7F4B307F04093F5F70F9167938739
:107B000097D0D9B78946631BD700B307F040B77544
:107B10000B0093F7F70F9385051BF1B78546631AA2
:107B2000D700B307F040DD6593F7F70F938565E362
:107B30005DBFD28535FBB305F04093F5F50FB3D5A6
:107B4000BA029DB783C72400C18B99C7854717E741
:107B5000FF1F230CF7FCA5BE97E7FF1F238707FC39
:107B6000BDB6854717E7FF1FA307F7FC8DB63C009E
:107B700017E7FF1F2328F70C094793070003231477
:107B8000F10097E6FF1F238FE6F82DBD639407569B
:107B9000A94763E5B742179701001307E7698A050C
:107BA000BA959C41BA97828717E4FF1F0344F4D229
:107BB000894C6306940D63E68C0685476303F408DD
:107BC0009307F00F17E7FF1F0347C7F563F6E700BA
:107BD00017E7FF1F2308F7F497ECFF1F83CC8CF403
:107BE0009307000413F4FC0F63F4970113040004DB
:107BF00097E7FF1F9387070503AD070022862685B9
:107C0000EA85B38C8C40229D97700100E78080FD4F
:107C100097E7FF1F238897F197E7FF1F23A4A70388
:107C200045BC8D47630CF40A9947E31BF4F897971A
:107C300001009387E76617E7FF1F2325F700A94791
:107C400051B717E7FF1F0347470397E7FF1F9387C6
:107C500067EF4946979501009385856D6306870018
:107C6000979501009385C5683E8597700100E78070
:107C700060F717E7FF1F2327A7FCC947A1B797E6BF
:107C8000FF1F83C686FF054797E7FF1F938787EB94
:107C90006394E6023E851306700297950100938572
:107CA000A56697700100E780E0F317E7FF1F232B1D
:107CB000A7F89307700239B73E85130630049795ED
:107CC00001009385A55E97700100E780A0F117E79A
:107CD000FF1F2329A7F693073004EDB597E5FF1F93
:107CE00083C5A5BF179501001305056E97700100A8
:107CF000E780A0FA054D97EDFF1F83CD0DF897E5BE
:107D0000FF1F83C585BD179501001305E56B6398BB
:107D1000AD0B97700100E78040F897E7FF1F83C71E
:107D2000C7BBB5CBE36EF4E8179401001304846479
:107D3000638CB701179401001304446463869701B0
:107D40001794010013040465228597700100E780F1
:107D5000E00D1375F50F93071500860717E7FF1F52
:107D60002302F7DE8D4717E7FF1FA30DF7DC97E728
:107D7000FF1F938727DD0147BE861376F70F89071C
:107D80006365A60297E7FF1F23AED7EA97E7FF1FB9
:107D900083C747DB05BD979701009387A75617E771
:107DA000FF1F2321F7EA914731BD3306E400034664
:107DB0000600A380070005072380C7007DBF9770DA
:107DC0000100E78080ED97E7FF1F83C707B1E1D788
:107DD000E368F4DE179401001304C456638CA70112
:107DE00017940100130484566386970117940100C9
:107DF00013044457228597700100E7802003137510
:107E0000F50F93071500860717E7FF1F230CF7D21E
:107E10008D4717E7FF1FA307F7D297E7FF1F938749
:107E200067D20147BE861376F70F8907E37CA6F475
:107E30003306E40003460600A380070005072380FD
:107E4000C700D5B797E5FF1F83C525A91795010082
:107E50001305455897700100E78020E497E7FF1F5E
:107E600083C717CE93E7470017E7FF1FA30AF7CC96
:107E700083C7240017E7FF1FA302F7CC89B8179523
:107E800001001305655697700100E780E0F897E759
:107E9000FF1F9387A7CA83C7070017E7FF1F230D9C
:107EA000F7A217E4FF1F0344E4C7333480000DB08A
:107EB000179501001305855497700100E780C0F500
:107EC00097E7FF1F83C7D7C793E7070117E7FF1F90
:107ED000A308F7C683C7240017E7FF1F2300F7C6D0
:107EE0006FF0EFFE179501001305855297700100A2
:107EF000E78080F203C704007D8B51EFB787004015
:107F000003C767021377C70B136727002383E702B2
:107F100003C7A7021377C70B136727002385E70260
:107F200003C7E7021377C70B136727002387E7020E
:107F300003C727031377C70B136727002389E702BB
:107F4000854717E7FF1F2309F7A417E7FF1F23073C
:107F5000F7B017E7FF1F2305F7BC17E7FF1F230242
:107F6000F7BC97E7FF1FA38907A297E7FF1FA38727
:107F700007AE97E7FF1FA38507BA97E7FF1FA38206
:107F800007BA97E7FF1FA38907BA97E7FF1FA386E2
:107F900007CE6FF0CFF389476312F70297E7FF1F11
:107FA00083C7C7939146638CD70863E0F604638E5A
:107FB000E70C6369F70A05476380E70EFD5717E78B
:107FC000FF1FA301F7B637074000B7E700E023A083
:107FD000E71801000100B78600401306F0FC23817A
:107FE000C60223A0E7106FF00FE213072008638298
:107FF000E7086362F70213071008E391E7FC37878D
:1080000000408347670293F7C70B93E727002303DA
:10801000F7026FF0CFEB130730086389E70213070D
:108020004008E39DE7F8378700408347270393F72D
:10803000C70B93E727002309F7026FF04FE9378753
:1080400000408347270393F73707F5B7378700408A
:108050008347E70293F7C70B93E727002307F7024D
:108060006FF0EFE6378700408347E70293F7370763
:10807000F5B7378700408347A70293F7C70B93E70D
:1080800027002305F7026FF08FE43787004083470E
:10809000A70293F73707F5B7378700408347670292
:1080A00093F73707ADB7179501001305653797703C
:1080B0000100E78060D697E7FF1F238F0780D5B3C5
:1080C000179501001305C53697700100E780C0D4ED
:1080D00097E7FF1F2392078097E7FF1F938787A4E7
:1080E00003C40700894763F3870009441374F40F3E
:1080F0006FF00FDE13070002E392E7EC631B0B0A3D
:10810000638FF500930720026383F508179501003C
:108110001305853597700100E78020B845B51795A0
:1081200001001305A53197700100E780E0CE0144FE
:10813000179D0100130DCD31A14CB387840083C579
:1081400007006A85050497700100E78000B5E31613
:1081500094FF178501001305257897700100E780CB
:10816000A0CB17D4FF1F0344647701E897D7FF1F04
:1081700023860774014B6FF0AFD58947E310F4E411
:10818000854717D7FF1F230BF7726FF04FD417D611
:10819000FF1F0346967497D5FF1F83C50574179577
:1081A00001001305652B97700100E78000AF6FF0A9
:1081B0000FD26380F50693071002E399F5F497D583
:1081C000FF1F83C5A571179501001305E52A977058
:1081D0000100E78080AC97E7FF1F23A597A697E7EC
:1081E000FF1F9387E794944383D7470017E7FF1F48
:1081F0000347679417D6FF1F2320D66E1D4497D6DA
:10820000FF1F239DF66C97D7FF1F238AE76C6FF043
:108210002FCC97D5FF1F83C5656C179501001305FB
:10822000252797700100E78040A797D7FF1F238776
:10823000076897D7FF1F2391076A6FF02FF925472B
:10824000638FE7C89946378700406394D7022300BD
:108250008702B7E700E0B706400023A0D718010067
:108260000100130600FC2301C70223A0D7106FF002
:108270008FB99306100A639FD70023008702B7E7E0
:1082800000E0B706400023A0D71801000100130644
:1082900080FCD1BF9306A009E381D7FE9306400A74
:1082A000E38DD7FC93062002639DD700B7E700E07B
:1082B000B706400023A0D718010001002300870261
:1082C000F9B78546E384D7FE93070008E300FBFE79
:1082D000B7E700E0B706400023A0D718010001006F
:1082E000130620FC23008702BDBF17E7FF1F0347CB
:1082F00077836302F71E63E7E70295476300F71091
:108300009947630AF704B786004023800602B7E75F
:1083100000E03707400023A0E71801000100130622
:10832000A0FC75B99307F005630AF700930750099D
:108330006306F70093071002E317F7FCB7E700E0C6
:108340003707400023A0E71801000100B78600406E
:10835000130620FC69B117DBFF1F034BAB7C9307AF
:1083600000045A8D63F46701130D000497E7FF1FA3
:108370009387478D83AC07001374FD0F2286E68533
:10838000268597700100E780E085B3078B406694EF
:1083900017D7FF1F2308F77897E7FF1F23A4878AC3
:1083A000B7870040630C0B022380A703B7E600E009
:1083B0003706400023A0C6180100010003C72702AA
:1083C000134707042381E70203C727021377C70F68
:1083D0002381E70223A0C6106FF0EFA223800702DB
:1083E00037E700E0B70640002320D718010001005E
:1083F000130620FC2381C7026FF0AFB93787004016
:108400008347370097D6FF1F83C6567393F7070835
:10841000D58FA301F700B7064000B7E700E023A01F
:10842000D718010001001306A0FC35BD97E7FF1F18
:1084300093878782CA9783C7070093F7F70FC1CF47
:1084400097E7FF1F83C76783D9E717D7FF1F034746
:10845000776D930700026310F70883AD040017DD02
:10846000FF1F034DAD4797DCFF1F83CC3C4717DB55
:10847000FF1F034BCB46E6876A87DA866E8697D561
:10848000FF1F83C5A543179501001305E5019770EC
:108490000100E780808097D7FF1F23ABB76997D78C
:1084A000FF1F2389A76997D7FF1FA385976997D7D0
:1084B000FF1F2382676997D7FF1FA3808740B7E715
:1084C00000E03707400023A0E71801000100B7864D
:1084D00000406FF04FA2B7E700E03707400023A04D
:1084E000E71801000100B786004015BD97D6FF1FB1
:1084F00083C6A6780547639CE60429472381E702E3
:1085000009472383E7022385E70297D7FF1FA38547
:10851000076297D7FF1FA3820776B7870040A38122
:10852000070017D7FF1FA30B076005472383E7004A
:10853000B640264496440649F259625AD25A425BE2
:10854000B25B225C925C025DF24D616182802947E0
:108550002381E70209472383E7022385E702238774
:10856000E7022389E70255B717D7FF1FA307F734A0
:108570006FE01FFF854717D7FF1F230FF74017D75F
:10858000FF1F230DF74C17D7FF1F230BF75817D7E3
:10859000FF1F2308F7586FE0BFFE854717D7FF1F5F
:1085A000230CF73E17D7FF1F230AF74A17D7FF1FE1
:1085B0002308F75617D7FF1F2305F75617D7FF1FB6
:1085C000A30C073C17D7FF1FA30A074817D7FF1FA5
:1085D000A308075497D7FF1FA38507548280411132
:1085E00006C697000000E78080FBB7870040238025
:1085F0000700130740FC2386E7001307C004A38687
:10860000E70017D7FF1F1307272D2398E70017D779
:10861000FF1F13076730239AE70017D7FF1F1307C1
:10862000E73B239CE70017D7FF1F13076747239EED
:10863000E70029472381E70209472383E7022385CF
:10864000E7022387E7022389E702A3810700930655
:1086500000F8A380D700930690022380D700FD5630
:108660002383D7002381E7009306000537E700E066
:10867000230BD740B70640002320D71003C71700AD
:1086800013671700A380E700B24097D7FF1F239717
:10869000074A41018280411106C697000000E78029
:1086A00000F0B787004023800700130700FC2386F3
:1086B000E7003147A386E70017D7FF1F1307C7213D
:1086C0002398E70017D7FF1F13070725239AE70012
:1086D00017D7FF1F13078730239CE7002947238103
:1086E000E70209472383E7022385E702A381070006
:1086F000930600F8A380D700930690022380D7004A
:10870000FD562383D7002381E7009306000537E752
:1087100000E0230BD740B70640002320D71003C743
:10872000170013671700A380E700B24097D7FF1F19
:108730002396074041018280F1679387072017D76E
:10874000FF1F2327F73E854717D7FF1F2314F73E48
:10875000A14717D7FF1F2300F73E97D7FF1FA38C12
:10876000073C97D7FF1F2389073C97D7FF1F238715
:10877000071497D7FF1FA3820714814717D5FF1F40
:1087800013050514FD5517D6FF1F13062614294798
:10879000B306F5002380B600B306F600238006007A
:1087A0008507E397E7FE97D7FF1FA38E073697D776
:1087B000FF1FA38C073697D7FF1F2387073697D74E
:1087C000FF1F2382073697D7FF1F2381073697D7CE
:1087D000FF1FA38B073497D7FF1F238807348147D8
:1087E00017D6FF1F130646464147B306F6002380FF
:1087F00006008507E39BE7FE828017D7FF1F03472C
:10880000C74785476316F700170300006700E3E8D2
:10881000170300006700E3DC411122C406C617D726
:10882000FF1F0347874585472E8613F4F50FAA855A
:108830006317F70417D5FF1F1305451E9760010046
:10884000E780403A97D7FF1F238A0720B787004069
:1088500023848702B7E600E03706400023A0C6184D
:108860000100010003C7A7021377C70F2385E702A2
:10887000B240224423A0C61001454101828017D591
:10888000FF1F1305650D97600100E780A03597D79E
:10889000FF1F23830710B787004023828702B7E6B4
:1088A00000E03706400023A0C6180100010003C7FE
:1088B00067021377C70F2383E7025DBF411106C626
:1088C00097000000E78080E7B240410117030000F5
:1088D0006700E3F2411106C697F0FFFFE78080BF13
:1088E00097D7FF1F83C7570BA1CB97D5FF1F83C512
:1088F000C50A89C917D5FF1F1305450A97E0FFFF71
:10890000E780E04897D7FF1FA388070897D7FF1F86
:108910002384072237E700E0B70640002320D7185A
:1089200001000100378600408347660293F7370F46
:108930002303F6022320D710B2404101828041C9AF
:10894000D9C597D7FF1F83C7671FD1C3011122CC99
:108950004AC84EC656C25AC006CE26CA52C42E892E
:10896000AA890144930A0004371B03006377240398
:10897000B3078940C207C183BE8463F4FA0093043D
:108980000004C204C180130A1BD497D7FF1F83C7FA
:10899000A7009DE37D1A631C0A00F2406244D244A2
:1089A0004249B249224A924A024B0561828097F0BD
:1089B000FFFFE78020B2D1BF338589002694A685CA
:1089C000420497000000E78060E5418045B782805F
:1089D000411106C622C429C12E8495C997D7FF1F0D
:1089E00083C7C71595CB97D7FF1F83C7E7FA8DC7F6
:1089F00013070004AE876374B70093070004139451
:108A000007014180A28597000000E78020E12285D0
:108A1000B2402244410182800144D5BF97D7FF1F55
:108A20009387472918429C4383D645000345070096
:108A300083C5C700035646006396A50083D5E700AB
:108A4000638DD502011106CE2386A7002397D70098
:108A5000B705CF00DC4B9385757D05077D162EC2CB
:108A6000230001003AC42316C1002317D10099C383
:108A70000A858297F240056182808280DC4DDC4B62
:108A800081CFB7E70400904503A38705914517D52B
:108A9000FF1F03456522028382806D713C083EC63C
:108AA000B707E500232291103EC8AA843C0832850E
:108AB000232611103ECA23248110232021112E8940
:108AC00097300000E780C0672A849795010093855E
:108AD00025A1177501001305A57B97600100E780AC
:108AE000C01BA28517950100130505B09760010012
:108AF000E780A01A294597600100E780E01EB705CE
:108B0000CB009385757D680097100000E780406D6D
:108B1000A285680097300000E780E0540147814655
:108B20007000CA85268597200000E780C09005CD9B
:108B30002A84979501009385A59A1775010013055E
:108B4000257597600100E7804015A2851795010003
:108B5000130545AA97600100E78020142945976016
:108B60000100E78060188320C11003248110832452
:108B70004110032901105161828097D7FF1F93870D
:108B8000671318429C43797122D406D60348070024
:108B900083C807012A8483D645000355460063969F
:108BA000080183D82701638DD802238807010507B0
:108BB0002399D7003708CC00DC4B1308787D3ACCDA
:108BC0001307F5FF42CA23080100231EE100231FFB
:108BD000D10099C7080832C62EC482973246A245F2
:108BE000228597000000E78080EBB2502254456157
:108BF00082806D713C083EC0B707E5003EC23C086C
:108C00003EC4232611102324811023229110231700
:108C100001002318010023190100231A0100231B5E
:108C2000010097A7FF1F83D7A77E99E3C167FD17B0
:108C30002316F10097A7FF1F83D7A77D91EB97D746
:108C4000FF1F938727079C439C43DC4783D707007C
:108C500017A4FF1F1304C47B584C2317F10083573C
:108C60004400484B2318F10031E1979501009385AA
:108C7000258E177501001305A56197600100E78037
:108C8000C001179501001305E58D97600100E7808D
:108C9000C000294597600100E78000058320C110CE
:108CA00003248110832441105161828097A7FF1F04
:108CB00083C7777689EBB7E70400BC5782975C4C93
:108CC00023AA0700E1BFFD1797A6FF1FA385F6742F
:108CD00003560701834704014C470A85230BF10023
:108CE00097300000E780403597D7FF1F938787FCB8
:108CF0009C430147814688430A866C009710000018
:108D0000E7806073AA8429C1979501009385458403
:108D1000177501001305C55797600100E780E0F75C
:108D2000A685179501001305A58497600100E780CB
:108D3000C0F6294597600100E78000FB584CB7E773
:108D40000400BC57484B9DBF97A7FF1F83C7B76C54
:108D5000F5D7B7E70400BC4F1044854517D5FF1F72
:108D6000034585F582971DBF5C4EDC4BB9CFB1CD75
:108D7000411122C417750100130585512E84978572
:108D800001009385257B06C697600100E780E0F02F
:108D9000A285179501001305658097600100E780A3
:108DA000C0EF294597600100E78000F4B7E70400B1
:108DB0002244B24003A3870517D5FF1F0345C5EF23
:108DC000130640069145410102838280411122C46D
:108DD00017A4FF1F130484611C4C06C689C7DC431B
:108DE00099C34C488297584CB7E70400BC57484B8E
:108DF00082975C4CB240224423AA07004101828042
:108E000017A7FF1F13078760834707009306F00B20
:108E1000850793F7F70F63E9F60097A6FF1F2387EF
:108E2000F65E034507008280930700F8FDB783577D
:108E300045006386071001114AC817A9FF1F1309CF
:108E4000295D52C4032AC90106CE22CC03274A0158
:108E500026CA4EC656C2F15735E31307D00DFD574B
:108E6000636EC704B7E9040083A709072A841305C2
:108E7000860042054181B284AE8A8297232AAA00E5
:108E80000325C9015C49A9E7978501009385856899
:108E9000177501001305C53F97600100E780E0DF0B
:108EA000178501001305C57797600100E780E0DEB4
:108EB000294597600100E78020E3DD57F2406244D6
:108EC000D2444249B249224A924A3E850561828093
:108ED00093874400B705CF002319F5009385757D6E
:108EE000310597100000E780A02F0325C9018345B5
:108EF0006400310597300000E780E0160325C901C2
:108F00002686D685310597300000E780E01271464D
:108F1000A2854A8597600100E780C0CC504419CAF9
:108F200083A78905854517D5FF1F0345E5D8829797
:108F3000814769B797000000E780E0CBD5BFFD57B8
:108F40003E858280411126C297A4FF1F9384444C22
:108F5000D84C22C437E404003C54484B06C68297E0
:108F6000DC4C0323C4052244B240924423AA0700E8
:108F700017D5FF1F034545D48545410102834111A3
:108F800026C297D4FF1F9384E4D29C4006C622C415
:108F90004AC0D5C3DC43C5C35CC12300B5002A84E5
:108FA0009785010093854552177501001305452EDD
:108FB00097600100E78060CE294597600100E78057
:108FC000A0D29C4023A4070023A2070097A7FF1F5D
:108FD0009387C741DC4FDC4B91C7295597000000B0
:108FE000E78000DF97A7FF1F93878742DC4FDC4BAA
:108FF00089C797000000E78020F537E90400832740
:10900000C905894517D5FF1F034505CB82978327DF
:10901000C905914517D5FF1F034505CA82979C4096
:1090200003A347016309030022852244B24092440E
:10903000024941010283B240224492440249410163
:1090400082800111328506CE22CC26CA2E8497302A
:109050000000E780E00EAA84978501009385054A09
:10906000177501001305C52297600100E780E0C273
:10907000030784000356640083554400A6861785C1
:1090800001001305A55397600100E78000C1294541
:1090900097600100E78040C597A7FF1F83C767352A
:1090A000639D9700014597000000E78060D28145ED
:1090B0000A8597000000E780C0ECF2406244D24489
:1090C000056182806D7123248110232611102322D3
:1090D000911093F745002E84638707143C083EC027
:1090E000B707E5003EC23C083EC423170100231821
:1090F000010023190100231A0100231B010097A777
:10910000FF1F83D7A72E99E3C167FD172316F10030
:1091100097A7FF1F83D7A72D91EB97D7FF1F9387A3
:1091200067B99C439C43DC4783D7070017A7FF1F01
:109130001307C72B2317F100544F835747002318F9
:10914000F100DC4AA1E7978501009385653F17751B
:1091500001001305E51397600100E78000B417854F
:1091600001001305254097600100E78000B3294501
:1091700097600100E78040B7134544008320C11089
:1091800003248110832441105161828097A7FF1F1F
:1091900083C737262555D9C3FD1717A6FF1FA30A76
:1091A000F62403D6060183470701CC460A85230B24
:1091B000F10097300000E78020E897D7FF1F9387E2
:1091C00067AF9C4317A7FF1F13074722978601002D
:1091D0009386463C88430A866C0097100000E7801F
:1091E0008025AA8451D99785010093856535177527
:1091F00001001305E50997600100E78000AAA68534
:10920000178501001305C53697600100E780E0A8C7
:10921000294597600100E78020AD26859700000072
:10922000E78000BB91BF93F725009DC7B7E7040017
:10923000BC47414681452808829725559700000084
:10924000E78000B928089305F00F97000000E78039
:1092500040D3134524001DB793F71500014599DF4E
:1092600097000000E78020991345140001BF5C4D72
:10927000411106C688C317D7FF1F232DF7A2B7E7F2
:10928000040083A70708170500001305E5E382978C
:10929000B24097D7FF1F2381A7A2014541018280D9
:1092A00001113335A000A307A100B7E7040083A78D
:1092B000471706CE1306F1008545130550308297F7
:1092C000F240056182808280411122C406C697D790
:1092D000FF1F83C7E79F014489EF97B7FF1F83C72D
:1092E00037F6054499E717B4FF1F034464F51344A8
:1092F0001400228597000000E780C0FA178501005E
:109300001305053D09E4178501001305653D224459
:10931000B24041011763010067002398797122D49C
:10932000A30F010037E404008327841726D24AD014
:1093300006D6AA842E89130550309305F10132C652
:10934000829732468347F10193150601C18185CB8F
:1093500001452EC697000000E780C0F4832744171C
:10936000B2454A8626858297054597000000E7802A
:1093700060F3B2502254925402594561828083278F
:1093800044174A8626858297EDB7411193970501C8
:1093900022C406C626C2C1872E8463D40702B7E45E
:1093A0000400FC5417A5FF1F03458509829719C1C6
:1093B000BC5482972165218DB240224492444101E0
:1093C000828093F715008DC7B7E7040083A7471A7B
:1093D00017A6FF1F1306C60597D5FF1F9385858E19
:1093E00017A5FF1F0345C505829713451400E9B76C
:1093F00093F7250099CFB7E70400BC4F130600642C
:10940000894517A5FF1F0345A5038297134524002F
:1094100065B793F7850085CF97D7FF1F83C7078C64
:1094200085E7B7E7040003A8871A1307401F97A72B
:10943000FF1F83C7E700814613064006994517D5ED
:10944000FF1F03552589029813458400B5B793F78C
:1094500045000145B5D3B7E4040083A7041817D528
:10946000FF1F035525878297BC4C13060064914566
:1094700017A5FF1F0345C5FC8297134544002DBF68
:1094800097D7FF1F83D707856398A70217D7FF1FBA
:109490002313B78417D7FF1F2310C78417D7FF1FC5
:1094A000231DD7822E86178501001305E529BE8569
:1094B000175301006700637E178501001305452AD5
:1094C00017630100670043950357450097D7FF1FB7
:1094D00083D74780631EF704C1674111F91722C47F
:1094E00017C7FF1F2328F77E37E4040097C7FF1F25
:1094F00023A4077E97C7FF1FA38C077C97C7FF1F76
:10950000238E077C7C4C06C6894517A5FF1F0345A3
:1095100025F382977C4C914517A5FF1F034545F223
:1095200082972244B240410117030000670003DA2A
:10953000178501001305C522176301006700C38D5D
:109540007D15954763E2A71C178701001307C7160F
:109550000A053A951C41011122CC06CEBA972E84F9
:109560008287178501001305252097600100E78099
:10957000A08AA1A203C7250099476311F7022E858F
:1095800097000000E78080F48345640017850100A0
:109590001305851E97500100E780207097B7FF1FC5
:1095A000238007CA178501001305C51E7DBF03C7A9
:1095B000250095476319F702C16717C7FF1F0357B7
:1095C0006771F91703D5A5006309F702B7E704002F
:1095D00083A7C7178297178501001305A51C9760FD
:1095E0000100E7806083854717B7FF1F230AF7C490
:1095F000178501001305851D8DBF97C7FF1F239B8E
:10960000A76C83D7E50097C6FF1F2396F66C83D718
:10961000050197C6FF1F2391F66C83D7250197C6D6
:10962000FF1F239CF66A97C7FF1FA383076A631B6C
:10963000E502B7E70400BC4F096613060690A14592
:1096400017A5FF1F0345C5DF82970356E400835526
:10965000A400178501001305251697500100E78027
:10966000C06351B79307700F2316F100B7E70400EA
:1096700083A7870D17A6FF1F034686DC6C00829721
:109680004DF9854717C7FF1FA304F7645DB717851A
:10969000010013056514D1BD83C525009147639270
:1096A000F502178501001305A51497500100E78006
:1096B000A07697000000E78060C1F2406244056137
:1096C000828099476392F502228597000000E78027
:1096D000E0DF83456400178501001305E509975015
:1096E0000100E780805BD1BF9547639AF50083470F
:1096F0001400E1F3178501001305C511BDB51785E9
:1097000001001305A511E1BF82800111B7F5070023
:1097100030008146E105194506CE9790FF1FE7808E
:10972000400C8347C1000347D100B7562D47A2071D
:10973000D98F938676D517A7FF1F1307A7D114C318
:10974000B736302D9386360354C395669386767468
:109750002314D7009306D0022305D70013D6C700E1
:1097600097860100938606FB36960345060013D6BE
:1097700087003D8A36968345060013D647003D8A0A
:10978000BD8B3696B69783C607000346060097A79B
:10979000FF1F9387A7CDA305A7002306B700A30645
:1097A000C7002307D700A3070700A386A7002387C6
:1097B000B700A387C7002388D700F24005618280E5
:1097C000411106C697000000E78060F4B7E7040087
:1097D00083A7871417A6FF1F1306C6C7D5450145E3
:1097E0008297B240694697A5FF1F938525C8130548
:1097F0007030410117030000670083B261712324B8
:10980000811A37E40400832704082326111A23222F
:10981000911A2320211B232E31191705000013054F
:1098200005B7829717A9FF1F130989C19947854476
:109830002300A900231CF10097850100938585EC86
:109840009307400617750100130585A4231CF10832
:109850002308910097C9FF1F938989F2975001004F
:10986000E780A04383D5090017850100130585E82B
:1098700097500100E7806042294597500100E7803A
:10988000A04603D50900896997000000E78020E819
:109890008327441710088545130550308297832786
:1098A000441717A6FF1F130666BCE9451305703061
:1098B00082978327441717A6FF1F1306A6B8B5453E
:1098C00013056030829783274417300889451305B4
:1098D00010318297832744173009894513052031B9
:1098E000829783274415938509900D458297832796
:1098F00044159385099011458297A305910023068D
:10990000910002CD23080100230C01008327841657
:1099100030099145130570408297832784161306FA
:10992000B100854513050040829783278416700097
:109930008545130510408297832784163008854596
:109940001305204082978327841610088545130548
:1099500050408297832704157D55829783274413AF
:109960007D5582977D5597A0FFFFE78060D08327C4
:10997000440C829797A0FFFFE780C0AB8327841435
:1099800017A6FF1F130606ADD545014582978947E7
:109990001306700F814528092306F1009780FFFF09
:1099A000E780E0768D471306000881452808230CE0
:1099B000F1089780FFFFE78080759147230CF10045
:1099C000976701009387477E984383C747003AC84B
:1099D000230AF10097D0FFFFE780C0A37000854500
:1099E000054597A0FFFFE780C0CF30099305700FB2
:1099F000094597A0FFFFE780C0CE30089305000817
:109A00000D4597A0FFFFE780C0CD10089545114593
:109A100097A0FFFFE780E0CCC16717C7FF1F1307C0
:109A2000672BF9171CC32322070017A5FF1F130577
:109A3000E5A097A0FFFFE780A0C98327C41D17C535
:109A4000FF1F1305A52782973C480345090085455C
:109A500082978320C11A0324811A8324411A03297F
:109A6000011A8329C1195D618280C16717C8FF1F70
:109A700003584826F9176301F8083DCDB5CD01110B
:109A800026CAB7E4040083A7841222CC2E862315AD
:109A9000B10006CE2A8401478146ED454285829772
:109AA0002AC611ED17850100130505C8975001005E
:109AB000E7808036F2406244D24405618280FC44F3
:109AC0000356A100A28582972C0017C5FF1F0355DE
:109AD000652097A0FFFFE78060CC69DD1785010056
:109AE0001305C5C597500100E780003383A7C41252
:109AF000ED45280082977DBF82800DC5854717A759
:109B0000FF1FA306F79497A7FF1F238307943546EB
:109B100097A5FF1F93850593130560301703000079
:109B20006700038097A7FF1FA3830792E9BF97C72A
:109B3000FF1F83C7A71AA9EFC16717C7FF1F0357E6
:109B40006719F9176306F7044111854722C417C73F
:109B5000FF1F2305F71837E404007C4C06C6A14517
:109B600017A5FF1F0345C58D82970323841A22443E
:109B7000B24097A7FF1F83C7A78C17C5FF1F0355C8
:109B800065151307401F81463146994541010283FF
:109B900082806D71232481102326111023229110BD
:109BA000328401CD8947630AF5028320C110032462
:109BB00081108324411051618280178501001305B3
:109BC000A5C6AE8497500100E7800025A2852685B2
:109BD00097C0FFFFE780C0A2C9BFB7E70400FC47FA
:109BE00028008297178501001305C5C4975001000E
:109BF000E78080228347810039C41307000B63800C
:109C0000E7021387A7051377F70F8D4663EDE6028A
:109C1000A285280097C0FFFFE780801279B78547AB
:109C2000E3F587F883459100177501001305459901
:109C3000B335B00097A7FF1F2388B748975001009E
:109C4000E780A0059DB703479100A207D98F35672C
:109C50001307D7556385E7086368F7022D67130775
:109C6000B7556387E70631671307C755638AE7046B
:109C700029671307A7556394E702A285280097C0B8
:109C8000FFFFE780404A15B739679306E7656381B0
:109C9000D70863E9F6001307E7556384E706A28552
:109CA00028003DB73D679306F755638AD70613072B
:109CB000F766E396E7FE97C0FFFFE7804064F5B5DF
:109CC0000146A285280097C0FFFFE7800033F1BD61
:109CD000A285280097C0FFFFE7802043F9B5894798
:109CE000E3F587EC97000000E780A0E49305E4FF2C
:109CF000C205C1811305A1009790FFFFE780A04C2A
:109D00006DB5A285280097C0FFFFE780C04271BDF6
:109D1000A285280097C0FFFFE780804D79B597C0E6
:109D2000FFFFE780805751B5C16717C5FF1F035577
:109D300065FAF9176307F500B7E7040003A3C7172F
:109D400002838280854717C7FF1F2303F7F8014569
:109D500017F3FFFF670003551783FFFFE702833602
:109D60002A8408452E89B28919C900C197150000B7
:109D70009385A586610597300100E7802005814421
:109D80007D5A97100000E780E03963C7A40481443E
:109D900097100000E780003A63C8A40497C7FF1F2C
:109DA000938707F49C43DC47B307F940918723026C
:109DB000F400638309048327C900B307F44095873F
:109DC000A302F4001C4C89C79C4799C32285829743
:109DD0001783FFFF670043325C4413971400850428
:109DE000BA972390470171BF1C481397140085044C
:109DF000BA972390070069BF832789000547B307F7
:109E0000F4409587A302F40083570400638EE702B1
:109E10008DC309476384E7040D47E395E7FA978705
:109E200001009387E7F31CCC97870100938747F4E1
:109E300011A897870100938727BA1CCC9787010048
:109E4000938787BA5CC8BDBF978701009387C7A572
:109E50001CCC97870100938727A6EDB79787010051
:109E60009387C7F41CCC97870100938727F5D9BF48
:109E700095E51783FFFFE7028326004618448347D2
:109E8000940075839D8B6317F70097100000E7809F
:109E900060B448C41783FFFF6700A326828017833E
:109EA000FFFFE702232213893500C16442094111F3
:109EB000AA890144F11413590901054A2EC69710C5
:109EC0000000E7802026B2456348A4000145410117
:109ED0001783FFFF6700432283A7090013171400AD
:109EE000BA9783D707006388B700639497006374B9
:109EF0002A010504E1B70545D9BF1783FFFFE70233
:109F0000831BAA892E89328BB6843A8ABE8A97A08F
:109F10000000E780C0FE71C9268597200000E78019
:109F2000C00C8D4763E7A7007D551783FFFF6700CF
:109F3000031C83DB440097100000E780A0242A84E0
:109F400097100000E78040259307740031443305E3
:109F5000850263CDA70297100000E780A02297102A
:109F60000000E78020222A8497100000E780C022AA
:109F70009307740031443305850263C3A704971027
:109F80000000E78020209307450029A897100000D3
:109F9000E7808020330585021307F0179307C01769
:109FA000E35FA7FA2D55E3C277F963040B02D68667
:109FB0005286A6854A8597200100E780C0BDB5B7C7
:109FC00097100000E780401D330585029307C5FF09
:109FD000D1BF832749001385C90083D52700970087
:109FE0000000E78000EC61F581B769553DBF97C778
:109FF000FF1F2399A7CE97C7FF1F938767CE904374
:10A0000081470C463307F500420741836393B7004D
:10A0100082805446139847008507C2962390E60035
:10A02000D5B797C7FF1F9387A7CB9C4303C587006E
:10A03000828017C5FF1F0355E5CA82801783FFFF83
:10A04000E702E309C1671387D7FF630BE502636A81
:10A05000A700F1176300F50201451783FFFF6700B2
:10A06000430A1387E7FF6302E502FD171D8D1335D1
:10A070001500E5B797500000E780602A7D15C5BF41
:10A0800097500000E780E0FED5BF97500000E780C2
:10A0900000FDEDB71783FFFFE70263044111AA84B7
:10A0A00001442EC697100000E780C008B2456348FF
:10A0B000A400014541011783FFFF670083049C480A
:10A0C000131514003E9583570500E385B7FE05047C
:10A0D000C9BF03485500814693F7F60F63E50701B2
:10A0E00081473E858280584593975600BA9703D79B
:10A0F00027006316B70003D70700E304C7FE8506F1
:10A10000E1BF8346450001479377F70F63E4D7002B
:10A11000814711A81C45131657000507B29703D6AF
:10A120000700E313B6FE3E8582801783FFFFE70238
:10A1300063F993170501C18797CAFF1F938A4ABA2B
:10A14000635BF00883A70A00C0479C4703570400DD
:10A15000198D420541816368F5000144228517830A
:10A16000FFFF670063F912052A94CDBFDC47139403
:10A170004900014A3E94834744006341FA02014A80
:10A18000834754006349FA028509C20993D909013A
:10A1900083A70A009847E3EBE9FCC1B71C441319F5
:10A1A0005A00A6853E994A8597000000E780C0EED8
:10A1B00005E1050AC9B75C4413195A00A6853E9902
:10A1C0004A8597000000E78020ED19E1050A4DBFA0
:10A1D000E30C09FA61B7AA8481495DBF1783FFFFC9
:10A1E000E702E3EF1C452A8481E79307C5001CC5FD
:10A1F0001C44231204001CC09307F00F63EDB7004A
:10A2000093F5F50F228597200000E780C0E51783BE
:10A21000FFFF670003EF93940501C167C18063F9F5
:10A22000F500A685228597200000E780E0E8C5B705
:10A23000C18193F5F50F228597200000E780A0E209
:10A24000A685228597200000E780E0E3C9B797C77D
:10A25000FF1F9387E7A8884382801C4599C797C74B
:10A26000FF1F23AFA7A6014582807D55828097C737
:10A27000FF1F9387E7A69843834745004847920707
:10A280003E9582801783FFFFE70263E56171004519
:10A290001C183EC6B70780013EC81C183ECA83572B
:10A2A000440002CE02D002CC231EF100834784007A
:10A2B0002A8902D22301F1023C083ED402D697003B
:10A2C0000000E78000FB835705002316F10297503A
:10A2D0000000E78000C82307A1025C40035564002A
:10A2E000F18313F717008347F10252055181F99B5F
:10A2F000D98FA307F10297100100E780207939CDAB
:10A30000AA840355050097A00000E78020C083D7EA
:10A3100004002AD26800231CF10083D72400231DE7
:10A32000F1001C4803D647008C4397200000E780CB
:10A33000A0D08347B400CA861776010013064650A2
:10A340008117A305F4006C00481097200100E780F6
:10A3500080845D611783FFFF6700A3DA2155D5BFB5
:10A360001C45B1CF03C5A700894613576500630B91
:10A37000D7028D46630ED70285466300D7021307C6
:10A3800040063305E50203C7B700418B15CB83C7F1
:10A39000B700BD8B3355F54082801375F503130765
:10A3A000803EC5B709671375F50313070771D1BF61
:10A3B000372709001375F5031307077CD9B7014543
:10A3C00082801783FFFFE70283D103A98500630C16
:10A3D00009048347B900AE8493F7070E85C303458C
:10A3E0009900930520030D810505B305B502884446
:10A3F000610597300100E78080AD35A02E8597007C
:10A400000000E78020F62A8419CD97000000E7803D
:10A41000605C8325C900B307B54063FA87002E94BA
:10A42000B305A440E9F51783FFFF670083CD854599
:10A430007DBF1783FFFFE70283CA2A8403D5050087
:10A44000011132C636C43AC22EC002CA02CC02CEB4
:10A4500097A00000E78080AB82452ACA22852ECCD7
:10A4600097000000E780E0E003570500231EE100AD
:10A4700097500000E780E0ADA24632469247230F96
:10A48000A10036874C08B28622850146970000005D
:10A49000E780E0A605611783FFFF670083C6178387
:10A4A000FFFFE702C3C361711C183EC6B7078001F6
:10A4B0003EC81C183ECA3C0800453ED4AA8402CCC3
:10A4C00002CE02D002D202D697000000E78060DA06
:10A4D0008357050035592316F10297500000E78095
:10A4E00040A72307A10209C48357440081EB2159E7
:10A4F0004A855D611783FFFF6700A3C003556400B1
:10A500005205518197100100E78040582A8965D192
:10A510008347B40093F7070E99C71305840197305A
:10A520000100E780009D83574400231EF10083470C
:10A5300084002301F1025C4003550900D98313F71D
:10A54000070883471102231CA10093F7F707D98F4F
:10A55000A300F10283572900231DF1005C40F18321
:10A5600013F717008347F102F99BD98FA307F10274
:10A5700097A00000E78080992AD235D983479400BC
:10A580006800139757008347B400FD8BD98FA3054C
:10A59000F4001C4803D647008C4397200000E78056
:10A5A000A0A9A6871777010013078729740005461D
:10A5B0004C10268597000000E78060942A890DD909
:10A5C0008347B400A685FD8BA305F4009700000027
:10A5D000E78060DF31BF1783FFFFE70243B08324CA
:10A5E00085FE2A844111268597000000E78080D7E8
:10A5F000834734FF93F7070E8DCB2AC62685970035
:10A600000000E78060C809CD834734FFB245FD8B69
:10A61000A309F4FE91C5228597300100E780208BC5
:10A6200041011783FFFF6700C3AD7DD98327C4FFB6
:10A630002685829775F5834734FF93F7070E91C7F8
:10A64000228597300100E780C08A032584FE9700A9
:10A650000000E78000E5E9B71783FFFFE70223A5C5
:10A660009C4141112A8903C7070089472E849356CC
:10A6700067006380F6040D466388C6049307F007FD
:10A680006304F7022E8597200000E78060ABAA8460
:10A690008149C16B130C490097B7FF1F938747642B
:10A6A0009C43984763E4E90441011783FFFF670077
:10A6B000C3A303D745008547E3F8E7FE2E8597201F
:10A6C0000000E78040ADE1B703D74500E3FEE7FCBB
:10A6D0002E8597200000E780A0A6AA8422859720D7
:10A6E0000000E78000A8C204C98C5DB7DC470355B1
:10A6F000A900139A49003E9A93170501C187635D2B
:10A70000F00083570A006397A70263E77403832767
:10A71000CA00034D5A002DA0A1672167A98F130716
:10A72000F7EFE374F7FE6397090097000000E780F6
:10A73000209161FD85098DB783278A00034D4A006A
:10A74000835DA90003576900216A138BC7003AC6CD
:10A75000814A33CA4D01631E5D0197B7FF1F93877E
:10A76000A7589C43E1DBA2866286814526858297B5
:10A77000D1B7A1679387F7EF930C4BFF63F24703C1
:10A78000B2455A8597F0FFFFE780A0710DC10327FE
:10A790008B00104709CE10436382C4023107D5BF36
:10A7A000EE85668597000000E780008F71F993863B
:10A7B0001A0093FAF60F130B0B0271BF8356440075
:10A7C0005C43E3E9F6F622853AC697200000E7806D
:10A7D0002081A1679387D7042A8A035D440032470A
:10A7E00063E897008347D90093E707F8A306F900C9
:10A7F0001C4766852286E2858297C1670844FD175B
:10A80000337AFA00529508C02312A40125B797B7EE
:10A81000FF1F9387E74C9843814715C3144781472F
:10A8200063FFD500939745004C47BE9519C903C7F0
:10A83000550081476375E600DC451606B2973E85F4
:10A84000828003C745008147E37BE6FE16069C45F0
:10A85000F5B71783FFFFE702E386AA892E8A8144B2
:10A8600097BAFF1F938ACA4783A70A00984763E6EF
:10A87000E4001783FFFF67002388DC47139444003C
:10A8800001493E9413BB140083474400634BF90015
:10A89000014913BB140083475400634FF90085043A
:10A8A000E1B70844931759005287DA860146A2851A
:10A8B0003E9582990509C9BF4844931759005287AC
:10A8C000DA860546A2853E9582990509E9B7178380
:10A8D000FFFFE702C380814517F5FFFF1305054819
:10A8E00097B7FF1F2390074097000000E780A0F66E
:10A8F0001783FFFF6700E38097B7FF1F9387473EEB
:10A900009C4395C31773FFFFE702637D814517F5ED
:10A91000FFFF1305A54497000000E780C0F31773FD
:10A92000FFFF6700037E82801773FFFFE7028379D2
:10A9300037E404008327841241112315E100AE8916
:10A940003289368A3A8681460147ED45AA84829744
:10A950002AC621C90356A100D28597400100E7808D
:10A9600060288327C413CE8526858297058905C96B
:10A970008327440D2314210101462C00268582974C
:10A980002A8401C9B7E7040083A7C712ED45280050
:10A990008297228541011773FFFF6700E3754944E1
:10A9A000D5B76554FDB75C41FD175CC18280177354
:10A9B000FFFFE702C372B7E70400FC5F8297954789
:10A9C0003305F50281450D811773FFFF670063733F
:10A9D0001773FFFFE702A370B7E70400FC5F8297DD
:10A9E00095473305F5020D811773FFFF670063710B
:10A9F0001773FFFFE702A36EB7E7040083A7870B77
:10AA00000355050082971773FFFF6700836F177365
:10AA1000FFFFE702C36C035505003287AE86179629
:10AA2000FF1F035646AB97B5FF1F9385252C970054
:10AA30000000E780A0EF1773FFFF6700836C1773B8
:10AA4000FFFFE702C369B7E7040083A7C717829730
:10AA50001773FFFF6700E36A1773FFFFE7022368BE
:10AA6000B7E7040083A7871397B5FF1F93850528D1
:10AA7000829701451773FFFF6700A3681773FFFFF5
:10AA8000E702E365B7E7040083A7C71F8145179571
:10AA9000FF1F035545A082971773FFFF670063668A
:10AAA0001773FFFFE702A363B7E7040083A78713C9
:10AAB00097B5FF1F93858524829701451773FFFF84
:10AAC000670023641773FFFFE7026361B7E70400C1
:10AAD00083A7C71F81451795FF1F0355C5A18297FF
:10AAE0001773FFFF6700E3611773FFFFE702235F40
:10AAF0002E8597800000E78080B397800000E78074
:10AB000080F01773FFFF6700C35F1773FFFFE70253
:10AB1000035D97800000E78080FA1773FFFF6700EE
:10AB2000435E5C49E1175CC95CC583572501A107F9
:10AB30002319F50083570501A1072318F50082802A
:10AB4000F1473305F50297B7FF1F9387271D9C43F5
:10AB50003E9582808D476315F60803D746008547EA
:10AB600063F0E7081773FFFFE70263573685368403
:10AB70002E8997100000E780A05C29C98357440004
:10AB800093140501C18063E39704228597100000A8
:10AB9000E780005BFD14231294009307A00263007A
:10ABA000F5029307B0026307F50293079002631F53
:10ABB000F500228597000100E780608901A8014621
:10ABC000CA85228597A00000E78000B41773FFFFB5
:10ABD00067002353228597100000E7806007FDB7C8
:10ABE000828097B6FF1F9386A6139C42014599CF9A
:10ABF0009843D44217B6FF1F2324E6126396D7006A
:10AC000097B6FF1F23A0E6121385C7FE8280177335
:10AC1000FFFFE702C34C97000000E780A04B7144A0
:10AC200033058502914597900000E780C0EC11E55F
:10AC300065551773FFFF6700C34C97B7FF1F23AD20
:10AC4000A70C97000000E780E04833058502914596
:10AC500097900000E78020EA61DD97B7FF1F23AFE0
:10AC6000A70A97000000E780E04697B7FF1F239FE1
:10AC7000A70897000000E780E04597B7FF1F2398DB
:10AC8000A708977701009387E7C017B7FF1F232313
:10AC9000F70897070000938707E917B7FF1F2329D5
:10ACA000F706014579B71773FFFFE7024343AA850B
:10ACB00017B5FF1F1305850597100000E780605F3B
:10ACC0001773FFFF6700E3431773FFFFE70223419A
:10ACD00097000000E78060FD97100000E780E05ECD
:10ACE00097B7FF1F9387C7039C4391CF1387C7FE76
:10ACF00019CB83D5C7FF17B5FF1F1305E5029720B2
:10AD00000100E780C01C1773FFFF6700833F1773C4
:10AD1000FFFFE702C33C97000000E780C0EC09CDCD
:10AD2000834785002A8493F7070499EB0355E500D0
:10AD300097000000E78080F91773FFFF6700633C0E
:10AD40008347C5009304450117B9FF1F130949FD47
:10AD500085E3832709005CC997B7FF1F23A297FCEF
:10AD600083274900F1FB97B7FF1F23AD97FAE9B797
:10AD7000FD172306F500610597800000E78060DA83
:10AD80008307840063CB07048347840093E707F8B5
:10AD90002304F400B7E704009C5F82974205A947AB
:10ADA00041813375F5028347840093F707FCC98F0F
:10ADB0002304F4008347D4003E951C402318A400CC
:10ADC00089CF984319CB8347C400504081458507FC
:10ADD0003305F502420541810297832709005CC8CB
:10ADE00097B7FF1F23AE97F28327490089E797B7EC
:10ADF000FF1F23A997F28347C4009DDF83550401F9
:10AE000017B5FF1F130545F297200100E780200CBE
:10AE100025B71773FFFFE702832C97B7FF1F9387B0
:10AE2000E7159C4701448583858B85E3AE84B28515
:10AE30003A8697100000E780204F2A8419C59710A2
:10AE40000000E7806045829408CC22851773FFFFDD
:10AE50006700232B1773FFFFE702C32641112E89DA
:10AE600032C6AA8997000000E780C0313247130636
:10AE70000502CA86970500009385C5CC17B5FF1F4C
:10AE80001305C5E897000000E780E0F82A8425C98B
:10AE90009304C50097000000E780E0411946AA85A9
:10AEA000268597100000E780201985452685971094
:10AEB0000000E7800015177501001305659B4E958E
:10AEC00083450500268597100000E780C0195C487F
:10AED00031468145A1075CC85CC483572401E11752
:10AEE0002319F40083570401E1172318F4001C4CC4
:10AEF0003E859770FFFFE7808021A304250122850E
:10AF000041011773FFFF6700231F1773FFFFE7025D
:10AF1000031D4111AA842EC632C497100000E78099
:10AF2000003A004DB2452246834784000CC050C011
:10AF300093F7F70393E707042304F40023180400AE
:10AF4000268597100000E780203583479400A946A6
:10AF50002317A40013D7370005073307D7029D8BAB
:10AF600085072306F400A306E40083C70401D8483C
:10AF70008507230FF7FE17B7FF1F130767DA58433C
:10AF8000232A04009307440129E317B7FF1F232B4B
:10AF9000F7D817B7FF1F2325F7D817B4FF1F1304DF
:10AFA000A4D8228597200100E780A0E41C44858B6B
:10AFB0005D8D19E58145228597200100E78020F10C
:10AFC00041011773FFFF6700C3131CC317B7FF1FAF
:10AFD000232AF7D4D9B71773FFFFE7024310970569
:10AFE0000000938565B7014597000000E78000B039
:10AFF00001451773FFFF6700C3101773FFFFE702D8
:10B00000030E97000000E78080B01773FFFF670012
:10B01000430F8347C500A5E31773FFFFE702230C27
:10B020002A840355E50097000000E78000C821C18D
:10B030008347840093F7F7FB2304F4001C4091C777
:10B04000DC4381C74C400145829797000000E780B0
:10B0500080B917B5FF1F130525CD97200100E780A4
:10B0600040E90355E40097000000E78020C617730D
:10B07000FFFF6700030982801773FFFFE7022306C3
:10B0800097B7FF1F9387C7C997050000938565C8C9
:10B0900017B5FF1F130545C923A0070023A207000A
:10B0A00097200100E78080D21773FFFF67006305D8
:10B0B0001C4D91CFDC4381CF1773FFFFE7022302C2
:10B0C0008345070082971773FFFF67008303828021
:10B0D00097B7FF1F938787C79C4303C507008280EC
:10B0E00097B7FF1F938787C69C4303C517008280CD
:10B0F00097B7FF1F938787C59C4303C527008280AE
:10B1000097B7FF1F938787C49C4303C5470082807E
:10B1100097B7FF1F938787C39C4303C5370082807F
:10B1200097B7FF1F938787C29C4303C55700828050
:10B1300097B7FF1F938787C19C4303C56700828031
:10B1400097B7FF1F938787C09C4303C57700828012
:10B1500097B7FF1F938787BF9C4303C587008280F3
:10B1600097B7FF1F938787BE9C4303C597008280D4
:10B1700097B7FF1F938787BD9C4303C5A7008280B5
:10B1800097B7FF1F938787BC9C4303C5B70011E1A6
:10B190001D45828097B7FF1F938747BB9C4303C51C
:10B1A000C700828097B7FF1F938747BA9C4303C5A8
:10B1B000D700828097B7FF1F938747B99C4303C589
:10B1C000E700828097B7FF1F938747B89C4303D55A
:10B1D0000701828097B7FF1F938747B79C4303C53A
:10B1E0002701828097B7FF1F938747B69C4303D5FB
:10B1F0004701828097B7FF1F938747B59C4303D5CC
:10B200006701828097B7FF1F938747B49C4303D59C
:10B210008701828097B7FF1F938747B39C4303C57D
:10B22000A701828097B7FF1F938747B29C4303C54E
:10B23000B701828097B7FF1F938747B19C4303C52F
:10B24000C701828097B7FF1F938747B09C4303C510
:10B25000D701828097B7FF1F938747AF9C438857DA
:10B26000828097B7FF1F938767AE9C4303D5C702C1
:10B27000828097B7FF1F938767AD9C4303D5E70292
:10B2800019E11305800C828097B7FF1F938707ACE5
:10B290009C4303C50703828097B7FF1F938707ABC3
:10B2A0009C43C85B828097B7FF1F9387A7A98843F9
:10B2B000828097B7FF1F938727A98843828019E16F
:10B2C0007D558280F5DE984265DFFDD917B7FF1FF7
:10B2D0001307C7CA1847AA877155058B631D072432
:10B2E00003C507001547E37DA7FC03C73700130517
:10B2F000F0057D171377F70FE364E5FC03C35700F0
:10B30000E30003FC83C86700E38C08FA03C77700F7
:10B31000494579171377F70FE364E5FA03C7A700E8
:10B3200011481305F7FF1375F50FE36BA8F803CE6B
:10B3300097000D481305FEFF1375F50FE362A8F89B
:10B3400003C8B7006309080065181378F80F1305E0
:10B35000600DE36705F703C5C700794879151375D4
:10B36000F50FE36FA8F403C8D7000D457D181378D7
:10B37000F80FE36705F503D80701930E401751183E
:10B38000420813580801E3ED0EF303C8E7007D18E7
:10B390001378F80FE36605F303C827017D181378C7
:10B3A000F80FE36F05F103C88700C54E75181378D1
:10B3B000F80FE3E70EF103D86701856E938EBEE0C8
:10B3C0006D18420813580801E3EC0EEF03D847014B
:10B3D0006D18420813580801E3E40EEF03D8870103
:10B3E0007918420813580801E36C05ED03C8A7015A
:10B3F0007D181378F80FE36505ED03C5B7011D4807
:10B400007D151375F50FE36DA8EA03C5D7017148E3
:10B4100079151375F50FE365A8EA03D5E70113085D
:10B42000E00F7D1542054181E36CA8E803C50702E2
:10B43000494879151375F50FE364A8E8C85301C9A5
:10B4400037C834005915130858BFE36BA8E603A8A2
:10B45000870237C53400130555BF5918E36205E765
:10B4600017B5FF1F2322C58E03C6050117B5FF1FA1
:10B47000232EF58C0545E375C5E403D82501D04995
:10B4800033760603E31E06E203C61501E30A06E26D
:10B4900017B6FF1F2328B68A83C527000146638796
:10B4A000A50003C61700F1453306B60283C707039C
:10B4B0009305C00272971A071307C70516031A9758
:10B4C00096084697B387B70241553E973297420791
:10B4D00041836362E8061773FFFFE70243C03685C6
:10B4E00097800000E780406C97000100E780C04B28
:10B4F0002A8497A00000E780205E2A9497F000003D
:10B50000E780002A2A9497900000E78040852A94DB
:10B5100097F0FFFFE780E06F2A9497400000E780F4
:10B5200000972A9497700000E78040A02295177337
:10B53000FFFF670003BD82801773FFFFE70223BA96
:10B540004111A307A10097A00000E78040C993051F
:10B55000F100170500001305E5B597F0FFFFE78040
:10B56000802F014541011773FFFF670083B91773EF
:10B57000FFFFE70243B417B4FF1F130424A00328FE
:10B58000840079599368180097B4FF1F23AC149F67
:10B590001378180063100802BA84BE89368B328A89
:10B5A0002E89AA8A97F0FFFFE780E0A77D152695F0
:10B5B00019E531594A851773FFFF670043B397F0C8
:10B5C000FFFFE78040A67D152695A167E353F5FEB2
:10B5D00097B7FF1F938787D198433E8C814B01CB50
:10B5E000014597F00000E780C047933B15004A856E
:10B5F000DA865686D28597900000E78060512A89C6
:10B6000011CD1C44F99B17B7FF1F232DF7968327F5
:10B610000C00CDD3E3800BFA829769BF268597B7DC
:10B62000FF1F23AF079497F0FFFFE780809C414600
:10B63000CE8517B5FF1F1305E59D97300100E78004
:10B64000605A97D00000E780E09C0325040B97D058
:10B650000000E780A0A0054597D00000E780A0A7E4
:10B66000054597000000E78060EDA9B797B7FF1F79
:10B670009387C7909C47858BEDC71773FFFFE70241
:10B6800003A617B5FF1F1305259797B7FF1F23A71D
:10B69000078E97B7FF1F23A5078E97B7FF1F23A31A
:10B6A000078E97200100E780C08497500000E78054
:10B6B00080F997100100E780405097100100E78063
:10B6C000405697B7FF1F9387E7899C4391C705456D
:10B6D00097800000E780E02397A7FF1F93874772BA
:10B6E0009C4399C741657D1597700000E780E0A5F0
:10B6F00097F00000E780804197D00000E78020931A
:10B7000097B7FF1F9387879C9C4313971701635636
:10B71000070097F00000E780A0B097B7FF1F23ABAA
:10B72000078E97B7FF1F23A9078E97B7FF1F23A781
:10B73000078E97B7FF1F23A5078E97000000E780AD
:10B74000008C97000000E780A07597F0FFFFE7806E
:10B75000401897F00000E780E0D91773FFFF6700FB
:10B76000439A828097B7FF1F9387478188438280DF
:10B7700097B7FF1F93878780C8438280B7E7B000E1
:10B780009387075063E1A70297A7FF1F9387077F5F
:10B79000D843FD576367E50097A7FF1F23A2A77E45
:10B7A00081473E858280B957EDBF1773FFFFE702DF
:10B7B000039397800000E780607597800000E78022
:10B7C000C0771773FFFF6700C3931773FFFFE7028C
:10B7D000638F2A849304140201112E85B289A685F1
:10B7E000214636C63A8997300100E780403D0DE991
:10B7F000B24638082686CE8513059404975000007B
:10B80000E780604121462C084A8597300100E78097
:10B81000003B1335150005611773FFFF6700C38DEB
:10B820000145D5BF1773FFFFE702638B93054506FC
:10B8300017A5FF1F1305C55197100100E780206968
:10B840001773FFFF6700E38B1773FFFFE70223897E
:10B8500041112EC697F0FFFFE780C017B24588C19F
:10B8600041011773FFFF6700C3891773FFFFE702EA
:10B870006385AA842E8497800000E780006CAA89E3
:10B880008545228597000000E780E07D83C7E401BD
:10B890001389940899E313890403CE8522859700C0
:10B8A0000000E780407C214693051902228597001D
:10B8B0000000E780607897A7FF1F9387276C8C4371
:10B8C000228597100000E780C0822146938584027C
:10B8D000228597000000E78020761773FFFF67003E
:10B8E000A3811763FFFFE702037D397197F0000022
:10B8F000E780E0B49305400661E997800000E780A7
:10B9000000606302051497A7FF1F83C7274613B77C
:10B91000170097A6FF1F238BE644014499CFC1640B
:10B9200017A9FF1F130989659309400EFD1497009D
:10B930000000E78020836342A40A97F0FFFFE780BE
:10B9400060094169B7290900096AFD7A2A8B814497
:10B950007D199389F97B130A0A71938A8AC7970024
:10B960000000E780208063D7A4041304400EB3874F
:10B97000840217A7FF1F130767600324070B3E9479
:10B980008357C4016382270B18403307EB4063EAF7
:10B99000E900834744008507B3874703D69763656B
:10B9A000F70801468145094597F0FFFFE780C04A47
:10B9B000AA8B29E597400000E780808385476317BD
:10B9C000F50689659385057117A5FF1F1305453891
:10B9D00097100100E780A04F95A0B3073403032719
:10B9E000090BBA9703D7C7016308970003C757002D
:10B9F000A38207002382E700050415BF9305C50055
:10BA0000228597000000E78080E65E8522869765A4
:10BA10000100938525E797F0FFFFE780404F5E85A3
:10BA200097100000E780608A850415BF97A7FF1F65
:10BA30009387C7549C478D83858BC1F7216117631A
:10BA4000FFFF6700C36A01468545094502D002D25F
:10BA500002D402D697F0FFFFE7800040AA8479DD88
:10BA600097F00000E780E09C1389C4002A84814598
:10BA70004A8597000000E780005F0C4041464A85F8
:10BA800097000000E780405B832944006385090C30
:10BA90004E8502D802DA02DC02DE97300100E78030
:10BAA000E0382ACE141005462C0808184ECC9750C2
:10BAB0000000E780E00A1375F50F51ED835584000F
:10BAC00093E525004A8597000000E780E05E114677
:10BAD0000C104A8597000000E780005601469765E4
:10BAE00001009385A5DA268597F0FFFFE7802042C5
:10BAF000268597000000E780407D5C40A1D3014689
:10BB000085450D4597F0FFFFE7800035AA841DD5D8
:10BB100048401389C40097300100E78020312AC6CD
:10BB20004A8597000000E780404C3246636FC500AD
:10BB30004C404A8597000000E7800050014681454F
:10BB4000268597F0FFFFE780803C26859700000060
:10BB5000E780A077E5B583558400ADB71763FFFF95
:10BB6000E702E35797A7FF1F938747419C471DC1F3
:10BB700093E7870017A5FF1F1305851D17A7FF1F54
:10BB80002322F74097100100E78040321763FFFF40
:10BB900067002357DD9B17A7FF1F2325F73E97302C
:10BBA0000000E780E0647DF117A5FF1F1305451A2B
:10BBB00097100100E780E033D1BF1763FFFFE70272
:10BBC000834F4169AA892E8AB28A368BBA8B814407
:10BBD00017ACFF1F130C8C3A930C400E7D1997F095
:10BBE000FFFFE780205863C4A40001443DA03384D4
:10BBF000940383270C0B3E948357C4016386270567
:10BC00005A87D6865286CE85130504039700000016
:10BC1000E780E0BB01C923800B0022851763FFFF8B
:10BC20006700E34C8347F40185C35A87D686528662
:10BC3000CE851305940897000000E78040B909C538
:10BC400085472380FB00D1BF850451BF8357450042
:10BC50006380071E1763FFFFE702C34601112A84B2
:10BC600097000000E780C04D09C985476309F506C4
:10BC700005611763FFFF6700234897E00000E78036
:10BC8000007C7DF5835744004947ED9BE392E7FE36
:10BC9000C145228597000000E7804033AA842285B1
:10BCA00097000000E780204F0357440002CE9147E1
:10BCB0002A89631AF700228597000000E780A051C7
:10BCC0003C082ACC3ECE97E00000E78080765C55A9
:10BCD000C5D374084A86A6850545829751BF035788
:10BCE0004400D147E3F6E7F8032A0400C16901499B
:10BCF00097AAFF1F938A8A28130B400EFD1997F00D
:10BD0000FFFFE7802046634FA90E2285032A040027
:10BD100097000000E780C042A1452A89228597004C
:10BD20000000E780A02AAA84228597000000E7800F
:10BD3000804A14402A86AA8978082685CA859700F1
:10BD40000000E780C0E7AA8405D503C7F40189474E
:10BD50006315F7008347C10181DF5546D2851385FE
:10BD6000640097300100E780E0E70145978000001C
:10BD7000E780C01901C583D7C401A5E797A7FF1FB6
:10BD80009387C71F9C4793551900858913D73700A0
:10BD9000058B01CF8983858B6399B70001452EC63A
:10BDA00097000000E780C0DBB2454E859780000019
:10BDB000E780601F0346C1012A8493751900268518
:10BDC00097900000E780E03935C126859780000014
:10BDD000E780E018268511C0014597800000E780C4
:10BDE000004C97300000E780A0408547E312F5E85B
:10BDF00083C754001307F00FE38CE7E68507A3829F
:10BE0000F400BDB5B304690383A70A0BBE9483D7BE
:10BE1000C401638B37015546D28513856400973082
:10BE20000100E780C0D955DD0509D1BD5DD86DB7EA
:10BE300082801763FFFFE702E32897800000E78016
:10BE4000000C05C1C164014417A9FF1F13090913A0
:10BE50009309400EFD1497F0FFFFE780A030634E7A
:10BE6000A40017A5FF1F1305A5EE97100100E7809A
:10BE7000E0031763FFFF670023283305340383279C
:10BE8000090B3E958357C50163889700231205006F
:10BE900097800000E780A00C050475BF97A7FF1FDF
:10BEA0009387C70D9C478D83858B8DE31763FFFFB9
:10BEB000E702E32217A5FF1F130585E9971001008C
:10BEC000E78020031763FFFF6700A32382801763C7
:10BED000FFFFE702C320970500009385C5A017A5C3
:10BEE000FF1F1305E5E697100100E78020EE1763BA
:10BEF000FFFF670003211763FFFFE702431E88412E
:10BF0000B7E70400BC5B050542054181829709C57E
:10BF100085472300F50005051763FFFF6700631ED3
:10BF200083C7F5FF2E858507A38FF5FE828083C723
:10BF3000F5FFFD1793F7F70FA38FF5FE99EF176342
:10BF4000FFFFE702C319B7E70400BC571385F5FFED
:10BF500082971763FFFF6700C31A82801C41035753
:10BF600045008D8FBA951CC12312B5003E85828095
:10BF700093D78500A2051441DD8D835745001387B3
:10BF8000E6FF18C189072312F50013D68500411179
:10BF9000238FB6FEA38FC6FE41018280184193070E
:10BFA000F7FF1CC18357450085072312F500A30F37
:10BFB000B7FE8280835745008D8F2312F5001C4108
:10BFC000BE950CC12E858280AA8703D74700084101
:10BFD0000D8FAA952392E7008CC3828018410845F3
:10BFE0003305A740828083574500035765001D8FA6
:10BFF0001C4108453385A7403305A740828017635D
:10C00000FFFFE702C30D41112EC62A8497000000EE
:10C01000E780A0FDB2456373B50001A083574400DB
:10C020000840BE952312B4003E9541011763FFFFFF
:10C030006700230D1763FFFFE702630A41112E8497
:10C04000B28532C697000000E780A0FB3246A28589
:10C0500097300100E78000B941011763FFFF6700D7
:10C06000430A1763FFFFE70283072E848545970085
:10C070000000E78000F9230085001763FFFF6700D9
:10C0800043081763FFFFE702830541112317B1003F
:10C09000894597000000E780C0F68347E100230050
:10C0A000F5008347F100A300F50041011763FFFF8E
:10C0B000670023051763FFFFE702630293D785003C
:10C0C000A2054111DD8D2317B100894597000000BD
:10C0D000E78020F38347E1002300F5008347F10068
:10C0E000A300F50041011763FFFF67008301176399
:10C0F000FFFFE702C3FE1397850193D78501C16651
:10C10000938606F0D98F13D78500758FD98FA20536
:10C110003707FF00F98D4111DD8D2EC6914597003F
:10C120000000E78000EE6C00114697300100E780C8
:10C1300060AB41011763FFFF6700A3FC1763FFFFBC
:10C14000E702E3F91C41854503C40700970000009E
:10C15000E78080E622851763FFFF670083FA176395
:10C16000FFFFE702C3F71C414111894503C70700E0
:10C1700083C717002307E100A307F1009700000021
:10C18000E78080E30355E10041011763FFFF67008B
:10C1900043F71763FFFFE70283F41C414111894510
:10C1A00003C7070083C717002307E100A307F100B7
:10C1B00097000000E78040E08357E100410113D57C
:10C1C0008700A2075D8D420541811763FFFF67006D
:10C1D00043F31763FFFFE70283F00C4141112A8408
:10C1E0001146680097300100E780C09F9145228585
:10C1F00097000000E78040DCB247C166938606F0F6
:10C200001397870113D58701598D13D78700758F31
:10C21000598DA2073707FF00F98F5D8D4101176324
:10C22000FFFF670003EE1C45BE950CC18280AE8700
:10C23000944391E6584101EF0CC15CC1828003C771
:10C24000570013671700A382E700B687D5B70CC362
:10C25000EDB7AA87084119CD1841D44398C3631399
:10C26000D500D8C32A87034657009376160081E687
:10C27000232007008280944381CA8C4203A8470090
:10C280008CC363930601CCC3799A14C3A302C7007D
:10C290003687D1BF1C45DC471D8DB777DBB693874A
:10C2A00077DB09853305F502420541818280F1473C
:10C2B000B385F50248452E95828083474500850762
:10C2C0002302F50082801763FFFFE70243E12A841F
:10C2D00009E41763FFFF6700C3E283474400F5DB0F
:10C2E000FD1793F7F70F2302F400E5F71C4403D77B
:10C2F000270005072391E700DC4399C32285829735
:10C300004C4889CD83475400898B99E71C4422858A
:10C310009C479C439C478297232A0400004023208B
:10C3200004007DB71763FFFFE70263DB8357250037
:10C3300041112EC681EB0144228541011763FFFFA5
:10C34000670023DC035705008147F146E305F7FE4C
:10C35000B385D702404585072E948345440008C421
:10C36000F5F5B247AA8481E7232A040009A81C45F1
:10C370006C0022859C439C43829748C84DDD8547CD
:10C380002312F400B24723200400231804002319C9
:10C39000F4005C485CC483D72400FD172391F400AB
:10C3A00061BF1763FFFFE70283D397A7FF1F938740
:10C3B000279C884323260500232405004105971068
:10C3C0000100E78000B31763FFFF670083D31763A3
:10C3D000FFFFE702C3D017A4FF1F130464991C409A
:10C3E000411199CF9C472300B5002AC65CC1970034
:10C3F0000000E78040FB1C40DC4399C33245829734
:10C4000041011763FFFF6700C3CF0347450029E3DE
:10C41000584DAA877D551DCF1763FFFFE70223CC38
:10C420001CC3DC4797A6FF1F23A4E694F15613050F
:10C4300007012390D7009705000093850502971008
:10C440000100E780A09801451763FFFF670063CBF9
:10C450007D55828082801763FFFFE70243C8011188
:10C460006146814528009760FFFFE78040CA97A793
:10C47000FF1F9387E78F9C4328009305F00FDC474D
:10C480003EC697000000E780C0F405611763FFFF18
:10C49000670023C797A7FF1F9387878D9C43D847C3
:10C4A000A1679387C702631EF70A397106DE22DC93
:10C4B00026DA80004AD84ED652D456D23285B2847B
:10C4C00097000000E780C0C7AA8926859700000072
:10C4D000E78020C92318A4FC268597000000E78088
:10C4E00040C82319A4FC268597000000E78060C798
:10C4F00083D744000A8A231AA4FC858393F7F70F95
:10C50000230EF4FC8607BD0793F7073F3301F14084
:10C510008A8A01498347C4FD6367F902CE85130502
:10C5200084FC232C54FD97000000E78080EA5281B0
:10C53000130104FCF2506254D2544259B259225AA7
:10C54000925A21618280268597000000E78060C1B1
:10C5500093171900D69705092390A7001379F90FAF
:10C5600055BF828097A7FF1F938787809C43D8473A
:10C57000A1679387A702631AF70A397106DE22DCE6
:10C5800026DA80004AD84ED652D456D23285B284AA
:10C5900097000000E780C0BAAA89268597000000AE
:10C5A000E78020BCFD572318A4FC26852319F4FC42
:10C5B00097000000E780E0BA83D744000A8A231A74
:10C5C000A4FC858393F7F70F230EF4FC8607BD07C1
:10C5D00093F7073F3301F1408A8A01498347C4FD3D
:10C5E0006367F902CE85130584FC232C54FD970064
:10C5F0000000E78000DE5281130104FCF250625417
:10C60000D2544259B259225A925A216182802685C7
:10C6100097000000E780E0B493171900D69705094A
:10C620002390A7001379F90F55BF82809797FF1FBA
:10C63000938707749C43D847A16789076310F70A5B
:10C64000397106DE22DC26DA80004AD84ED652D472
:10C6500056D23285328997000000E78060AEAA8901
:10C660004A8597000000E780C0AF835749000A8AD7
:10C670002318A4FC858393F7F70F230CF4FC86079B
:10C68000BD0793F7073F3301F1408A8A814483470E
:10C6900084FD63E7F402CE85130584FC232A54FD50
:10C6A00097000000E780E0D25281130104FCF250B1
:10C6B0006254D2544259B259225A925A216182800C
:10C6C0004A8597000000E780C0A993971400D69789
:10C6D00085042390A70093F4F40F55BF82809797A9
:10C6E000FF1F9387E7689C43D847A1679387E704B8
:10C6F000631EF70A397106DE22DC26DA80004AD88A
:10C700004ED652D456D23285B28497000000E780CC
:10C7100020A3AA89268597000000E78080A423181B
:10C72000A4FC268597000000E780A0A3231AA4FCA0
:10C73000268597000000E780C0A283D744000A8ABC
:10C740002319A4FC858393F7F70F230EF4FC8607C7
:10C75000BD0793F7073F3301F1408A8A01498347B8
:10C76000C4FD6367F902CE85130584FC232C54FDB8
:10C7700097000000E780E0C55281130104FCF250ED
:10C780006254D2544259B259225A925A216182803B
:10C79000268597000000E780C09C93171900D69764
:10C7A00005092390A7001379F90F55BF8280979749
:10C7B000FF1F9387E75B9C43D847A1679387C70414
:10C7C000631AF70A397106DE22DC26DA80004AD8BD
:10C7D0004ED652D456D23285B28497000000E780FC
:10C7E0002096AA89268597000000E7808097FD574C
:10C7F0002318A4FC2685231AF4FC97000000E78088
:10C80000409683D744000A8A2319A4FC858393F7B2
:10C81000F70F230EF4FC8607BD0793F7073F33019C
:10C82000F1408A8A01498347C4FD6367F902CE85D6
:10C83000130584FC232C54FD97000000E78060B9A9
:10C840005281130104FCF2506254D2544259B2593D
:10C85000225A925A21618280268597000000E78043
:10C86000409093171900D69705092390A7001379D4
:10C87000F90F55BF82809797FF1F9387674F9C439F
:10C88000D847A167DD076317F7041763FFFFE702C7
:10C89000038579713285328497000000E780408AF1
:10C8A0002AC6228597000000E780A08B2311A102F1
:10C8B000228597000000E780A088B2452300A102EE
:10C8C000280897000000E780C0B045611763FFFFAC
:10C8D0006700238382809797FF1F938767499C4354
:10C8E000D847A167938787046317F7041753FFFF9F
:10C8F000E702E37E79713285328497000000E78099
:10C9000020842AC6228597000000E78080852311B5
:10C91000A102228597000000E7808082B2452300B3
:10C92000A102280897000000E780A0AA45611753DC
:10C93000FFFF6700037D82809797FF1F9387474320
:10C940009C43D847A1679387A7046312F702175344
:10C95000FFFFE702C378011128008145970000001E
:10C96000E78020A705611753FFFF67008379828066
:10C970009797FF1F9387C73F9C43D847A16793872B
:10C9800057026319F7021753FFFFE70243750111BE
:10C99000328597F0FFFFE780A07A2308A100814548
:10C9A000280097000000E780C0A205611753FFFF31
:10C9B0006700237582809797FF1F9387673B9C438F
:10C9C000D847A1679387E702631BF7041753FFFF5C
:10C9D000E702E37001113285328497F0FFFFE780B0
:10C9E0004078AA84228597F0FFFFE780807785470B
:10C9F00009E9228597F0FFFFE78080744205B3378D
:10CA0000A00028008145231891003ECA970000002D
:10CA1000E780209C05611753FFFF6700836E8280CB
:10CA20009797FF1F9387C7349C43D8479947631351
:10CA3000F7081753FFFFE702836A79713285328462
:10CA400097F0FFFFE780C06F2AC6228597F0FFFFAF
:10CA5000E78020712310A102228597F0FFFFE78075
:10CA6000206E2301A102228597F0FFFFE780406D31
:10CA7000A301A102228597F0FFFFE780606C2302EB
:10CA8000A102228597F0FFFFE780806B2313A102AC
:10CA9000228597F0FFFFE780A06AB2452314A10228
:10CAA000280897000000E780C09245611753FFFFF8
:10CAB0006700236582809797FF1F9387672B9C43AE
:10CAC000D847A1679387C7036313F7081753FFFF7E
:10CAD000E702E36079713285328497F0FFFFE780E7
:10CAE00020662AC6228597F0FFFFE7808067231023
:10CAF000A102228597F0FFFFE780A0662311A10223
:10CB0000228597F0FFFFE780A0632302A102228520
:10CB100097F0FFFFE780C062A302A102228597F091
:10CB2000FFFFE780E0612303A102228597F0FFFF6A
:10CB3000E7800061B245A303A10228089700000026
:10CB4000E780208945611753FFFF6700835B828080
:10CB50001753FFFFE702A35801112A8497F0FFFF44
:10CB6000E780005EAA84228597F0FFFFE780605F80
:10CB7000228597F0FFFFE780C05E035744008D4792
:10CB800063F7E700228597F0FFFFE780805D22854D
:10CB900097F0FFFFE780E05C2800A6859700000083
:10CBA000E780208305611753FFFF67008355979740
:10CBB000FF1F9387E71B9C43D847A167FD07631FAF
:10CBC000F7001753FFFFE7028351328597000000FB
:10CBD000E78040F81753FFFF6700A35282809797C2
:10CBE000FF1F9387E7189C43D847A167E5076315A4
:10CBF000F7081753FFFFE702834E797132853284BD
:10CC000097F0FFFFE780C0532AC6228597F0FFFF09
:10CC1000E7802055228597F0FFFFE780805423109E
:10CC2000A102228597F0FFFFE780A05352055181B2
:10CC30002311A10222852302010297F0FFFFE78062
:10CC40002050A302A102228597F0FFFFE780404F0A
:10CC50002303A102228597F0FFFFE780604EB245D3
:10CC6000A303A102280897F0FFFFE78080764561C3
:10CC70001753FFFF6700E34882809797FF1F938752
:10CC8000270F9C43D847A1679387E703631FF700EB
:10CC90001753FFFFE702A344328597000000E780A7
:10CCA00060EB1753FFFF6700C34582809797FF1F14
:10CCB0009387070C9C43D847A16793874704631E5B
:10CCC000F7021753FFFFE7028341797132853284FF
:10CCD00097F0FFFFE780C0462AC6228597F0FFFF46
:10CCE000E7802048B245280897F0FFFFE780606E94
:10CCF00045611753FFFF6700C34082809797FF1F6E
:10CD0000938707079C43D847A167938787026310DF
:10CD1000F7041753FFFFE702833C797132853284B1
:10CD200097F0FFFFE780C0412AC6228597F0FFFFFA
:10CD3000E7800041B2452300A102280897F0FFFFD9
:10CD4000E780206945611753FFFF6700833B8280BE
:10CD50001753FFFFE702A338011197F0FFFFE780A9
:10CD6000203EAA85280097F0FFFFE78080660561D6
:10CD70001753FFFF6700E3389797FF1F938747FF1D
:10CD80009C43D847A167D107631FF7001753FFFFE4
:10CD9000E702E334328597000000E780A0FB1753D9
:10CDA000FFFF6700033682809797FF1F938747FC3A
:10CDB0009C43D847A167C507631FF7001753FFFFC0
:10CDC000E702E331328597000000E780A0F81753AF
:10CDD000FFFF6700033382809797FF1F938747F910
:10CDE0009C43D847A167B907631FF7001753FFFF9C
:10CDF000E702E32E328597000000E780A0F5175385
:10CE0000FFFF6700033082809797FF1F938747F6E5
:10CE10009C43D847A167AD07631FF7001753FFFF77
:10CE2000E702E32B328597000000E780A0F217535A
:10CE3000FFFF6700032D82809797FF1F938747F3BB
:10CE40009C43D84789476318F7021753FFFFE7024F
:10CE500003290111328532C897F0FFFFE780402E89
:10CE6000AA85280097F0FFFFE780A05605611753B9
:10CE7000FFFF6700032982809797FF1F938747EF83
:10CE80009C43D847A1678D076311F7041753FFFF31
:10CE9000E702E32401113285328497F0FFFFE78037
:10CEA000202A13066100AA844C00228597300000D6
:10CEB000E780C0232800A68597F0FFFFE780605138
:10CEC00005611753FFFF6700C32382809797FF1FF9
:10CED000938747EA9C4381CFDC4391CB1753FFFFF5
:10CEE000E702E31F82971753FFFF670083218280C9
:10CEF0001753FFFFE702A31E79713C08AE843ED2B0
:10CF0000A165B7070A002A843ED448103C08DD0515
:10CF10003ED636C432C63AC297D0FFFFE780402CD7
:10CF200012474810BA8597F0FFFFE780C0133246DA
:10CF30004810B28597F0FFFFE780E014A246481042
:10CF4000B68597F0FFFFE780001250100147814639
:10CF5000A685228597D0FFFFE780E04D45611753F6
:10CF6000FFFF6700031A1753FFFFE7024317011182
:10CF70007C000329C501AE843ECAA165B70707003E
:10CF80002A843ECC48087C00C5053ECE97D0FFFFE2
:10CF9000E78000258345D900480897F0FFFFE78028
:10CFA000800C500801478146A685228597D0FFFF57
:10CFB000E780604805611753FFFF6700831417532C
:10CFC000FFFFE702C31183C7950093F7F707A38418
:10CFD000F50097000000E78040F91753FFFF670056
:10CFE00043121753FFFFE702830F79713C08AE84A9
:10CFF0003ED2A165B70709002A843ED448103C08F8
:10D00000938545043ED632C636C497D0FFFFE780ED
:10D01000201DA2464810B68597F0FFFFE780A004C8
:10D0200032464810B28597F0FFFFE780C0055010E8
:10D0300001478146A685228597D0FFFFE780A03F64
:10D0400045611753FFFF6700C30B1753FFFFE7024C
:10D05000030983C7950041112A8493F7F707A38436
:10D06000F50032852EC697F0FFFFE780800F8567B9
:10D070002AC46370F50297700000E78020E9224619
:10D08000B24509ED11478146228597000000E780EF
:10D0900060E641011753FFFF6700A306014783467F
:10D0A000F501DDB71753FFFFE702C30101113C0093
:10D0B0003ECAB7070A003ECC3C003ECE83C795006F
:10D0C000AA89328593F7F707A384F5002E8497F099
:10D0D000FFFFE78000098567637DF504A165AA84E9
:10D0E00093858504480897D0FFFFE780600F268569
:10D0F00097700000E78080E12A8929E1914548087E
:10D1000097F0FFFFE78020F6A685480897F0FFFF1D
:10D11000E78060F7CA85480897F0FFFFE780A0F432
:10D12000014781465008A2854E8597D0FFFFE780D2
:10D13000803005611753FFFF670003FC81454808F5
:10D1400097F0FFFFE78020F20349090275BF1753EC
:10D15000FFFFE70223F779711C103ECAB7070F00E3
:10D160003ECC404D1C10AA84AE894808994532C671
:10D1700036893ECE97D0FFFFE780800632464808CA
:10D18000B28597F0FFFFE78000EE630C0902A5452A
:10D19000480897F0FFFFE780C0E62546CA8597203C
:10D1A0000100E78020A4500801478146CE852685EE
:10D1B00097D0FFFFE780202845611753FFFF6700E6
:10D1C000A3F38355C402480897F0FFFFE780A0EB64
:10D1D0000355E402814505C5854785456301F50290
:10D1E000C167FD179305F00F630BF5007D15977070
:10D1F0000000E780208E9305150093F5F50F480891
:10D2000097F0FFFFE78020E683450403480897F086
:10D21000FFFFE78040E583451403480897F0FFFFD0
:10D22000E78060E483552403480897F0FFFFE78018
:10D2300080E583554403480897F0FFFFE780A0E4AA
:10D240009DB71753FFFFE70283E983C79500814627
:10D25000014693F7F707A384F50097000000E780E5
:10D2600040EF1753FFFF6700C3E91753FFFFE702C3
:10D2700003E779713E841C103ECA2E89B7070F0060
:10D28000A1653ECCFD051C10AA84480842C03AC2E4
:10D290003ECE36C432C697D0FFFFE78060F43246F8
:10D2A0004808B28597F0FFFFE780E0DBA246480818
:10D2B000B68597F0FFFFE78000DD12474808BA8582
:10D2C00097F0FFFFE78020DC0248630C08029145DD
:10D2D000480897F0FFFFE780C0D21146A28597204B
:10D2E0000100E7802090500801478146CA852685C5
:10D2F00097D0FFFFE780201445611753FFFF6700B9
:10D3000043E08945480897F0FFFFE78080CF8347D7
:10D3100004002300F50083471400A300F500E1B7E3
:10D320001753FFFFE70203DA83C7950001112A8A2A
:10D3300093F7F707A384F5003285AE8432C697F0E1
:10D34000FFFFE78000E232462A89328597F0FFFF2F
:10D35000E78000DF85676373F902AA894A859770C1
:10D360000000E780A0BA2A8419ED114781464A8659
:10D37000A685528597000000E780C0B70561175366
:10D38000FFFF670063D79387E9FF93F7F70F054720
:10D39000E366F7FE8347F50195EB8947E380F9FEE5
:10D3A0008346F401528501474A86A685970000000E
:10D3B000E78040B4A167D90748083ECC230A0100A2
:10D3C00002CE97000000E780A0B04DBF639EE7004B
:10D3D0008947639EF90093071020231FF50097707B
:10D3E0000000E780C0B76DBF0947E39BE7FA8D47B0
:10D3F000E398F9FA228597700000E78080DF97971D
:10D40000FF1F938727B69C4399E79797FF1F938742
:10D41000279F9C4399C703D5040097800000E780AD
:10D42000A0CE231F040022855DBF1753FFFFE70234
:10D4300003CB01113C003ECAB7070B003ECC3C00B9
:10D440003ECE83C795002A89328593F7F707A384D8
:10D45000F500AE8497F0FFFFE780A0D09317050199
:10D46000C187635AF006A1652A849385E5024808BE
:10D4700097D0FFFFE780C0D6A285480897F0FFFF4E
:10D48000E78060C09797FF1F938787979C43A9EB1E
:10D4900001449375F40F480897F0FFFFE780A0BCA4
:10D4A0009355844093F5F50F480897F0FFFFE78008
:10D4B00080BB9355044193F5F50F480897F0FFFFA3
:10D4C000E78060BA014781465008A6854A8597D013
:10D4D000FFFFE78040F605611753FFFF670063C257
:10D4E000416585460546A2857D1597500000E78079
:10D4F00060BD59DD510597000100E780808F13045E
:10D5000040063344850271B71753FFFFE70223BD7E
:10D510000111B70706003EC683C7950021642A891A
:10D5200093F7F707A384F500AE8428009305A404BD
:10D530000AC40AC897D0FFFFE78080CA30000147BD
:10D540008146A6854A8597D0FFFFE780C0EE97E029
:10D55000FFFFE780E01113049404480822CC230A5B
:10D56000010002CE97000000E78080960561175306
:10D57000FFFF670003B91753FFFFE702A3B4C164BD
:10D580002A8901449799FF1F9389499F130A8002B2
:10D59000FD1497E0FFFFE780E0BD6347A40001456D
:10D5A0001753FFFF670043B5B307440303A7C90A36
:10D5B000BA9703D707006306970083D727006384D1
:10D5C00027010504F9B70545E1BF1753FFFFE7023F
:10D5D00063AF2A8A2E8999C123A00500814981441D
:10D5E000978AFF1F938A4A79614B97E0FFFFE78094
:10D5F000A0BE63C7A4004E851753FFFF6700C3AFEB
:10D600003384640383A70A003E948357040099E798
:10D6100063040900232089008504C1BF4146D285E7
:10D620001305440097100100E780605975F5A28941
:10D63000E5B71753FFFFE702E3A839717C083ED432
:10D64000B7070A003ED67C083ED883C795002A8AD1
:10D65000328593F7F707A384F5002E8932C697F039
:10D66000FFFFE78000B085676373F5083246AA8440
:10D67000328597F0FFFFE780A0AC8547AA8963E871
:10D68000A706A16593858504281097D0FFFFE78042
:10D6900020B5268597700000E78040872A8429ED11
:10D6A0009145281097F0FFFFE780E09BA6852810A2
:10D6B00097F0FFFFE780209DCE85281097F0FFFFB1
:10D6C000E780609A014781463010CA85528597D01D
:10D6D000FFFFE78040D6A1679387770448183EDCB8
:10D6E000230A010202DE97F0FFFFE780607E2161DE
:10D6F0001753FFFF670043A08145281097F0FFFFF5
:10D70000E7806096A685281097F0FFFFE780A09736
:10D710009797FF1F938747BD9C4381CB22856389E1
:10D72000090097D00000E78040248345040271B7C8
:10D7300097D00000E780C022CDBF1753FFFFE7025C
:10D74000639883C795004111AA8993F7F707A384CB
:10D75000F5003285AE84328A97F0FFFFE78060A043
:10D760008567637FF5022A8997600000E780007A69
:10D770002A84914631C58347F50105476387E7024F
:10D7800091C70D476366F704AD461DA893050503D1
:10D7900003250A00414697100100E78040420DE949
:10D7A00041011753FFFF6700239593059508032553
:10D7B0000A00414697100100E7806040814669F504
:10D7C0004A86A6854E8597000000E780C081C9BFC4
:10D7D00083250A001305940897700000E780A029AC
:10D7E00019C1C146F1BF9787FF1F9387A7779C4355
:10D7F00099E79787FF1F9387A7609C4399C7228566
:10D8000097800000E780208A69FD8547A30FF40018
:10D81000228597B00000E780608422859760000031
:10D82000E780E0734E8581464A86A68597F0FFFF24
:10D83000E780607BA1679387570448003EC42302BA
:10D84000010002C697F0FFFFE780806891BF175381
:10D85000FFFFE702438683C795004111AA8993F72A
:10D86000F707A384F50032852E89B28A97F0FFFF6F
:10D87000E780208F85676374F50EAA8497600000A7
:10D88000E780C0682A840DED416B014A978BFF1F2A
:10D89000938BCB6E130C400E7D1B19A833048A03A7
:10D8A00083A70B0B3E948357C40163836705050A66
:10D8B00097E0FFFFE780008BE342AAFE95460DA0AC
:10D8C0008357C501639697029305050303A50A00D4
:10D8D000414697100100E780802E994611E181466C
:10D8E0002686CA854E8597F0FFFFE780C06F85A822
:10D8F00083A50A001305040397700000E780A017B2
:10D90000C14679FD2285231E940097A00000E78080
:10D91000E074228597600000E78060649797FF1F9E
:10D920009387879C9C43A9C323000402228597D038
:10D930000000E78040F04E8581462686CA8597F034
:10D94000FFFFE780406AA1679387070448003EC451
:10D950002302010002C697F0FFFFE78060574101F4
:10D960001743FFFF6700A37889472300F402E1B75C
:10D97000397106DE22DC4AD8800052D456D25AD001
:10D9800026DA4ED65ECE2E8A32892A8B97D0FFFFBA
:10D99000E780407A0605710541998A8A3301A140E2
:10D9A000232224FC231404FC97D0FFFFE780807817
:10D9B00083479A000605350593F7F7072315A4FC5E
:10D9C000A304FA004A85232624FC97E0FFFFE780A2
:10D9D000407993170501C1876340F0025681130116
:10D9E00004FCF2506254D2544259B259225A925A0B
:10D9F000025BF24B21618280AA844A8597E0FFFF97
:10DA0000E7802076AA894A8597E0FFFFE780607566
:10DA1000A1659385C5022A89130544FC97C0FFFFC1
:10DA2000E780007C268597C0FFFFE7804070854532
:10DA300011C94A86CE8597C0FFFFE780C069AA8BCF
:10DA400021E98945130544FC97E0FFFFE780A061C9
:10DA5000A685130544FC97E0FFFFE780C062CE85F2
:10DA6000130544FC97E0FFFFE780E061CA851305DA
:10DA700044FC97E0FFFFE780006101478146130601
:10DA800044FCD2855A8597D0FFFFE780C09AB9B78A
:10DA90008145130544FC97E0FFFFE780C05CA68545
:10DAA000130544FC97E0FFFFE780E05DCE8513059A
:10DAB00044FC97E0FFFFE780005DCA85130544FC46
:10DAC00097E0FFFFE780205C814497D0FFFFE7806D
:10DAD0006066E3D4A4FA83A70B0113971400BA97E6
:10DAE00083D5070099C5130544FC97E0FFFFE78045
:10DAF00080598504D9BF797106D622D44AD000183E
:10DB00004ECE52CC56CA26D25AC8AE893289AA8A7B
:10DB100097D0FFFFE78000620605690541990A8AF0
:10DB20003301A140232A24FC231C04FC97D0FFFFCF
:10DB3000E780406083C7990006052D0593F7F70736
:10DB4000231DA4FCA384F9004A85232E24FC97E01E
:10DB5000FFFFE780006193170501C187634FF00065
:10DB60005281130104FDB250225492540259F249D9
:10DB7000624AD24A424B45618280AA844A8597E034
:10DB8000FFFFE780005EA1659385A5022A89130542
:10DB900044FD97C0FFFFE780A064268597C0FFFF84
:10DBA000E780E058854509C9CA8597C0FFFFE7802F
:10DBB00080552A8B29E18945130544FD97E0FFFF35
:10DBC000E780604AA685130544FD97E0FFFFE780E4
:10DBD000804BCA85130544FD97E0FFFFE780A04A0C
:10DBE00001478146130644FDCE85568597D0FFFF39
:10DBF000E7806084B5B78145130544FD97E0FFFFDA
:10DC0000E7806046A685130544FD97E0FFFFE780A7
:10DC10008047CA85130544FD97E0FFFFE780A046D3
:10DC2000814497D0FFFFE780E050E3DBA4FA83272D
:10DC30000B0113971400BA9783D5070099C51305F4
:10DC400044FD97E0FFFFE78000448504D9BF1743F8
:10DC5000FFFFE702C34883474500404DD5EFFD571E
:10DC60005DC48346940009476363D70A0346B40042
:10DC7000854663EEC6088306E40063CA06085C4571
:10DC8000F9562390D7009787FF1F83C7270F99E383
:10DC9000A304E4009787FF1F938787169C4381E7BF
:10DCA0008947A306F4009787FF1F9387E7639C4388
:10DCB00081E789472306F400970500009385450610
:10DCC000AA841305040197F00000E7802010FD5797
:10DCD000231AF40281471CDC01489787FF1F23ABFE
:10DCE00087089787FF1F93872709232E040304C003
:10DCF000804397D0FFFFE780204E61463306C50280
:10DD0000814522859740FFFFE780604081473E853F
:10DD10001743FFFF6700E33EFD57D5BF1743FFFFE3
:10DD2000E702E33B2A840355450297600000E78041
:10DD3000E01D19E5231E04001743FFFF6700633C45
:10DD40008357E401F5DB930504FF17450100130534
:10DD5000A5ED97E00000E780E014F9BF1743FFFF4F
:10DD6000E702E3372E89A16541119385E5032A84F3
:10DD700036C432C6BE843AC297C0FFFFE780404631
:10DD800012472285BA8597E0FFFFE780C02D324613
:10DD90002285B28597E0FFFFE780E02EA24622852C
:10DDA000B68597E0FFFFE780002E630309029145E7
:10DDB000228597E0FFFFE780C0241146A6859710D3
:10DDC0000100E78020E241011743FFFF6700633352
:10DDD0008945228597E0FFFFE780A02283C70400E2
:10DDE0002300F50083C71400A300F500E9BF174323
:10DDF000FFFFE702C32E83C79500444D054793F705
:10DE0000F707A384F5001C42411183C7070063672D
:10DE1000F7062E842A89B1C003C7D400630FF70226
:10DE20001787FF1F1307C7FD184305C3A386F40018
:10DE300097A00000E780404A83C7D40099E7416576
:10DE40007D1597400000E780403083D72403918BF5
:10DE500089C797E00000E780C0134A85A28597F044
:10DE6000FFFFE7808010A167C10748003EC423027E
:10DE7000010002C697F0FFFFE780800541011743CC
:10DE8000FFFF670003281743FFFFE702432503D77F
:10DE900045008D47AA8441112E8432892E8563E383
:10DEA000E70297E0FFFFE780C02BAA852300090067
:10DEB000268597C0FFFFE780002541011743FFFF3C
:10DEC0006700232497E0FFFFE780A0292AC6228568
:10DED00097E0FFFFE780E028B24585472A862300C8
:10DEE000F900268597C0FFFFE780E01EF9B739717A
:10DEF00006DE22DC26DA80004ED652D456D24AD82C
:10DF00005AD05ECEAE89B284AA8A97D0FFFFE7804E
:10DF1000602106051305250241990A8A3301A140B3
:10DF2000232224FC231404FC97D0FFFFE780801FEA
:10DF300083C7990006054D0593F7F7072315A4FC41
:10DF4000A384F9002685232624FC97E0FFFFE780C1
:10DF5000402193170501C1876340F00252811301EC
:10DF600004FCF2506254D2544259B259225A925A85
:10DF7000025BF24B21618280AA8B03AB040097C045
:10DF8000FFFFE780C01A51E583D74400014985446B
:10DF9000F11793B71700A301F4FC834734FCA16584
:10DFA000C9C79385E504130544FC97C0FFFFE780CC
:10DFB0002023A685130544FC97E0FFFFE780A00A15
:10DFC000DE85130544FC97E0FFFFE780C00B834725
:10DFD00034FC114691E30946DA85130544FC97E0C9
:10DFE000FFFFE78060058144630A0900416B7D1BE8
:10DFF00097D0FFFFE780001363CCA402014781465E
:10E00000130644FCCE85568597C0FFFFE780A042EB
:10E01000B1B7A685130634FC97000000E780E0E660
:10E02000933415002A8986048DBF9385C504A5BF46
:10E030008327C90013971400BA9783D50700638814
:10E040006501130544FC97E0FFFFE780C0038504EA
:10E0500045B71743FFFFE702030679711C103EC462
:10E06000B7070F003EC61C103EC883C79500AA8A9A
:10E07000328593F7F707A384F500AE89328497E0E1
:10E08000FFFFE780000E93170501C187635AF00672
:10E090002A8A228597E0FFFFE780A00C2A89528513
:10E0A000032B040097C0FFFFE780600839ED83571A
:10E0B000440081440544F11793B71700A303F1000E
:10E0C00083457100DA872287CA8652862800970026
:10E0D0000000E780E0C8014781463000CE855685C4
:10E0E00097C0FFFFE7802035A1679387D7034808D3
:10E0F0003ECC230A810026CE97F0FFFFE78040DD6B
:10E1000045611743FFFF670083FEA2851306710078
:10E1100097000000E78060D7AA84094455D13544B0
:10E12000E30055FB4A8597F0FFFFE78000450D446B
:10E1300041D9014497D0FFFFE780C0FE634DA400A2
:10E14000C16B0144FD1B97D0FFFFE780A0FD634E2C
:10E15000A4001544B5B7DC4413171400BA9783D74D
:10E160000700638327030504F1B7D844931714000D
:10E17000BA9703D70700631B7701239027012685F1
:10E1800097A00000E78080DB01441DBF050465BF48
:10E190001743FFFFE70203F383C7950041112A8A63
:10E1A00093F7F707A384F50032852E89328497E030
:10E1B000FFFFE78000FB93170501C1876353F0065B
:10E1C000AA89228597E0FFFFE780A0F92311A1002B
:10E1D0004E85832A040097C0FFFFE78040F539E5AC
:10E1E0008357440085440144F11793B71700A300F7
:10E1F000F1000348110003572100D6875285CE86CF
:10E200002686CA8597F0FFFFE7806006A167F107C1
:10E2100048003EC42302910022C697F0FFFFE7802A
:10E2200020CB41011743FFFF670003EDA2851306D2
:10E23000110097000000E78040C52A84894455D921
:10E240008357210011678544BA97C2071167C183BC
:10E250001307F7EFE36FF7F89787FF1F938787D0D0
:10E260009C4381CB85451305210097500000E78032
:10E270002075835521002285814497C0FFFFE780E8
:10E28000A0E125D923100500228597A00000E78092
:10E2900040CD85B71743FFFFE702E3E183C7950051
:10E2A00041112A8B93F7F707A384F50032852E8A54
:10E2B000328497E0FFFFE780C0EA93170501C1872A
:10E2C0006351F006AA8A228597E0FFFFE78060E9A4
:10E2D0002A895685832B040097C0FFFFE78020E53D
:10E2E00031E58357440081440544F11793B7170083
:10E2F000A301F10003483100DE875A854A87D6869C
:10E300002286D28597F0FFFFE78060F6A167ED07D0
:10E3100048003EC42302810026C697F0FFFFE78035
:10E3200020BB41011743FFFF670063DCA285130692
:10E33000310097000000E78040B5AA8409445DD908
:10E340009167CA97C2071167C1831307F7EF0544A6
:10E35000E362F7FACA8597C0FFFFE780E0D3014484
:10E3600051F9814997D0FFFFE780C0DC63DBA9004A
:10E37000984893971900BA9703D7070005EF2390A1
:10E38000270197D0FFFFE780E0DA1544E384A9F680
:10E39000268597A00000E780C0BC9787FF1F938762
:10E3A00067BC9C430144B9D74A8597500000E78079
:10E3B000C05889B785097DB71743FFFFE70283D0AF
:10E3C00079713E847C083EC82E8AB7071400A16587
:10E3D0003ECAE5057C08AA89080836C4428932C6C7
:10E3E000BA8AC6843ECC97C0FFFFE78060DFCA854B
:10E3F000080897E0FFFFE78000C732460808B285AB
:10E4000097E0FFFFE78020C8A246630A09049D4504
:10E41000080897E0FFFFE780C0BE1D468145974092
:10E42000FFFFE780C0CE63890A089145080897E09E
:10E43000FFFFE78000BD1146A68597000100E78039
:10E44000607A100801478146D2854E8597C0FFFF4C
:10E45000E78060FE45611743FFFF6700E3C9B685AB
:10E46000080897E0FFFFE78000C21C400808D84377
:10E470009355C701858912075183B205D98D97E05D
:10E48000FFFFE78040C01C40080883C5870097E075
:10E49000FFFFE78040BD1C40080883C5A70097E048
:10E4A000FFFFE78040BC1C40080883C5970097E049
:10E4B000FFFFE78040BB85BF8945080897E0FFFF65
:10E4C000E78020B483C704002300F50083C714004D
:10E4D000A300F500BDB71743FFFFE702A3BE83C744
:10E4E00095004111AA8993F7F707A384F5003285B7
:10E4F000AE84328497E0FFFFE780A0C69317050142
:10E50000C187635DF0042A89032A040097C0FFFFD6
:10E51000E780E0C119E9835744000548F11793B734
:10E520001700A307F100814631A81306F100A28568
:10E5300097000000E78060951DC51C459DC783D6E8
:10E54000470001480347F10093078500D2884A86B7
:10E55000A6854E8597000000E78040E641011743FD
:10E56000FFFF670063B909487DBF1D486DBF1743B2
:10E57000FFFFE70223B565715C083EC4B7077B0166
:10E580003EC65C083EC883C795002A8A328593F749
:10E59000F707A384F500AE8997E0FFFFE78040BA54
:10E5A0008357E100E1C78945280097C0FFFFE78056
:10E5B00020C38145280097E0FFFFE780C0AA97C0ED
:10E5C000FFFFE78000C99787FF1F9387E7D19C4330
:10E5D0001774FF1F0344847AAA843334800099C3DC
:10E5E000136424009787FF1F938787819C4399C3F7
:10E5F000136444009787FF1F9387C7969C4399C372
:10E600001364840083D504002800014997E0FFFFCC
:10E61000E78060A783D52400280097E0FFFFE7800C
:10E6200080A683D54400280097E0FFFFE780A0A5DF
:10E6300097D0FFFFE78000AB93150501C18128004B
:10E6400097E0FFFFE78020A4A285280097E0FFFF66
:10E65000E78060A39C446360F90201478146300073
:10E66000CE85528597C0FFFFE780E0DC59611743F4
:10E67000FFFF670063A8DC441314490028003E94A0
:10E6800097E0FFFFE780609683474400034754000C
:10E6900089070607BA978607E36AF5FC83552400C5
:10E6A0002800814A97E0FFFFE780E09D8345440012
:10E6B000280097E0FFFFE780009B83455400280077
:10E6C00097E0FFFFE780209A8347440063C9FA0080
:10E6D000814A8347540063C1FA020509A5BF1C445F
:10E6E00013975A002800BA9783D50700850A97E048
:10E6F000FFFFE7804099C9BF032BC40093975A00DE
:10E7000028003E9B83552B00850A97E0FFFFE7809A
:10E71000809783550B00280097E0FFFFE780A096C5
:10E720004DBF1743FFFFE702839B5C4993E7170048
:10E730005CC997A00000E78020B61743FFFF670081
:10E74000439C1743FFFFE70283992E84814597F08E
:10E75000FFFFE780C0E705C583570500FD172310BD
:10E76000F50009C4835725002310F400970000002A
:10E77000E78060FB01451743FFFF67008398314541
:10E780007DD823100400C5BF1743FFFFE702839322
:10E7900083C7950041112A8A93F7F707A384F500F0
:10E7A00032852E89328497E0FFFFE780809B9317A4
:10E7B0000501C1876356F006AA89C145228597E005
:10E7C000FFFFE780A0802A8B4E85832A040097C034
:10E7D000FFFFE780C09531E9835744002311010012
:10E7E0000544F11793B71700A300F10081440348D3
:10E7F000110003572100D6875285CE862286CA850E
:10E8000097F0FFFFE780A0A6A16793871702480053
:10E810003EC42302810026C697E0FFFFE780406BDD
:10E8200041011743FFFF6700238D13061100A285E6
:10E8300097F0FFFFE7806065AA8409E523110100D6
:10E84000094475B7930521005A8597000000E780B9
:10E8500080EF835721002A84D9DB9777FF1F9387A6
:10E8600067709C4381CB85451305210097500000BC
:10E87000E7800015835521002685314497C0FFFFAE
:10E88000E78080812DD52310050026859790000014
:10E89000E780206D0144A1BF1743FFFFE7022384F7
:10E8A00041112E896C00AA8402C697F0FFFFE78011
:10E8B00000D20DC10357050005072310E50097009E
:10E8C0000000E78040E681473E8541011743FFFF96
:10E8D000670023833247954765DBCA8526859730D5
:10E8E0000000E780400DC147E34005FE3244854704
:10E8F00041462310F40083570900A6851305440000
:10E900002311F40097000100E780C02D228545BF48
:10E910001733FFFFE702037B83C795004111AA8AE3
:10E9200093F7F707A384F5003285AE89328497E028
:10E93000FFFFE780008393170501C1876356F00648
:10E940002A8AC145228597D0FFFFE7802068AA84E4
:10E950005285032B040097B0FFFFE780407D31E92B
:10E9600083574400231101008544F11793B7170022
:10E97000A300F10001440348110003572100DA8786
:10E980005685D2862686CE8597F0FFFFE780208EBB
:10E99000A1679387070248003EC42302910022C664
:10E9A00097E0FFFFE780C05241011733FFFF670088
:10E9B000A374A2851306110097F0FFFFE780E04CD7
:10E9C0002A8409E523110100894475B7268593053A
:10E9D000210097000000E78060ECAA8449FD835580
:10E9E0002100228597B0FFFFE780006B49F50149C0
:10E9F00097C0FFFFE7800074635DA9001848931774
:10EA00001900BA9703D707000DEF03572100239091
:10EA1000E70097C0FFFFE780E07163062503977763
:10EA2000FF1F938727549C4399C703552100975094
:10EA30000000E78080F0228597900000E780605218
:10EA40001DBF050975B795443DB705C19307F00F84
:10EA5000630FF500C547630CF5009307F5FF054507
:10EA60003315F50042054181828001458280416570
:10EA70007D158280B9E91733FFFFE702436603453E
:10EA80000603328497000000E78060FC9305803E17
:10EA9000B305B502C205C18181CD0357E4028547A4
:10EAA00063F8E7001305040197E00000E7802042C7
:10EAB0008357E40241677D176385E700FD1723173D
:10EAC000F4021733FFFF6700C36382801733FFFF31
:10EAD000E702635E004283C79500444D034914007A
:10EAE00093F7F707A384F500834704002209116711
:10EAF0003369F900A167B347F90041112A8BAE8A47
:10EB000063ECE70E834724001307C00EB91793F791
:10EB1000F70F6373F71003473400C14763EEE70E46
:10EB2000834744001307E00793C707086371F70C96
:10EB30008349840083477400A209B3E9F90085671B
:10EB400063F7F90A034A6400834754004E85220A9A
:10EB5000336AFA0097500000E780403B61C123967A
:10EB60002403834B3400137AFA00239A3403238856
:10EB700074032399440393890401631C090023A6A9
:10EB80000402239804024E8597E00000E780603677
:10EB90003DA0034924004A8597000000E78020EB50
:10EBA0002397A402834744004E85A388F402E38D93
:10EBB0000BFCE30B09FC97E00000E780202F979007
:10EBC0000000E780007381460146D6855A8597E0AC
:10EBD000FFFFE7800058A167938797033EC4230295
:10EBE0000100480002C697E0FFFFE780602E410168
:10EBF0001733FFFF6700A34F8544A2862686D6857C
:10EC00005A8597E0FFFFE780C054A1679387970379
:10EC10003EC423029100F1B7BD44C5B79144F1BF92
:10EC20001733FFFFE702034A01111C08404D3EC2A3
:10EC3000B7070F003EC41C083EC62A89AE8997C09C
:10EC4000FFFFE78000D7585C1C5C6346B70E6394F7
:10EC5000E50063E2A70E3385A740B3B7A700B3056D
:10EC6000B7401306803E81469D8D97000100E780E6
:10EC700080B793140501C180A1659385C503480041
:10EC800097B0FFFFE780C0558145480097D0FFFF50
:10EC9000E780603D83550404480097D0FFFFE7807C
:10ECA000803E83552404480097D0FFFFE780A03DB5
:10ECB000814589CCC167FD179305F00F6388F40087
:10ECC000268597500000E780E0E0AA85480097D0AD
:10ECD000FFFFE780403903554404814501CDC167FA
:10ECE000FD179305F00F6307F50097500000E780CC
:10ECF00060DEAA85480097D0FFFFE780C0368345D5
:10ED00006404480097D0FFFFE780E0358345740432
:10ED1000480097D0FFFFE78000355000014781464B
:10ED2000CE854A8597B0FFFFE780E0700561173315
:10ED3000FFFF6700633C814481B71733FFFFE702A1
:10ED4000033A83C7950093F7F707A384F50097006C
:10ED50000000E78020ED1733FFFF6700833A173389
:10ED6000FFFFE702233683C795004111404D93F71B
:10ED7000F707A384F5002A8A3285B284AE8997D03A
:10ED8000FFFFE780003E2A8B268597D0FFFFE780B4
:10ED9000403D2A89268597D0FFFFE780603A931788
:10EDA0000B0163CA0702E177CA97C207C1831167E3
:10EDB00063E3E70293070910C207C1831307B00F8B
:10EDC000637BF70093170901C187AA8A634AF000A1
:10EDD000C54763FE570141011733FFFF6700C33189
:10EDE00097B0FFFFE7802025E31725FFD5B763081D
:10EDF0000B0263060902814463890A02B7077F0098
:10EE000023106405231124057CC05685970000005B
:10EE1000E780E0C39304803EB304950239A0B707AE
:10EE20007F00232004047CC081440355240497E020
:10EE30000000E780A0A3A1C497C0FFFFE78060B7F0
:10EE4000269593D7F44133379500AE97BA9708DCEF
:10EE50005CDCCE85528597000000E780A0DC99E05D
:10EE600023220404A1679387B70348003EC423020A
:10EE7000010002C697E0FFFFE7808005A9BF814738
:10EE800001481CDC232E0403E9B71733FFFFE70218
:10EE9000032597C0FFFFE7802034E1473305F502E3
:10EEA000914597500000E78000C5E55711C5977759
:10EEB000FF1F23A3A7EC81473E851733FFFF6700A1
:10EEC000432485471777FF1F230AF7EA8280173309
:10EED000FFFFE702C3209777FF1F9387A7E98043CF
:10EEE0003DC0835704046390A70683572404639CA2
:10EEF000B7043689B28497C0FFFFE78080AB5C5CC3
:10EF000063C3B7046395B7001C5C63EEA702834735
:10EF1000640463F3F400A6872303F40483477404B2
:10EF200063F39700A687A303F4048357440441675F
:10EF30007D176385E70085072312F4043C4481C7ED
:10EF4000CA85268582971733FFFF6700831B977753
:10EF5000FF1F938727E29C43014599C303C58700A0
:10EF600082801733FFFFE70283170111B7070700FD
:10EF70003EC683C79500584D0AC493F7F7070AC8E1
:10EF8000A384F5002A89AE8411CB1C4283C70700F5
:10EF90002304F70097900000E78000342164930574
:10EFA0005402280097B0FFFFE780802397000000FD
:10EFB000E78020FAAA85280097D0FFFFE780A00A03
:10EFC000300001478146A6854A8597B0FFFFE7805C
:10EFD000804613044402480822CC230A010002CED2
:10EFE00097E0FFFFE780C0EE05611733FFFF670082
:10EFF00043111733FFFFE702830E01117C003ECA65
:10F00000B70707003ECC7C003ECE83C795002E8418
:10F01000AA8493F7F707A384F500A16593855502A9
:10F02000480897B0FFFFE780A01B97000000E7802B
:10F0300040F2AA85480897D0FFFFE780C002500839
:10F0400001478146A285268597B0FFFFE780A03E55
:10F0500005611733FFFF6700C30A9777FF1F938788
:10F0600067D19C43094599C303C597008280977770
:10F07000FF1F938727D09C43094599C303C5D70039
:10F0800082809777FF1F9387E7CE9C43014599C302
:10F0900003C5A70082801733FFFFE702A302011117
:10F0A000B70708003EC683C79500404D0AC493F7D2
:10F0B000F7070AC8A384F5002A89AE8429C414423C
:10F0C000854703C7060063E0E70A834794000946C3
:10F0D00081496380C702B307F740A304E400B33952
:10F0E000F00083C716002305F40097900000E78026
:10F0F000A01E03572403058B19C76386090097D008
:10F100000000E78000E9216493058402280097B09D
:10F11000FFFFE780E00C97000000E78040F4AA853D
:10F12000280097D0FFFFE78000F497000000E780F9
:10F1300080F5AA85280097D0FFFFE780C0F201473D
:10F1400081463000A6854A8597B0FFFFE780A02E54
:10F1500013047402480822CC230A010002CE97E06F
:10F16000FFFFE780E0D605611733FFFF6700C3F8B4
:10F170001733FFFFE702A3F601117C003ECAB70771
:10F1800008003ECC7C003ECE83C795002E84AA8426
:10F1900093F7F707A384F500A165938585024808D6
:10F1A00097B0FFFFE780C00397000000E78020EBE7
:10F1B000AA85480897D0FFFFE780E0EA97000000A3
:10F1C000E78060ECAA85480897D0FFFFE780A0E9B8
:10F1D000500801478146A285268597B0FFFFE7804A
:10F1E000802505611733FFFF6700A3F19777FF1FA5
:10F1F000938747B89C43014599C303C5B7008280F4
:10F200001733FFFFE702A3ED0111B70707003EC662
:10F2100083C79500404D0AC493F7F7070AC8A38433
:10F22000F5002A89AE8405C81C42054783C707003C
:10F230006368F7060347B400630FF700A305F40003
:10F2400097900000E78040098347B400B9CF97D07A
:10F25000FFFFE78040BE21649305B400280097B00B
:10F26000FFFFE780E0F797000000E78060F8AA85DD
:10F27000280097D0FFFFE78000DF0147814630007C
:10F28000A6854A8597B0FFFFE780E01A2904480861
:10F2900022CC230A010002CE97E0FFFFE78040C3A3
:10F2A00005611733FFFF6700C3E597D0FFFFE780D5
:10F2B00020BF55B71733FFFFE70263E201117C005F
:10F2C0003ECAB70707003ECC7C003ECE83C7950000
:10F2D0002E84AA8493F7F707A384F500A165AD05F2
:10F2E000480897B0FFFFE780A0EF97000000E78095
:10F2F00020F0AA85480897D0FFFFE780C0D65008C5
:10F3000001478146A285268597B0FFFFE780A012BE
:10F3100005611733FFFF6700C3DE9777FF1F9387F1
:10F3200067A59C43094599C303C5C700828017336D
:10F33000FFFFE702C3DA01117C00AE843ECAA1657B
:10F34000B70707002A843ECCD1057C0048083ECE92
:10F3500097B0FFFFE780C0E897000000E78020FC3F
:10F36000AA85480897D0FFFFE780E0CF5008014703
:10F370008146A685228597B0FFFFE780C00B056117
:10F380001733FFFF6700E3D71733FFFFE70223D5EB
:10F3900083C7950093F7F707A384F5009700000053
:10F3A000E78020F91733FFFF6700A3D51733FFFF6E
:10F3B000E70243D183C795000329C501411193F7A3
:10F3C000F707A384F5001C4283C90700854763E65D
:10F3D00037079777FF1F938727F19C432E84AA84D2
:10F3E00085CF97000000E78080F389476306F50228
:10F3F000630409028347C900638037032306390188
:10F4000097900000E78040ED83572903898B89C7D7
:10F4100097D00000E780E0B72685A285970000001E
:10F42000E78020F1A167CD0748003EC42302010018
:10F4300002C697E0FFFFE780A0A941011733FFFF55
:10F44000670083CB9777FF1F9387C7929C431D4527
:10F4500099C303C5E70082801733FFFFE70223C883
:10F460000111B70707003EC683C79500584D0AC46F
:10F4700093F7F7070AC8A384F5002A89AE8415C755
:10F480001C4283C7070093968701E18663C4060682
:10F4900085466381D7068346E7006388F600230725
:10F4A000F70097900000E78020E321649305E400D3
:10F4B000280097B0FFFFE780A0D297000000E78008
:10F4C000A0F8AA85280097D0FFFFE780C0B90147C0
:10F4D00081463000A6854A8597B0FFFFE780A0F5FA
:10F4E0003504480822CC230A010002CE97E0FFFF32
:10F4F000E780009E05611733FFFF670083C0173365
:10F50000FFFFE702C3BD01117C003ECAB707070039
:10F510003ECC7C003ECE83C795002E84AA8493F710
:10F52000F707A384F500A165B905480897B0FFFF68
:10F53000E78000CB97000000E78000F1AA8548082B
:10F5400097D0FFFFE78020B2500801478146A2858F
:10F55000268597B0FFFFE78000EE05611733FFFFB8
:10F56000670023BA1733FFFFE702C3B5AA8401443B
:10F570001779FF1F13094980E14997C0FFFFE78012
:10F58000A0C56344A400014519A8330534038327AB
:10F5900009003E958357250063979700110517339F
:10F5A000FFFF670063B50504C9BF032E8500630A2A
:10F5B0000E121773FF1F1303E39A0323030063154F
:10F5C000030029436390061203234E0163150300D1
:10F5D0001D43639907101733FFFFE702C3ADC689C8
:10F5E000428A3E89BA8AB684328BAE8B2A84B5E1D0
:10F5F00003554E0019E501431A851733FFFF6700D5
:10F6000003AFA167A98F116763FBE70097000000B4
:10F61000E78080F5814597F0FFFFE780C01208443E
:10F62000B70700E05841F98F18455CC1B707001FC4
:10F63000F98F1CC55C4991C7610597E00000E78020
:10F64000408BE38A09FA228597900000E78060C624
:10F650005DB7328597C00000E78040430D4349DD28
:10F660001C44116703D54700A167A98F63FBE7001E
:10F6700097000000E78040EF814597F0FFFFE780AB
:10F68000800C0323840093164B01D1828347B3007F
:10F69000035663008588FD8BA305F300FD777D8EFF
:10F6A000558EFD76FD16B204F18E83274301C58E7B
:10F6B000231273012313D3002304530123052301D1
:10F6C000A3044301BDDF228597B0FFFFE78080C917
:10F6D000AA850844B5D1610597D00000E780207F56
:10F6E0008DB71D431A8582801733FFFFE702839D84
:10F6F0000569AA84AE89328A0144FD5A7D1997C0F2
:10F70000FFFFE78020A26347A40001451733FFFFF6
:10F710006700839ED84493171400BA9703D7070055
:10F72000631F37032390570163070A0026859790CC
:10F730000000E780A0809C449DC383D76700B3F797
:10F740002701639E3701D2880148814701478146DE
:10F7500001468145268597000000E78040E50504C5
:10F7600079BF1733FFFFE702E39579711C103EC4A0
:10F77000B7070F003EC61C103EC883C79500AA8A73
:10F78000328593F7F707A384F5002E89328497D04A
:10F79000FFFFE780009D93170501C187635AF006BC
:10F7A000AA89228597D0FFFFE780A09B2A8A4E85F1
:10F7B000032B040097B0FFFFE780609739ED835774
:10F7C000440081440544F11793B71700A303F100E7
:10F7D00083457100DA872287D2864E86280097E01B
:10F7E000FFFFE780E057014781463000CA85568514
:10F7F00097B0FFFFE78020C4A1679387F70348080D
:10F800003ECC230A810026CE97D0FFFFE780406CD4
:10F8100045611733FFFF6700238EA2851306710031
:10F8200097E0FFFFE7806066AA84094455D15285BE
:10F8300097E0FFFFE78060D40D4459D90546D28593
:10F84000268597000000E78060EA2A8451B71733C5
:10F85000FFFFE702C38883550700034627004111D5
:10F860002A842E8532C62EC497E0FFFFE780E0D0C1
:10F8700001C93246A245228597000000E78000E7D3
:10F8800041011733FFFF6700C3871733FFFFE7020C
:10F89000838283C795004111AA8A93F7F707A3844F
:10F8A000F5003285AE89328497D0FFFFE780608B08
:10F8B00093170501C1876357F00AC1452A8A22853B
:10F8C00097C0FFFFE78080702A8D228597D0FFFFC9
:10F8D000E78020892A89228597D0FFFFE78040862C
:10F8E000930705F893F7F70F1307E007AA8B637BDD
:10F8F000F706228597D0FFFFE78080842A8C228537
:10F9000097D0FFFFE780C083AA8C5285032B0400A9
:10F9100097B0FFFFE780A08139E9835744002311A6
:10F9200001008144F11793B71700A300F1000544CB
:10F930000347110083562100938784005685DA8897
:10F9400022885286CE8597F0FFFFE78020A7A16727
:10F95000E90748003EC42302810026C697D0FFFF76
:10F96000E780005741011723FFFF67004378130624
:10F970001100A28597E0FFFFE7802051AA8409E5E6
:10F980002311010009446DB7930521006A8597F0A2
:10F99000FFFFE780A0F02A8441FD835521009356A4
:10F9A000C9001316490185486688E2875E87858A03
:10F9B0005182268597000000E78060BF2A848DBFB2
:10F9C0001723FFFFE702236F83C7950041112A8B9E
:10F9D00093F7F707A384F5003285AE89328497C088
:10F9E000FFFFE780007893170501C1876352F00A93
:10F9F0002A8A228597C0FFFFE780A076AA8A2285FF
:10FA000097C0FFFFE780E0752A89228597C0FFFF36
:10FA1000E7800073930705F893F7F70F1307E007E4
:10FA20002A8C6377F706228597C0FFFFE780407135
:10FA3000AA8C228597C0FFFFE78080702A8D5285AF
:10FA4000832B040097A0FFFFE780606E39E58357A2
:10FA5000440085440144F11793B71700A301F10056
:10FA600003473100930784005A85DE882688D686AE
:10FA70005286CE8597F0FFFFE78040948D4748007F
:10FA80003EC42302910022C697D0FFFFE780404486
:10FA900041011723FFFF67008365A285130631002C
:10FAA00097E0FFFFE780603E2A84894455D993564A
:10FAB000C9001316490185486A88E6876287858AE6
:10FAC0005182D68597000000E78060AEAA8449BFC6
:10FAD0001723FFFFE702035F2A8981440144617A0B
:10FAE000916A176BFF1F130BEB4797B0FFFFE7807F
:10FAF000606463C7A40022851723FFFF6700C35F0C
:10FB00008327090093991400CE9703D50700330784
:10FB10004501420741836364570305C103270B0076
:10FB200019C785453E8597400000E78060E9832737
:10FB300009000504CE972390070085047DB7970040
:10FB40000000E78060A2832709000504CE97239078
:10FB5000070065D5814597F0FFFFE780C0BEF1BF84
:10FB60001723FFFFE702035683C7950041112A8A36
:10FB700093F7F707A384F50032852E89328497C066
:10FB8000FFFFE780005E93170501C187635AF00409
:10FB9000AA89832A040097A0FFFFE780405931E536
:10FBA0008357440085440144F11793B71700A3011C
:10FBB000F10003483100D68752850147CE8626865C
:10FBC000CA8597D0FFFFE780806AA167F5074800E4
:10FBD0003EC42302910022C697D0FFFFE780402F4A
:10FBE00041011723FFFF67002351A285130631004F
:10FBF00097E0FFFFE78060292A8489445DD99767F1
:10FC0000FF1F938727369C4381CF044997B0FFFF9E
:10FC1000E7804052AA85268597400000E78040DAB9
:10FC20001305040197000000E780C0EA2285978051
:10FC30000000E78000338144ADBF1723FFFFE702D8
:10FC4000834783C795004111AA8A93F7F707A384D6
:10FC5000F5003285AE8932842311010097C0FFFF81
:10FC6000E780205093170501C1876354F0062A8A64
:10FC7000C145228597C0FFFFE7804035AA8B52859A
:10FC8000032B040097A0FFFFE780604A21E9835718
:10FC9000440085440144F11793B71700A300F10015
:10FCA0000348110003572100DA875685D28626863D
:10FCB000CE8597D0FFFFE780805BA16793872702FF
:10FCC00048003EC42302910022C697D0FFFFE78080
:10FCD000202041011723FFFF67006341A28513061F
:10FCE000110097E0FFFFE780401A2A8489444DD92C
:10FCF0009767FF1F9387072798433E8901CF0449E1
:10FD000097B0FFFFE7800043AA8526859740000053
:10FD1000E78000CB1305040197000000E78080DB3B
:10FD200097B0FFFFE780004195443DD9930521003E
:10FD30005E8597F0FFFFE78060B6AA8435F11C4826
:10FD40000357210022852390E70097800000E78079
:10FD5000402183270900A9D70355210097400000BF
:10FD6000E780A0BD35BF1723FFFFE702C33483C779
:10FD700095004111AA8A93F7F707A384F50032850D
:10FD8000AE89328497C0FFFFE780A03D931705013D
:10FD9000C1876351F0062A8A228597C0FFFFE7805A
:10FDA000403C2A895285032B040097A0FFFFE7807F
:10FDB000003831E58357440085440144F11793B777
:10FDC0001700A301F10003483100DA8756854A87FE
:10FDD000D2862686CE8597D0FFFFE7804049A1676F
:10FDE000F90748003EC42302910022C697D0FFFFC6
:10FDF000E780000E41011723FFFF6700432FA28514
:10FE00001306310097E0FFFFE78020082A84894429
:10FE10005DD99167CA97C2071167C1831307F7EFCE
:10FE20008544E362F7FA9767FF1F9387A713984308
:10FE3000BE8B01CF044997B0FFFFE780A02FAA85B2
:10FE4000268597400000E780A0B7130504019700BE
:10FE50000000E78020C897B0FFFFE780A02D954401
:10FE60003DD11C48228581442390270197800000C2
:10FE7000E780200F83A70B00B9D74A859740000081
:10FE8000E780A0AB89B71723FFFFE70243252A8449
:10FE90004105B28497000000E780C0C311C52285E8
:10FEA00097800000E780E00B81460146A685228509
:10FEB00097800000E780C04E1C4C89C7DC4799C37F
:10FEC000228582971723FFFF6700A3239767FF1FF1
:10FED000938747EA9C43014599C3138507018280B4
:10FEE0009767FF1F938707E9884382801723FFFFE7
:10FEF000E702E31E9317C600DD8DC2054111C181E3
:10FF00002A8432C697C0FFFFE780E0173246228579
:10FF100011829375F60F97C0FFFFE780C01441016F
:10FF20001723FFFF6700E31D1723FFFFE702831975
:10FF300079713C083ED2B7070C003ED43C083ED64F
:10FF400083C79500AE842A8993F7F707A384F50049
:10FF5000A16593853504481097A0FFFFE7804028EE
:10FF6000C165FD150144176AFF1F130A2A01930A90
:10FF7000400EAE892E8B2EC697B0FFFFE780801E05
:10FF80004205931704014181C183B24563E9A70289
:10FF9000C167FD176387F500481097C0FFFFE78032
:10FFA000800E501001478146A6854A8597A0FFFF25
:10FFB000E780604845611723FFFF6700E3133307BD
:10FFC000540383270A0BBA9703D6C701630A360185
:10FFD000638A3501481097000000E78060F1DA85F8
:10FFE000050451BFB285EDBF1723FFFFE702A30C45
:10FFF00079717C083EC8B70711003ECA7C083ECC28
:020000040001F9
:1000000083C79500AA89328593F7F707A384F50083
:100010002E8997C0FFFFE780C01485676378F504D9
:10002000A165AA848905080897A0FFFFE780401B07
:10003000268597400000E78060ED133415000A0420
:10004000A285080897C0FFFFE780E001A6850808A1
:1000500097C0FFFFE780200325CC014781461008A9
:10006000CA854E8597A0FFFFE780E03C45611723D6
:10007000FFFF6700C307B30754030327CA0ABA97F1
:1000800003D70700631C970003D62700638065052C
:10009000080897000000E780A0E5DE8505042EC66D
:1000A00097B0FFFFE780000D4205931704014181DF
:1000B000C183B245E3E1A7FCC167FD17E38FF5F803
:1000C000080897C0FFFFE78000FC41BFB285F9B781
:1000D000C165FD150144176AFF1F130A2AEA930A36
:1000E00080022E8BAE8B65BF1723FFFFE70223FF35
:1000F00018418347170083460700A207D58FD20710
:10010000D1832390F50083472700034717008D45CF
:10011000A207D98F91832310F60097C0FFFFE780D5
:10012000A0E91723FFFF6700C3FD1723FFFFE702C6
:1001300063F9C16401441769FF1F130929E4930996
:100140008002FD1497B0FFFFE780C0026347A40060
:1001500001451723FFFF670023FA33053403832784
:10016000C90A3E9583570500E38597FE0504D9BF6C
:100170001723FFFFE70203F52A8AAE89B284B68A05
:1001800097400000E78080D819E591473E85172306
:10019000FFFF670063F62A894E8597C00000E7805D
:1001A000E08E2A84638E0A048D476DD103570500C3
:1001B000C547E31D47FD0347F9018546AD47E317F2
:1001C000D7FC8347450081CF4146A6855D0597F062
:1001D0000000E780C09E814755D9AD4745BF130950
:1001E00065012302E500CA85268597100000E78097
:1001F000606231C1A547E38B0AF82302040079B796
:1002000005C183570500E39247F94146A6851905C4
:1002100097F00000E780A09A81472DD99947BDB794
:100220004E8597000000E78080F02A84954739DDED
:10023000130955004DBF4146A685231044012311E3
:1002400034011305190097F00000E780A09922857A
:1002500097800000E780A0EA81470DBF1723FFFFCA
:10026000E702E3E779717C003ECCB7070A003ECE97
:100270007C003ED083C79500B2842E8493F7F707A5
:10028000A384F5001306A1002A892C002685970077
:100290000000E780A0E5A16528088D0597A0FFFF75
:1002A000E78000F490408355A10003558100854606
:1002B00097000000E78000ECAA84AA85280897C070
:1002C000FFFFE78040DA0356A1008355810028082C
:1002D00097000000E780C0C1300801478146A28531
:1002E0004A8597A0FFFFE7800015854748103ED458
:1002F0002302910202D697D0FFFFE78060BD4561DF
:100300001723FFFF6700E3DF1723FFFFE70223DD6B
:1003100079717C003ECCB7070A003ECE7C003ED00F
:1003200083C79500B2842E8493F7F707A384F50062
:100330001306A1002A892C00268597000000E7807B
:10034000E0DAA16528088D0597A0FFFFE78040E966
:1003500090408355A100035581008146970000001D
:10036000E78040E1AA84AA85280897C0FFFFE780BC
:1003700080CF0356A1008355810028089700000014
:10038000E78000B7300801478146A2854A8597A0DB
:10039000FFFFE780400A48102302910202D402D6F0
:1003A00097D0FFFFE780C0B245611723FFFF6700CA
:1003B00043D51723FFFFE70283D297000000E780B1
:1003C00060DB1723FFFF6700C3D39767FF1F938787
:1003D000A79A884382801723FFFFE70243D0835701
:1003E00025004111AE842A842307B10017F5FFFFD1
:1003F000130525466C002316F10097A0FFFFE78048
:10040000804591C4228597800000E780E0D6FD57A3
:100410002310F40013062002814513055400972091
:10042000FFFFE780C0CE41011723FFFF670063CDC8
:100430001723FFFFE70203C979717C003ECCB707A1
:100440000A003ECE7C003ED083C79500AA89AE84C8
:1004500093F7F7073285A384F5001306A1002C005B
:1004600097000000E78080C8035581001144974041
:100470000000E780A0A915C50355A100014497B06D
:100480000000E780A06011CD03570500835781006D
:1004900045446318F700854597000000E780E0F3C6
:1004A0000144216993053900280897A0FFFFE780E0
:1004B00020D3A285280897C0FFFFE780C0BA035663
:1004C000A10083558100280897000000E78040A222
:1004D000300801478146A6854E8597A0FFFFE7803B
:1004E00080F548104AD42302810202D697D0FFFF3C
:1004F000E780009E45611723FFFF6700E3BF1723D6
:10050000FFFFE70223BC9767FF1F9387A7862A8414
:1005100088432E8915C5035745038357C4016311CA
:10052000F7022326050223180502410597D0000093
:10053000E780209C6306090097800000E78060DB6D
:1005400081449769FF1F938969A3130A800297B0BA
:10055000FFFFE78020C263C4A4049767FF1F93874F
:10056000278A9C4399C70355C40197200000E78060
:10057000C0BD63070900228597800000E780C0A006
:100580001306400E814522859720FFFFE78020B8A3
:10059000FD57231EF4001723FFFF6700E3B53385E3
:1005A000440383A7C90A3E95035705008357C40136
:1005B0006317F700CA8597000000E78000E2850412
:1005C00079B71723FFFFE702E3AF83C79500411117
:1005D000AA8993F7F707A384F5003285AE8497C004
:1005E000FFFFE78000B885676378F5042A899740A4
:1005F0000000E780A091014401CD83D7040031447D
:1006000063882701854597000000E78080EF01445B
:100610004E85A2864A86A68597D0FFFFE780A09CDC
:10062000A1679387170448003EC42302810002C6D5
:1006300097D0FFFFE780C08941011723FFFF6700C4
:10064000A3AB1723FFFFE702E3A79757FF1F93878B
:100650006772804329C4014597C00000E7800021EC
:1006600081470148C1641CDC232E040323200404B9
:100670001769FF1F1309899001449309400EFD1467
:1006800097B0FFFFE78000AE634FA400814517F5E8
:10069000FFFF1305857F97A0FFFFE780C01B17238F
:1006A000FFFF670063A5330534038327090B3E95DD
:1006B0008357C50163879700854597000000E78051
:1006C00040E4050475BF9357050113D78700A38045
:1006D000F50093170501C183A1832380E5002381E1
:1006E000F500A381A50082801723FFFFE702239F67
:1006F0002300050083C71500A300F50083C725006C
:100700002301F50083C73500A301F50083C7450029
:100710002302F50083C75500A302F50083C76500D7
:1007200093059500A30305002303F50023040500AA
:10073000328597000000E78040F91723FFFF67002C
:10074000439C1723FFFFE702E3974111E9540DCDC6
:1007500085CD93F9C5FF2E842A89AA84338AA900FE
:10076000B7EA040063189A020D88854411CCB7E7F4
:1007700004009C5F82972AC622866C0033053901EB
:1007800097E00000E7800046268541011723FFFF20
:100790006700839683A78A039104829793170501C4
:1007A000C183A183A38EF4FE93570501238FF4FE2A
:1007B000A183238EA4FEA38FF4FE6DB763E6D5025A
:1007C0001723FFFFE702A391B28741113686BE854A
:1007D00036C697E00000E780E040B246410136852A
:1007E0001723FFFF6700E391814636858280838768
:1007F00005001387F5003D05FD8793F777088346CD
:1008000007007D158606B58FA300F5006307B700C6
:100810007D17834717009D83DDB782801723FFFF75
:10082000E702E38BB7E7040083A7070932872A862C
:100830003A858297133515001723FFFF6700638CF5
:1008400015C181478DC11723FFFFE7024389414648
:1008500097E00000E780003985473E851723FFFFBA
:100860006700238A81473E8582801DCD1723FFFFC5
:10087000E702E386414681452A849720FFFFE7800F
:10088000008941468145130504039720FFFFE78057
:1008900000880147C1672322040438C87CC8054585
:1008A0001723FFFF6700E3850145828081473DCD27
:1008B000B5CD1723FFFFE7028382B2842E8913068A
:1008C000800581452A849720FFFFE7804084CA8500
:1008D00024C4268597000000E780C0F64146814584
:1008E00022859720FFFFE78080823044A285228501
:1008F00097000000E780C0F293040401A2852685DA
:1009000097000000E780E0EEA6851305040297003B
:100910000000E78000EE228597000000E78020F5C8
:1009200085473E851713FFFF6700A37D3E858280C4
:100930001713FFFFE70203794111E9540DCD85CD6F
:1009400093F9C5FF2E842A89AA84338AA900B7EABD
:100950000400639844030D88814411CCB7E7040078
:100960009C5F82972AC622866C003305390197E086
:100970000000E7802027268541011713FFFF67004D
:10098000A37783A78A039104829793170501C183F4
:10099000A183A38EF4FE93570501238FF4FEA18358
:1009A000238EA4FEA38FF4FE6DB765CD1713FFFF52
:1009B000E7024371B28411E605451713FFFF670094
:1009C000A3732A842E890145EDD93C487848B3E6C3
:1009D000E700E5D69386F7FFB3B7F6007D17032A45
:1009E0004404BA9734C87CC863050A06C149130594
:1009F0000A03B38949412295637D3601B2862E866A
:100A0000A68597000000E780A0DB7C40BE9464C010
:100A100065B7CE862E86CE8597000000E78040DA47
:100A2000C114D2944E9923220404A2879306040190
:100A300003C7070003C607038507318FA38FE7FEAF
:100A4000E398F6FE3044A285228597000000E780F7
:100A500020DD2699C1493306994063EC9900A9DC51
:100A6000A686A6851305040397000000E78040D5FD
:100A700079BF8147B306F4003307F6000347070048
:100A800083C5060085072D8F2380E600E39437FF9A
:100A90003044A285228597000000E78060D8C11409
:100AA0005DBF014582800DC11713FFFFE70223637D
:100AB0001306800581459710FFFFE78040650545D7
:100AC0001713FFFF6700E36301458280814749C533
:100AD000C1C51713FFFFE7028360FC4141462E8426
:100AE000AA846399C70413860501A2878146C1457C
:100AF00003C7070003C507038507298F3305D60001
:100B0000034505008506298FA38FE7FEE392B6FE15
:100B10003044A285268597000000E78060D02285BA
:100B200097000000E78060F885473E851713FFFFB8
:100B30006700235D138507031D8E8145229597105D
:100B4000FFFFE780C05C7C40130700F81306040237
:100B5000A2972388E70251BF3E8582801713FFFFCB
:100B6000E702E3576D712E84B284AA8590102800A5
:100B7000368997000000E780A0D309EDD55725A05E
:100B800050400C40280097000000E78040E27DD5EF
:100B9000FD142104F5F42C004A8597000000E7803D
:100BA00020F3814761DD3E8551611713FFFF670028
:100BB00043551713FFFFE702835241112EC432C67B
:100BC0002C00054697000000E78080F941011713CB
:100BD000FFFF670003531713FFFFE70243500111A4
:100BE0002A842EC602C802CA02CC02CE97E00000B8
:100BF000E780C023B2462A86A28508089700000035
:100C0000E78060FB1375F50F05611713FFFF6700A1
:100C1000434F1713FFFFE702834C7971B2872A8491
:100C200021462308B10013051101BE853AC436C61A
:100C300097E00000E78000FBB246930591013685FE
:100C400097000000E78060A82285141035460C0844
:100C500097000000E78020F62A84224701E9214618
:100C60000C103A8597E00000E780C0F722854561C7
:100C70001713FFFF6700E3481713FFFFE702234640
:100C80007171AE84AA850A85328497000000E780DE
:100C900060BB11C90A86A685228597000000E780FF
:100CA00020B8814711E1C5473E854D611713FFFF0D
:100CB000670023451713FFFFE702633F1D712A8A70
:100CC000B289BE8435468547130511012E8CB68A3C
:100CD0003A8BC28C468D2308F10097E00000E78034
:100CE00060F010100C085285231F010097000000CF
:100CF000E780C0F82A843DEDA1476313FD08930700
:100D0000900591E0E5473546E285130511011399F9
:100D10000A012308F1001359090197E00000E78058
:100D200060EC1357890093978A00D98F90080C08BC
:100D30005285231FF10097000000E78020F42A84E9
:100D400015E9A1E49387FA0091831379F9003EC66F
:100D5000631309004149668B8144C14B854DB247FD
:100D6000639F970C6A868C0033855C0197E00000D6
:100D7000E78040E7228525611713FFFF6700E33610
:100D800093079004C9F0A547BDBF834701050947F4
:100D9000C14B2308F10083471105A58FA308F1007B
:100DA00093872400814463E1FB04014714083386E0
:100DB000E6008C08B386E400BA95DA9683C606008E
:100DC00083C505000507AD8E2300D600E390E7FE3E
:100DD0004147639CE70490080C0852859700000087
:100DE000E780C0E925D181A0B3069B00BA8710082F
:100DF000B305F60090083E9603C5060003460600BC
:100E000085078506298E2380C500E39277FF998F99
:100E100090080C085285BE9497000000E78000E619
:100E20008947014749D12A84B1B790083E960346C5
:100E300006001408BE962380C600850759BFB24736
:100E400085046387971481471808B306F70098084C
:100E50003E973386F90003470700034606008507DF
:100E6000318F2380E600E39177FF90080C085285CC
:100E700097000000E78080E05DF53546E2851305C8
:100E800011012308B10197E00000E780A0D5139776
:100E900004014183939784002183D98F10180C0893
:100EA0005285231FF10097000000E78020DD25FD1B
:100EB000814710183387F9003E9603470700034621
:100EC0000600B306FB008507318F2380E600E3921E
:100ED00077FF65A81808B306F70098083E97338691
:100EE000F90003470700034606008507318F23807A
:100EF000E600E3E127FFCA87639E770990080C08A4
:100F0000528597000000E78060D711FD8147980067
:100F1000B306F700900818103E973E960347070067
:100F2000034606008507318F2380E600E39177FFB3
:100F30003546E285130511012308B10197E0000051
:100F4000E78040CA1397040141839397840021836B
:100F5000D98F10180C085285231FF100970000004C
:100F6000E780C0D1E31105EC814710183387F90001
:100F70003E960347070003460600B306FB008507BD
:100F8000318F2380E600E3E227FFC109410BC1BB9B
:100F9000814785B79408BE9683C6060018083E9719
:100FA0002300D700850789BF638006321713FFFF30
:100FB000E702E30F59712A84BE89B28B8547354613
:100FC000130511022E8B468C4289BA8A368A230079
:100FD000F10297E00000E780E0C010180C102285B5
:100FE0002317010297000000E78040C9631805122B
:100FF000A147631FFC069307900563930900E5472B
:101000003546DA851305110293140A012300F10213
:10101000C18097E00000E780E0BC93178A0013D7F7
:101020008400D98F90080C1022852317F1029700B5
:101030000000E780A0C47DE1639209049307FA00F1
:10104000BD88918391E0C144C207C183DE8C814A8F
:101050003EC6414DB24763E2FA0E6286B3854B014C
:10106000881097E00000E78080B54DC93D557DA010
:1010700093079004E39609F8A54759B783470105FC
:101080000947C14C2300F10283471105B3C7F9009A
:10109000A300F10293872900814963E1FC048146A2
:1010A00018103306D7008C083387D900B6955697A9
:1010B0000347070083C5050085062D8F2300E60042
:1010C000E390D7FE41476390E70690080C10228515
:1010D00097000000E78080BA35D189A0B3863A0135
:1010E000BA871010B305F60090083E9603C50600B7
:1010F0000346060085078506298E2380C500E392F6
:1011000097FF3387EC4090080C102285BA9997001E
:101110000000E780A0B68947014741D165611713F8
:10112000FFFF670083FC90083E96034606001410FC
:10113000BE962380C600850779B7B247850A939982
:101140000A01939D8A0093D909016391570F85473E
:101150003546DA85130511022300F10293D989007F
:1011600097E00000E78000A8B3ED3D0190000C106F
:1011700022852317B10397000000E78020B059FDB6
:101180008147A68963EA970626860C084A8597E078
:101190000000E78020A581471810B306F70010086B
:1011A00098083E973E9603470700034606008507CA
:1011B000318F2380E600E3E197FE639FA905900845
:1011C0000C10228597000000E78040AB21F9814791
:1011D0009810B306F700900818183E973E960347FC
:1011E0000700034606008507318F2380E600E39160
:1011F000A7FF4109C10CB9BD18089000B306F7005C
:101200003E963387FC000347070003460600850728
:10121000318F2380E600B5B798084E970347070043
:101220001C10CE972380E700850941BF85473546CE
:10123000DA85130511022300F10293D9890097E0A2
:101240000000E780209AB3ED3D0190000C1022854C
:101250002317B10397000000E78040A2E31005ECDC
:10126000814718089000B306F7003E963387FC00CC
:1012700003470700034606008507318F2380E600F9
:10128000E391A7FF41460C084A8597E00000E780FC
:10129000609581471810B306F700100898083E972C
:1012A0003E9603470700034606008507318F2380DB
:1012B000E600E391A7FF90080C102285970000003C
:1012C000E780C09B1DD599BD7D5582801713FFFF18
:1012D000E702E3E001112A842E859305510032894B
:1012E00002C002C202C402C69304740097F0FFFF5A
:1012F000E780A03D1D46A6851305910097E00000FC
:10130000E780408E10088A854A8597000000E780B4
:10131000E09619ED93071400180883C607000346EA
:10132000070085070507B18EA38FD7FEE397F4FE6C
:1013300005611713FFFF6700C3DC1713FFFFE70208
:1013400063D82E848C414111AA8983871500328984
:10135000914463D30700A1449757FF1F9387C7F8B1
:101360009C43A1C7C1CA8D472310F10083C7250044
:101370004A852301F10083C73500A301F10083C72B
:1013800045002302F10083C75500A302F10083C783
:10139000650093059100A30301002303F1002304DA
:1013A000010097F0FFFFE78040320C404A860A8533
:1013B00097F0FFFFE7808033032804008356440042
:1013C000A6881D0881470147E51642868A854E8515
:1013D00097000000E780408E2A8919E5A6852285BE
:1013E00097B0FFFFE780E0C14A8541011713FFFF77
:1013F000670083D04A860A8597F0FFFFE780002FB9
:101400006DB71713FFFFE702E3CB2E848C41411128
:10141000AA89838715003289914463D30700A144C8
:101420009757FF1F938747EC9C43A1C7C1C68D47C1
:101430002310F10083C725004A852301F10083C7EB
:101440003500A301F10083C745002302F10083C7E3
:101450005500A302F10083C7650093059100A30323
:1014600001002303F1002304010097F0FFFFE78050
:10147000C0250C404A860A8597F0FFFFE7800027C9
:1014800083564400032804008A85858EC2061D0801
:10149000C1822312D400A68881470147E5164286FF
:1014A0004E8597000000E78060B041011713FFFFF1
:1014B000670083C44A860A8597F0FFFFE780002310
:1014C0004DBF1713FFFFE70283C1B335B000011111
:1014D00085052A891315F601336515012308B10026
:1014E0009305110136843AC632C03EC442C297F019
:1014F000FFFFE780801DA2471248425593D6870020
:10150000230BF1009305910193578800A30AD100A2
:10151000A30BF100230C010197F0FFFFE780E01A15
:101520003247024603280400B337E00083564400E4
:101530009207914411C2A1444A85A68842860C08AC
:1015400097F0FFFFE78040772A8919E5A685228575
:1015500097B0FFFFE780E0AA4A8505611713FFFFF8
:10156000670023BA1713FFFFE702C3B501113EC698
:101570008647B335B0008505AA891315F6015D8D40
:101580002308B1009305110136843A89B28442C41C
:1015900046C297F0FFFFE780401322489248164565
:1015A00093578800A30AF1009305910193D788000F
:1015B000230B0101A30BF100230C110197F0FFFF96
:1015C000E780A0103247104083564400B337E00054
:1015D000920703280900914891C0A1480C084E8544
:1015E00097000000E780809CAA8401E983554400AD
:1015F0004A8597B0FFFFE780C0A0268505611713D5
:10160000FFFF670063AFAA959307F00F170701006C
:10161000130707656317B50013C5F7FF1375F50FBB
:10162000828005058346F5FFB58FBA9783C707000B
:10163000D5B70357450014419307F00F1706010073
:1016400013060662369742074183139506014181CE
:10165000631BE500AD8FB29703C50700130515F3B3
:10166000133515008280850603C5F6FFA98FB29752
:1016700083C70700D9BF1713FFFFE70243A6B2874E
:1016800036842E86BA86AA853E85BA8497F0FFFFF7
:10169000E7806052634F0500228597D00000E78005
:1016A000E0782A86A686A285268597F0FFFFE78048
:1016B00080501713FFFF6700C3A41713FFFFE70253
:1016C00063A05D712A8BAE8A170501001305C5560C
:1016D0002C00B284368ABA893E8997F0FFFFE780F2
:1016E000C04F2A845DE134104146DA85280097F026
:1016F000FFFFE780404C2A8449E98547A303F100B6
:10170000A6C2930771002408BEC4A68685470D466D
:101710002C18281002DC02DED6C0BEC697F0FFFFF0
:10172000E78000442A8435E183477102A6860D468E
:1017300093F7F7072300FA00C1473EDE2C188947CC
:10174000281026DCA303F10097F0FFFFE78040415B
:101750002A8405ED4146A6854E8597D00000E78096
:1017600060488D47A6860D462C182810A303F1006B
:1017700097F0FFFFE780C03E2A8401E94146A68535
:101780004A8597D00000E780E04522856161171304
:10179000FFFF670063961713FFFFE702439497F775
:1017A00000009387E7A0984383C7470079712A898F
:1017B000AE84170501001305A5480C083AC423069A
:1017C000F10097F0FFFFE78040412A8405ED1410F7
:1017D0004146CA85080897F0FFFFE780C03D2A848C
:1017E00015E1140815462C00081097F0FFFFE7805C
:1017F000803C2A8401E921462C08268597D00000E8
:10180000E780403E228545611713FFFF6700638F25
:101810001713FFFFE702A38C97F700009387479900
:101820009C477971AA842E84170501001305C541D0
:101830000C083EC697F0FFFFE780203A0DE9141030
:101840004146A685080897F0FFFFE780C03605E10E
:10185000140811466C00081097F0FFFFE780A035D0
:1018600019E58347F10193F7F7032300F40045617D
:101870001713FFFF6700E3881713FFFFE7022386B4
:101880003688A14881470147E54697F0FFFFE7808A
:10189000A0421713FFFF6700C3861713FFFFE7027D
:1018A00003843688A14881470147E54697F0FFFF4A
:1018B000E780C06F1713FFFF6700A3841713FFFFB4
:1018C000E702E38101112A842E850C0832C697F0C5
:1018D000FFFFE780803009ED3247970601009386CD
:1018E00026351008C145228597000000E780E0D822
:1018F00005611713FFFF6700C3801703FFFFE702AF
:10190000037E4111C1472EC032C48A8509463EC2BA
:101910003EC697F0FFFFE780A02441011703FFFFB9
:101920006700237E1703FFFFE702637B4111AE864A
:1019300013061009AA850A8502C002C202C402C6A3
:1019400097F0FFFFE780202741011703FFFF6700A3
:10195000437B1703FFFFE702837832879706010076
:101960009386062F2E869305000297000000E780DD
:10197000C0D01703FFFF6700C3781703FFFFE7021C
:1019800003767971C1472ACC2ED032D42C080D466B
:1019900028003ECE3ED23ED602C402C602C802CACB
:1019A00097F0FFFFE780C01B45611703FFFF67004B
:1019B00043751703FFFFE70283720111AA842E8487
:1019C00017050100130545298A8597F0FFFFE78079
:1019D000C02015E514084146A6850A8597F0FFFF4B
:1019E000E780601D09ED8347E1010347F101A2078C
:1019F000D98FCA07C9836177D98F2310F400056195
:101A00001703FFFF6700E36F15CD1703FFFFE70222
:101A1000036D9747FF1F9387A73A90439745FF1F92
:101A20009385453A1745FF1F1305853597D000006C
:101A3000E78000C51745FF1F130585341703FFFF17
:101A40006700236C1745FF1F1305853382808DCDFA
:101A50001703FFFFE702A3689747FF1F93874736E7
:101A6000944301112E840A869745FF1F938585357F
:101A700097D00000E78040C60A85029401450561C1
:101A80001703FFFF6700E3677D5582801703FFFFA1
:101A9000E702E36497D00000E78080D19747FF1FFB
:101AA00023A0A73217F5FFFF1305E5C997B0000083
:101AB000E780C0741703FFFF6700A3641747FF1F89
:101AC000130747329317150008433E95FD5723101F
:101AD000F50082801703FFFFE70263602A84084055
:101AE00009E51703FFFF6700C3611C4158401CC094
:101AF0006313E5005CC08347550023200500F99B74
:101B0000A302F50097A0FFFFE780207CC9BF170361
:101B1000FFFFE702235B9747FF1F9387A72E98439A
:101B20002A8411CB8347350093F7070289C70355F1
:101B30000500894502971305440197B00000E7802E
:101B4000403B835504000355E40097300000E780D4
:101B5000A00C485819C597A0FFFFE7800077232AFB
:101B600004021305840397000000E780E0F6814437
:101B7000B1499790FFFFE780206A63CBA4028347B7
:101B800034002320040493F727FCA301F400004849
:101B90009790FFFFE7804069131615008145228565
:101BA0009700FFFFE780A0561703FFFF6700C354AD
:101BB000B38734030329040385043E994A859700BB
:101BC0000000E78060F12304090065B78347350012
:101BD00093F7070299E3014582808357E500E39C70
:101BE000B7FEC167FD176316F600054582800545FF
:101BF00099A81703FFFFE702834E93170601C187D9
:101C0000B2842A8401496359F002835705009DCBB1
:101C100001456367F600034584003E953325A60021
:101C20001375F50F0DA01C4813171900BA9783D729
:101C30000700E38E97FA05099790FFFFE780C05EE3
:101C4000E343A9FE01451703FFFF6700834B17031A
:101C5000FFFFE7022347AE89AA849790FFFFE78042
:101C600060522A8497D0FFFFE780A02EAA86014702
:101C70001306840197050000938585E41745FF1F2F
:101C8000130585169790FFFFE780E0182A8925C97C
:101C90008C441304C50022859E0593F5050897A082
:101CA000FFFFE780403CCC4083877400E18163DD27
:101CB000070493E50508228597A0FFFFE780A03A77
:101CC0000D4693854400228597A0FFFFE780C0362C
:101CD00083D50400228597A0FFFFE780E03D83D5F0
:101CE0002400228597A0FFFFE780003D03D649002E
:101CF00083A50900228597A0FFFFE780E0334A858E
:101D00001703FFFF6700433F93F5F5076DB7170310
:101D1000FFFFE702C33C01112A84328532C697A037
:101D2000FFFFE780E0279780FFFFE780C030835701
:101D300004001747FF1F130767243246231BF100D7
:101D4000930700F8A30DF1001C471843231AA100C4
:101D50008983858BB307F740B28548083ECE231CA4
:101D60000100230D010097000000E78080EE05616F
:101D70001703FFFF6700E3381703FFFFE702833411
:101D8000004101453DC49304C40026853289AE89D3
:101D900097A0FFFFE780C02495452A8A2685035B2C
:101DA000040197A0FFFFE7802021268597A0FFFF71
:101DB000E780603E8D45AA8A268597A0FFFFE780D1
:101DC000A01F268597A0FFFFE780E03C5C48420A01
:101DD000135A0A01D2975CC423186401814763989F
:101DE0003A0146054D81330625419337160013F518
:101DF000F70F1703FFFF670023301703FFFFE7020A
:101E0000832B89692A8BAE8B328AB68A814401443E
:101E1000314CFD199790FFFFE780004063CDA4008F
:101E20009790FFFFE7804042018D33B5AA0017036A
:101E3000FFFF6700C32B3389840383270B003E9980
:101E400063170A008347890085043E94E1B703566F
:101E50000A00DE854A8533F6C90097000000E78056
:101E6000E0F16DD10545E1B71703FFFFE702232736
:101E700001112A847C000355E5003ECAB70707001C
:101E80003ECC7C003ECE97200000E78020082A89C7
:101E90008545480897A0FFFFE78020399945480805
:101EA00097A0FFFFE780E015AA844A8597200000ED
:101EB000E780A0082380A4009747FF1F9387070CA3
:101EC0009C434166130606F09396870113D787015A
:101ED000558F93D68700F18E558FA207B706FF0066
:101EE000F58FD98F11462C00138514003EC497D06E
:101EF0000000E78020CF5008A38204008945228596
:101F000097000000E780E0E019C9AA851305840363
:101F100097A0FFFFE780E0313C4085073CC00561AA
:101F20001703FFFF6700E31D1703FFFFE702231BF3
:101F30009790FFFFE78040312A8405049790FFFFC8
:101F4000E780802F3305A402F14791453305F50260
:101F500097200000E78020BA11E565551703FFFFC1
:101F60006700231A9747FF1F23A6A7E89790FFFF54
:101F7000E780802D2A8405049790FFFFE780C02B1F
:101F80003305A4028945060597200000E780A0B626
:101F900069D59747FF1F23A7A7E49790FFFFE78026
:101FA000A02A2A8405049790FFFFE780E0283304E5
:101FB000A4029747FF1F239987E29790FFFFE780CE
:101FC000A0282A849790FFFFE7800027930714003A
:101FD0003385A7029747FF1F2399A7E097070100C2
:101FE0009387478B1747FF1F2324F7E00145BDB7B1
:101FF0001703FFFFE702030DAA842E8901449749C6
:10200000FF1F9389A9F7130A80069790FFFFE780C7
:10201000A0226347A40001451703FFFF6700C30D1B
:102020003305440383A709024A86A6853E95970097
:102030000000E780E0B919E10504C1BF0545E9BF2B
:102040001703FFFFE7022307AA8A2E8BB28B368C79
:102050003A8A814401448149974CFF1F938C0CF2CA
:10206000130D80069790FFFFE780001D63C9A40051
:1020700011E085494E851703FFFF67004307338949
:10208000A40383A70C025E86D6853E994A859700F5
:102090000000E780E0B31DC19790FFFFE780C01A02
:1020A0000544636D4501D2866286DA85130509030E
:1020B00097000000E780A0D411C1854985045DB771
:1020C0001703FFFFE7020300C16441112A8901449D
:1020D0009749FF1F938989EA130A8006FD1436C6C3
:1020E00032C42EC29790FFFFE7800015924522462A
:1020F000B2466348A400014541011703FFFF670092
:10210000A3FF3305440383A709023E9509C683470D
:102110003500C18B9DC791C68347350093F70702F1
:102120008DC3630699008357E500639C270103571D
:10213000050001CB63E7E50083478500BA97E3CD4F
:10214000F5FA050469BF1703FFFFE702A3F7C164AF
:102150002A8901449749FF1F938949E2130A80069F
:10216000FD149790FFFFE780200D6346A40017033E
:10217000FFFF670063F83305440383A709023E9518
:102180008357E500638A97006304990063962701EB
:1021900097000000E780E0970504E1B71703FFFF11
:1021A000E702E3F089692A8AAE8A328BB68B8144D2
:1021B000174CFF1F130C8CDC930C8006314DFD195E
:1021C0009790FFFFE780400763C6A4001703FFFF57
:1021D0006700A3F13389940383270C028355CA0156
:1021E0005A863E994A8597000000E780609E31C17B
:1021F000814D15A03384AD038327090303D60B005B
:10220000D68533F6C9003E94228597000000E7800A
:10221000E0B609E9850D9790FFFFE780E0FFE3CB8B
:10222000ADFC01A8228597000000E780E08A230426
:102230000400850471B71703FFFFE702C3E7416994
:10224000AA8A014A174BFF1F130B4BD37D19C14BB1
:10225000054C9790FFFFE78020FE6346AA00170316
:10226000FFFF6700C3E893098006B3073A03832999
:102270000B02BE9983D7E900638E270163842A018C
:10228000639A570103A4890301E84E859700000073
:10229000E780C0BD050A75BF8357040163997709BC
:1022A0009304C400268597A0FFFFE78060D385458F
:1022B0002A8D2685835C040197A0FFFFE780C0CFAD
:1022C000268597A0FFFFE780A0E762056185635937
:1022D00005048D45268597A0FFFFE780E0CD894561
:1022E000268597A0FFFFE78020CD8945268597A00A
:1022F000FFFFE78060CC8545268597A0FFFFE7803C
:10230000E0CC83470500094793F7F707639AE70096
:102310009945268597A0FFFFE78040CBA302850162
:102320004848337D2D01231894016A9548C4004024
:10233000A1BF1703FFFFE70283DA37E40400832716
:10234000041D82979747FF1F83C747B01715FF1FCC
:102350001305C51FA300F5008327441C829783271C
:10236000841C81461306F00F8145014582971703AF
:10237000FFFF670003D91747FF1F1307279D184367
:102380009745FF1F83C585AC9747FF1F938787AA93
:1023900083468703034697036397D5009747FF1F3C
:1023A0002386C7AA828083C587010347A7036317D3
:1023B000B6009747FF1F238BE7A8828003C68701DB
:1023C0006317C7009747FF1F2382D7A8828083C661
:1023D0008701130750026319D7009307600217475C
:1023E000FF1F2305F7A6828083C6870113066002BC
:1023F0006315D60093077002DDB783C7870155BF09
:102400009747FF1F938707A3D44B0947638DE608BF
:102410001703FFFFE702A3CC1749FF1F1309C99E4B
:102420003E8483470900918B9DCFB7E4040083A7C6
:10243000041D829783A7441C1745FF1F1305459D64
:10244000829783A7841C81461746FF1F0346469E3A
:1024500081450145829721C583470900ED9B1747B8
:10246000FF1F2303F79A8347040093F7F70F85CBE9
:1024700091471747FF1F2329F79C97000000E7802B
:1024800080EB97000000E78040EFB7E70400BC4F07
:10249000414691451745FF1F0345459A829717030B
:1024A000FFFF670003C682801703FFFFE70223C315
:1024B0008D4741116306F504C5476308F50285475A
:1024C0006310F5029747FF1F2384A798B7E704001E
:1024D000BC4B930500101745FF1F034525968297B7
:1024E00041011703FFFF6700C3C185471747FF1F5F
:1024F0002300F796B7E70400BC4B93050020E1BF2B
:102500009747FF1F93870793D44B1147638DE600CE
:10251000B7E7040083A7071D8297B7E70400BC4B09
:10252000930500044DBF05491747FF1F232E279130
:1025300083C7070032C62E8493F7F70FD5D3B7E4CD
:10254000040083A7041D7D141374F40F8297E376AF
:1025500089FCB245994703C61500E3F0C7FCFC446B
:1025600009061745FF1F1305E58E8297BC489305A2
:1025700000081745FF1F0345658C829779BF170335
:10258000FFFFE702C3B51747FF1F1307A78A40479E
:10259000184B1C409746FF1F23A4F68A6316E400DD
:1025A0001747FF1F2320F78A130584FE9790FFFF2C
:1025B000E78060A6035564FF9780FFFFE780E06E29
:1025C00097A0FFFFE78060D01703FFFF670063B3AA
:1025D0001703FFFFE702A3B09747FF1F9387878585
:1025E000D84BDC4789C797000000E78080F9854712
:1025F0001747FF1F232AF7849737FF1F9387077515
:102600009C43930500021745FF1F0345258383C79D
:1026100087031747FF1F230BF782B7E70400BC4B64
:1026200082971703FFFF6700C3AD9747FF1F23A5DE
:10263000A78082801703FFFFE702C3A837E40400E6
:102640007C4CA1451735FF1F0345457F82977C4889
:10265000A1451735FF1F0345657E9734FF1F9384FF
:10266000647D8297DC4489EB97000000E78080D985
:102670001703FFFF670043A803D567FF9780FFFF9D
:10268000E780A062AA896DD1D84891476310F7020C
:102690007C4C91451735FF1F0345457A82977C484E
:1026A00091451735FF1F03456579829703A94901B5
:1026B00003D409018947B7E904001737FF1F232511
:1026C000F77883A7091D21044204829783C78401F8
:1026D0001715FF1F130585E761191717FF1FA307BC
:1026E000F7E683A7491C418082979737FF1F238114
:1026F000077683A7C91C814609469375F40F4A855E
:10270000829711E99747FF1F83C7C78489C797003E
:10271000FF1FE780204EB7E70400BC4F2146A145CC
:102720001735FF1F03458571829799B71703FFFF80
:10273000E702E39A93F7052001112E8481CF9700D9
:102740000000E78020E91345042005611703FFFF1F
:102750006700239B93F70510A9CF9734FF1F93843D
:10276000646DDC4897000000E78020C11737FF1F29
:102770001307C75D184383C78401034787036318A2
:10278000F700DC4489C797000000E78080DF8547B9
:102790001737FF1F232AF76AB7E70400BC4B9305DE
:1027A00000021735FF1F0345656982971345041022
:1027B00069BF93F70508BDC79737FF1F83C79769A0
:1027C000E91719469735FF1F9385E5681305D10072
:1027D00093F4F70F1739FF1F0349C96797C000002B
:1027E000E780404093970401C1831737FF1F130709
:1027F000E766231DF100231CF1009737FF1F938725
:1028000067633ACE3ACAD8432306010009CBDC43BA
:102810009315890154080D46E18568008297134598
:10282000040825B793F72500A5C39737FF1F9387A3
:102830006760D84B89476306F7029737FF1F83C746
:10284000A75C13F7270011EF918B99CFB7E704002E
:10285000BC4F1306000A89451735FF1F0345055E67
:10286000829713452400D5B59737FF1F9387074EEE
:102870009C4383C787031737FF1F2309F75C970023
:102880000000E78060DBF1BF93F7050281CB970082
:102890000000E78060DA1345040245BD93F7850028
:1028A00081CB97000000E780E0D21345840071BD22
:1028B00093F7150081CB97000000E780A0B4134583
:1028C000140061B593F7450081CB97000000E780C5
:1028D00060B31345440095BD93F7050495C397373E
:1028E000FF1F83C7275591CB97000000E780A0A466
:1028F00091471737FF1F2329F75413450404B1B537
:1029000093F705010145E38207E49737FF1F93879B
:102910006752D84B91476310F7049737FF1F93878F
:10292000A74E9C4313D727008583D98F858B91E7CA
:10293000B7E7040083A7071D8297B7E70400FC4FA1
:1029400091451735FF1F0345654F82978547173718
:10295000FF1F232BF74E13450401C5BB9737FF1FFD
:10296000238AA75E828017F3FEFFE702437797373B
:10297000FF1F23A7074C9737FF1F23A5074C854749
:102980001734FF1F1304843C1737FF1F232EF74A09
:102990001C4083C787031737FF1F2309F74A979007
:1029A000FFFFE780A08F29C59717FF1F23A4A7BAB1
:1029B0001C40170500001305A5D783C787031737E9
:1029C000FF1F2305F7481717FF1FA301F7B8973715
:1029D000FF1FA3810746B7E7040083A70708829774
:1029E0009737FF1F238CA74417F3FEFF670063711F
:1029F000B7C7898E938767ED1717FF1F232CF7B48E
:102A000045BF1737FF1F0347E742795555E797370B
:102A1000FF1F9387274203C7170005079736FF1F3D
:102A2000A38AE64003C717008D463377D70297364F
:102A3000FF1FA381E64083C617001737FF1F130748
:102A4000E730184393F6F60FA9EE8347870317374D
:102A5000FF1F230DF73E85471737FF1F230CF73C59
:102A60009737FF1F9387473A9C430145998BA9E706
:102A700017F3FEFFE702A36637E404007C48C14574
:102A80001735FF1F0345853B82973C488545173521
:102A9000FF1F0345A53A8297014517F3FEFF670024
:102AA000436683C7170085466395F60083479703FF
:102AB00079BF8347A70361BF82809737FF1F83C712
:102AC0006737A1CF17F3FEFFE702636137E4040025
:102AD0009737FF1F238007367C4885451735FF1F32
:102AE0000345C53582977C4C91451735FF1F03453B
:102AF000E53482977C4891451735FF1F034505341F
:102B000082973C48C1451735FF1F034525338297FF
:102B1000014517F3FEFF6700C35E7955828017F306
:102B2000FEFFE702C35B2A84035565FF9780FFFF22
:102B3000E780A0179737FF1F9387C72FD847BE841A
:102B40001DEF9790FFFFE78080779C4823200400CB
:102B50009DEB9737FF1F23A7872E9737FF1F23A1D2
:102B6000872EB7E70400BC4B89451735FF1F034587
:102B7000E52C8297014517F3FEFF67008358630A2F
:102B80008700184375BF80C39737FF1F23AC872A80
:102B9000C9BF7955CDB717F3FEFFE7024354973706
:102BA000FF1F9387673B88432326050023240500E6
:102BB000510597A00000E780C03317F3FEFF6700C0
:102BC000435417F3FEFFE70283511734FF1F13042A
:102BD000A4381C40411199CF9C472302B5002AC656
:102BE0001CC197000000E78040FB1C409C4B99C330
:102BF00032458297410117F3FEFF6700835017F3B8
